:020000040000FA
:040000006FD00400B9
:101000006F009044000000000000000090200020CD
:10101000A4220020A9BDF9F55C23002000000000F7
:10102000000000005C230020902000200000000051
:101030000000000090200020000000009020002010
:101040000000000090200020902000209020002030
:101050009020002090200020B82B0020902000201D
:10106000000000009020002090200020EC230020B1
:1010700090200020C22300209020002090200020FB
:101080009020002090200020902000209020002020
:101090009020002001A04111B7170040985F3AC688
:1010A000945F3247E39CE6FE3245410182800111A4
:1010B00013078008F337078093F787083EC20100C3
:1010C0000100B7170040930570052380B70413068D
:1010D00080FA2380C7040100010083C6B70493F699
:1010E000F60DA385D704238007049246F3A6068055
:1010F0000100010093760502D5CEF336078093F602
:10110000860836C4010001002380B7042380C70489
:1011100001000100B70614007D89558D88C70100C4
:1011200001000100010023800704A246F3A6068007
:101130000100010073370780137787083AC6010062
:1011400001002380B7042380C704010001000100CF
:1011500001003727004093061005A303D7802380A2
:101160000704B247F3A70780010001009307800836
:10117000F3B7078093F787083ECE01000100B71749
:101180000040130770052380E704130780FA2380CB
:10119000E7040100010003C7B70413670708A3852C
:1011A000E70423800704F247F3A70780010001004A
:1011B0000561828093760504BDC6F336078093F6F9
:1011C000860836C8010001002380B7042380C704C5
:1011D00001000100B7061400938606047D89558D31
:1011E00088C7010001000100010023800704C246F6
:1011F000F3A6068001000100733707801377870884
:101200003ACA010001002380B7042380C70401000B
:1012100001003727004093062005A303D7802380D1
:101220000704D24781B773370780137787083ACC12
:10123000010001002380B7042380C70401000100DE
:1012400098471367070C98C723800704E24719BF24
:101250000111814601468145114506CE6D24930753
:101260008008F3B7078093F787083EC601000100A6
:10127000B7170040130770052380E704130780FAAF
:101280002380E7040100010003C767041367170008
:101290002383E70423800704B247F3A707800100F4
:1012A0000100F2400561828041118146014681457D
:1012B0001145912C13078008F337078093F78708AF
:1012C0003EC401000100B7170040130670052380DB
:1012D000C704930680FA2380D70401000100FD555E
:1012E0002396B70223800704A245F3A505800100D9
:1012F000010073370780137787083AC601000100A1
:101300002380C7042380D7040100010003C76704BA
:10131000136717002383E70423800704B247F3A76A
:1013200007800100010001A0BD473305F50201005F
:101330007D1575FD8280411122C426C206C6AA848D
:10134000014463179400B2402244924441018280D8
:1013500005041305803E4204C13F4180DDB7000013
:101360009305000273A04580824573901534924026
:101370002242B2424243D2436244F2440255925561
:101380002256B2564257D2576258F25806499649E9
:10139000264AB64A464BD64B664CF64C065D965DE1
:1013A000265EB65E465FD65F09617300203041114C
:1013B000B7170040985F3AC6945F3247E39CE6FE59
:1013C000324541018280B71700401307000323888C
:1013D000E7028547171700002326F7F47300203033
:1013E000411122C406C6370400201C408297F5BF75
:1013F00037370040834747009146BD8B6389D7004C
:1014000099466394D700834757407300203097165E
:10141000000083C6F6F39387160017160000A30991
:10142000F6F203478700973700009387E75CB6978B
:101430002380E700B7E70400BC4F0946894517152C
:1014400000000345C5E98297C9B723030480154707
:101450002303E48001002302A48082808307648048
:10146000E3CE07FE23030480828083076480E3CEFB
:1014700007FE03454480828083076480E3CE07FE35
:101480002302A4808280411126C44AC24EC006C6EF
:101490001377F50BAD47AA892E8995446306F700AB
:1014A00019456537653F8D444E854537FD59FD1417
:1014B00063983401B240A2441249824941018280BA
:1014C000135509011375F50F453F2209CDB70111D9
:1014D00026CC06CEB704080051371545BD37713705
:1014E00069372AC6A53F32459377150089EB136506
:1014F00015001375F50FF240E24405618280FD147A
:10150000E9FC0145CDBF397126DC4ADA4ED852D606
:1015100056D45AD25ED006DE62CE66CCB7E700E083
:101520007D5783AA070022C603AA470023A0E71815
:1015300023A2E718B7170040130770052380E704BC
:10154000130780FA2380E70483C74704930B75FFD2
:10155000B684E20793FBFB0F8546AA892E8B32895E
:1015600037240040E187015763FA76016308D5000C
:101570008946130700026313D5000157D98F93F7EB
:10158000F70FB71C00402382FC0411472303E480BB
:101590001305F00F5D3D094CD135636D7C11B70526
:1015A0000700DA9537870700795563F2E504B387BA
:1015B0009500636EF702370B0800A94733EB65010E
:1015C0006399F90689E48144513D26850DA0DA85A9
:1015D0000945553D05090345F9FFFD14050B693D16
:1015E00081C49377FB0FFDF7DD3569FD7D55B71796
:1015F0000040130770052380E704130780FA238057
:10160000E70403C74704418B2382E704F250B7E79E
:1016100000E023A0571123A24711E254324452594B
:10162000C259325AA25A125B825B724CE24C21615F
:101630008280A5476395F90685691309F00FB30603
:101640009900B3742B01B6941349F9FFB374990050
:10165000856B33796901416B9387F9FFB3F72701F4
:1016600099E363FC340193D94900C147E3E637FFAE
:1016700099BF0569C1697D19D9B71305800D6388C4
:101680006901130500026384790113051008CA85F6
:10169000DD3B353D21DD4E99B3843441D9B7DA8540
:1016A0002D45D533CA94E30099F205097D3BA30F7C
:1016B000A9FED5BF9387F9FF93F7F70F6361FC0C81
:1016C00083C71C0413073008631FF704370708009B
:1016D000636BEB04B3079B00B706100063F5D704F8
:1016E000334BEB0089476393F9068980D549E38C36
:1016F00004ECDA850945413B11090327C9FF9147ED
:101700002320E48003076480E34E07FE2303348133
:10171000FD17EDFBFD14110B81C49377FB0FE9FF5F
:101720007D3371F5E1B5B717004003C75704B7071C
:1017300008001377070219E3B78707007955E378A4
:10174000FBEA33079B00E3FFE7F855B58547E382E3
:10175000F9F2DA852D45053B9389F4FFE38504E62C
:10176000293393F7390091EB83260480032709007E
:1017700093074900E39AE6E43E89CE84F1BFB5477A
:101780006396F9001305900BC93135BDB1471305B8
:10179000B00AE38BF9FE99476391F904B705080095
:1017A000B365BB002D45C53181448D4BA1497539C9
:1017B00063967401832704802320F9008504E3984D
:1017C00034FF8327048013172B016355070023126E
:1017D000F900D5BB2322F900FDB39D476399F902B7
:1017E00081451305B0044531BD442320090023225F
:1017F0000900FD599D3993F77400CA9703C7070084
:10180000FD14398D2380A700E39634FF6DBBA147FB
:101810006392F9046D398144630D0B008D47930485
:10182000C0036308FB009304000563048B01930469
:1018300040041375C507E30895D81945393139397E
:101840000545213126850D3909453D314931E31CD6
:1018500005D669BB91476399F90013056006F53613
:10186000F53E130590090DB7E38F09D4F154A9BBD8
:10187000BD660147173600001306C644938606A6C8
:1018800085458347060093F7F70F91C382800507CC
:10189000E3F9E6FE973700002386B742DDB77D16F1
:1018A0006206618693178601E18763D407000145CC
:1018B0008280931726003307F500AE9718439C43A8
:1018C00063E7E7007D16E37FF7FC7D5582800545E1
:1018D0008280FD15E205E18513978501618793F705
:1018E000F50F63480700FD15139725002A97584305
:1018F00065D7138517006205618582803308B502BC
:101900001C4283A80600B335B502C29733B5070160
:10191000AE98469585486367B5006394A50063E378
:10192000070181480C43C6950CC388C21CC2828043
:1019300081471397870161876343B70082801397BC
:1019400027002A97232007008507E5B7814701472D
:1019500093968701E18663C5B60013351700828030
:1019600093962700AA9694428507558FD5B793D7AB
:1019700055408A07AA979C4305453315B5007D8DD0
:10198000828017F3FFDFE702C33B2A84993705C53E
:10199000931725003E940327C4FF814711EB7D1563
:1019A00016053E954205418517F3FFDF6700A33B0F
:1019B00005838507E5B70145C5BF814713978701B3
:1019C00061876343C700828013972700B386E500D1
:1019D00094422A97850714C3D5B77D16620661869F
:1019E000014793178601E18763D507001335170078
:1019F000828093172600B306F500AE9794429C436D
:101A00007D16B58F5D8FF1BF8A05AA950147636387
:101A1000B500828083A6C5FFF11593D71600D98F34
:101A20009CC11397F601E5B72A8301480147014598
:101A30006343D7008280B387050183A80700B307FB
:101A400006019C43C697AA976384F80033B5170133
:101A50000507B3080301620723A0F8006187110896
:101A6000C1BF2A8301478147014563C3D7008280F4
:101A70003388E50083280800330EE600032E0E00AD
:101A80003388A8403308C8416384080133B508018E
:101A90008507B308E300E20723A00801E1871107E7
:101AA000E9B717F3FFDFE702C3290111B286B28459
:101AB0002E86AA850A8575372A84A6850A857935F2
:101AC00033348000060413351500018D056117F3CA
:101AD000FFDF6700432917F3FFDFE702032441110B
:101AE000AA89AE8A328BB68402C202C402C60144FD
:101AF000131C8401135C8C4163499C02939B14006A
:101B0000FD1B0549138CF4FFF15C33048901620469
:101B10006184634D740592478E04CE9423AEF4FE27
:101B2000410117F3FFDF6700C32213192400B30B31
:101B30002B01014A93172A00D69783A50B008843EF
:101B40007800340050005D3B050A93178A01E18755
:101B5000F11BE351FCFE92474E9905042320F90046
:101B6000A2473EC2B24702C63EC459B7131A890102
:101B7000135A8A41131D240093178A01E18763CF0A
:101B8000970092470A044E941CC0A2470509137996
:101B9000F90F3EC2B24702C63EC485BFB3079A03DF
:101BA00013152A0056950841780034005000050AA4
:101BB000EA97DA978C439933C1B70000197106C2CE
:101BC00012C416C61AC81ECA22CC26CE2AD02ED2BD
:101BD00032D436D63AD83EDA42DC46DECAC0CEC26D
:101BE000D2C4D6C6DAC8DECAE2CCE6CEEAD0EED29D
:101BF000F2D4F6D6FAD8FEDA97050000938505727E
:101C00008841E700050092402242B2424243D2435B
:101C10006244F244025592552256B2564257D25768
:101C20006258F25806499649264AB64A464BD64B60
:101C3000664CF64C065D965D265EB65E465FD65FE8
:101C40000961730020300000972100209381813BBF
:101C500017510020130101BB17F5FFFF1305C53A0B
:101C6000970500209385053A171600201306C6FD38
:101C700063FAC5008322050023A0550011059105D4
:101C8000E3EAC5FE17A501001305C54F971500200F
:101C90009385C5FB171600201306C66563FAC500B9
:101CA0008322050023A0550011059105E3EAC5FE36
:101CB0001715002013050564974500209385854C72
:101CC0006377B500232005001105E36DB5FEFD42E5
:101CD000739002BC8D4273904280B72200009382C1
:101CE000828873900230970200209382A23193E29F
:101CF00032007390523097420000938202F1739049
:101D000012346FC0E42F73002030397101436EC666
:101D100019A0397141536AC866CA62CC5ECE19A057
:101D2000397101535AD056D252D44ED64AD826DAF7
:101D300022DC06DE33016140828241114AC026C2A4
:101D400022C406C68282B24D4101024D924C224C01
:101D5000B24B4101024B924A224AB2494101024927
:101D600092442244B240410182803D432A876373FA
:101D7000C3029377F700BDEFADE5937606FF3D8A8A
:101D8000BA960CC34CC30CC74CC74107E36BD7FED4
:101D900011E28280B306C3408A069702000096963D
:101DA0006780A6002307B700A306B7002306B70085
:101DB000A305B7002305B700A304B7002304B700A9
:101DC000A303B7002303B700A302B7002302B700A1
:101DD000A301B7002301B700A300B7002300B70099
:101DE000828093F5F50F93968500D58D9396050126
:101DF000D58D61B79396270097020000969686824C
:101E0000E78086FA9680C1171D8F3E96E374C3F86B
:101E1000A5B73367B500FD530D8B79E7B7877F7F93
:101E20009387F7F710419441B372F6003363F600DD
:101E3000BE92B3E262006397720C6318D6065041FB
:101E4000D441B372F6003363F600BE92B3E262008F
:101E50006398720A631BD60410459445B372F6006A
:101E60003363F600BE92B3E262006391720A631EAE
:101E7000D6025045D445B372F6003363F600BE92E5
:101E8000B3E26200639A72086311D6021049944962
:101E9000B372F6003363F600BE92B3E2620063935E
:101EA00072085105D105E30FD6F613170601939773
:101EB0000601631CF7001357060193D7060133058B
:101EC000F7409375F50F91E982804183C183330513
:101ED000F7409375F50F91E182801377F70F93F731
:101EE000F70F3305F74082800346050083C60500DF
:101EF000050585056313D60065FA3305D640828053
:101F000011059105E312D6FE014582802105A10548
:101F1000E31CD6FC014582803105B105E316D6FCF1
:101F2000014582804105C105E310D6FC0145828050
:101F3000B717004003C777051377E70FA38BE704B4
:101F4000130700F8A38DE7043D47238CE70413072C
:101F50005003A38CE70403C7A7051377D70F238D7E
:101F6000E7048280B717004003C7E7020D894111DB
:101F70001377C70F498F93068008F3B6068093F650
:101F8000860836C601000100930670052380D70439
:101F9000930680FA2380D704010001002387E7021B
:101FA00023800704B247F3A7078001000100410125
:101FB000828041112A83014E930E407E130F001937
:101FC000930F400663E56E12930800191303400651
:101FD000B3781503854E0D4FA14F337365020D89FC
:101FE0001335150063EFBE121308F6FF7946729899
:101FF0004208135808013307C70213D61700BE075B
:1020000032976146B3F6C60213068070B386C602E5
:102010003697A166F58F42075D8FB716004083C7DC
:10202000F60293F70708A303F1000346710083C784
:10203000F60293F70708E394C7FE83477100B716CB
:10204000004093F7F70F6388071293078008F3B7F0
:10205000078093F787083EC401000100B7170040CE
:10206000930670052380D704930680FA2380D70453
:102070000100010023AA070383C6170393E606089D
:10208000A388D70223800704A247F3A70780010093
:1020900001001166B71700407D16D45BC85F9385B9
:1020A0004703A98EF18EF5FA93068008F3B60680F1
:1020B00093F6860836C6010001009306700523805A
:1020C000D704930680FA2380D7040100010098C149
:1020D00003C7170313670704A388E70223800704D5
:1020E000B247F3A7078001000100410182807D1300
:1020F0003368E3039308E016630E08003368F303C4
:102100009308D016630808009378330093B818003A
:102110009388D81633081E01131E0801135E0E01A2
:1021200055B56393E50305486386080001486303DA
:1021300003002A8871087298FD15131E0801C20554
:10214000135E0E01C18179BD13F8150063F4BF0061
:102150007908D5B713381800E5BF83C7F60293F79F
:102160000708A303F1000346710083C7F60293F743
:102170000708E394C7FE8347710093F7F70FF1DF79
:10218000E9B531714AD966CB06DF22DD26DB4ED7B1
:1021900052D556D35AD15ECF62CD6AC96EC7AA8CCA
:1021A00002D8EF00901C2A8993078008F3B70780B4
:1021B00093F787083EDA01000100B71700401307C4
:1021C00070052380E704130780FA2380E7040100E9
:1021D000010003C7F7021377770FA387E70203C74E
:1021E000F70213678700A387E70223800704D2570B
:1021F000F3A70780010001000545AD33130780C137
:102200003347E902116A93070AE893065002BD6951
:10221000930BA004814A014B1304800893047005BA
:102220007D1AB347F9023307D7023EC0FD873ECC83
:10223000938709A69309803E3347F7023AC27D8708
:102240003AC4334739038549B399990193D9394041
:10225000B306D702B30B7703B3C6F602B3CBFB02C8
:1022600036C6FD8636C893D6FB4136CEB7460F003C
:10227000938606243349D9028566938606FAB39677
:102280009601B389E902130760553309D902930611
:102290000010B389E9023349D902B3C9F902931690
:1022A000390036CA37190040FD8636D0930D09042F
:1022B00093D7F9413ED2F336048093F6860836DC94
:1022C00001000100930770052380FD00930680FA4A
:1022D0002380DD00010001008346390593F6860F57
:1022E000A309D9048346390593E61600A309D90446
:1022F00023800D00E256F3A6068001000100130CB6
:1023000080FA116DF336048093F6860836DE0100FC
:102310000100930770052380FD0023808D010100DB
:10232000010083463905216693E60602A309D90414
:1023300083560905B3E6A6012318D9048356090577
:10234000D18E2318D90423800D00F256F3A60680FF
:10235000010001008346390593F60602638A0618D8
:1023600003463905218A6DDE0818EF001004733624
:10237000048013768608B2C20100010023809D000C
:1023800023808D0101000100B717004003C6370507
:102390001376F60DA389C70403C637051366060234
:1023A000A389C704835609052166B3E6A60123184D
:1023B000D90483560905D18E2318D90423800D0032
:1023C0009646F3A60680010001008346390593F680
:1023D00006026386061483463905A18AEDFE97003E
:1023E0000020E78040CBAA8636D497000020E78003
:1023F00080CAA256E30AD5FE835609054255B3E6C4
:10240000A6012318D904C12783463905A18AEDDE28
:10241000035609058346290582473376CA00B30669
:10242000DA0293D5F641B296B388F640E24733B864
:10243000C6002E983308F840A247B3B616013308F9
:10244000D84063C70701631DF800924763FA17017C
:10245000C247634DF80E63950701B24763E8F80E73
:10246000894663E7660FF2469315180013D3F80107
:102470005E8613951800B365B30042D646D4EF606C
:1024800081363258050B137BFB0F63470001631243
:102490000838A258638F083613081500B336A80011
:1024A000B69513D6F5013298B336C800AE961358D8
:1024B0001800FE06B3E6060173360480137686081C
:1024C000B2C60100010023809D0023808D01010020
:1024D00001000356C902B296C206C1822316D90270
:1024E00023800D00B646F3A606800100010019BD49
:1024F000F336048093F68608B6C0010001002380FD
:102500009D0023808D01010001008346390593E67B
:102510000602A309D90423800D00864605BDF336C3
:10252000048093F68608B6C40100010023809D0054
:1025300023808D01010001008346390593E60602E0
:10254000A309D90423800D00A646A5BDE30D0BF019
:10255000F336048093F68608B6C80100010093069E
:1025600080FA23809D002380DD0001000100834666
:10257000390593F5FC0F93F6860FA309D90483461A
:102580003905CD8EA309D90423800D00C646F3A6D4
:10259000068001000100130580FA03463905930601
:1025A00039051D8A631496297336048013768608CC
:1025B000B2CC01000100130680FA23809D00238025
:1025C000CD000100010003C606001376F60D23803E
:1025D000C60003C60600136606022380C6008356A3
:1025E00009051166D18E2318D90483560905216681
:1025F000D18E2318D90423800D00E646F3A6068069
:1026000001000100130680FA8346390593F606029D
:102610006388062483463905130C3905A18AFDDA3F
:1026200008186123F336048093F68608B6D00100BB
:102630000100930680FA23809D002380DD000100C5
:10264000010083460C00116693F6F60D2300DC00B2
:1026500083460C0093E606022300DC00835609053E
:10266000D18E2318D904835609052166D18E2318EB
:10267000D90423800D008656F3A6068001000100D0
:10268000130680FA8346390593F606026385062011
:1026900083463905A18AEDFE97000020E780A09FC0
:1026A0002A8C97000020E780009FE30C85FF83566B
:1026B000090511664255D18E2318D9042923834672
:1026C000390513063905A18AFDDAF336048093F63D
:1026D0008608B6D401000100930680FA23809D008D
:1026E0002380DD00010001008346060093F6F60D0D
:1026F0002300D60023800D00A656F3A60680010015
:1027000001008356090503462905D247B376DA004E
:102710003306CA021305800C9355F6413696330DE5
:10272000F6408257333CD6002E9C3336A601330C3C
:10273000FC40330CCC403308850392564E86B335AB
:10274000A5033305A503C295EF60E1096346800147
:10275000631E0C16630C0D16130615003335A60008
:102760002E959356F5013696B335D600AA959396D5
:10277000F50105828585D18E6346B000639D051AFB
:10278000638B061A0356C90215823305D600333609
:10279000C500B2956348B000639105241306F00F9D
:1027A000637DA622894663F3561593078008F3B725
:1027B000078093F78708BED6010001003717004055
:1027C000930770052300F704930780FA2300F704AA
:1027D000010001008356C70289678117D58FC207A0
:1027E000C1832316F70223000704B657F3A7078017
:1027F00001000100FA506A54DA544A59BA592A5A67
:102800009A5A0A5BFA4B6A4CDA4C4A4DBA4D296126
:1028100082801308F5FF3335A800FD152E95135659
:10282000F5013298B336C800AA9651B1F336048048
:1028300093F68608B6CA0100010023809D0023801C
:10284000AD000100010083463905CD8EA309D904EE
:1028500023800D00D646F3A606800100010035BB9B
:10286000F336048093F68608B6CE0100010023807B
:102870009D002380CD00010001008346390593E6C9
:102880000602A309D90423800D00F646F3A60680AC
:102890000100010095BBF336048093F68608B6D29A
:1028A0000100010023809D002380CD000100010074
:1028B0008346390593E60602A309D90423800D0057
:1028C0009656F3A60680010001006DBB9306F5FF46
:1028D00033B5A600FD152E959355F501AE96B3B50B
:1028E000B600AA951396F501858269B5F336048082
:1028F00093F68608B6D801000100930680FA23807B
:102900009D002380DD00010001008356C902056699
:10291000011693F6F60FD18EC206C1822316D90294
:1029200023800D00C656F3A6068001000100850A2B
:1029300093FAFA0F49B233E6B60045C20356C9020C
:102940003305D0403338A000B305B040B38505410E
:1029500015826345B000D1E16371A608894663F032
:10296000560593078008F3B7078093F78708BEDA08
:1029700001000100B7170040130770052380E7042A
:10298000130780FA2380E7040100010003D7C70280
:102990007D8B2396E70223800704D65781BDF3364B
:1029A000048093F68608B6DC01000100930680FAE5
:1029B00023809D002380DD00010001008356C902B1
:1029C0000566011693F6F60FD18EC206C182231654
:1029D000D90223800D00E656B9B793078008F3B7F4
:1029E000078093F78708BEDE01000100371700401B
:1029F000930770052300F704930780FA2300F70478
:102A0000010001000356C70293975600B297C20710
:102A1000C1832316F70223000704F657C1BB914771
:102A200063EEB70217870100130787AC8A05BA95D2
:102A30009C41BA978287B717004003A7470B1345FD
:102A4000F5FF698F23AAE70A03A7070B698F23A85D
:102A5000E70A03A7070A798D23A0A70A8280B71780
:102A6000004083A6470B1347F5FFF98E23AAD70A28
:102A700083A6070B558D23A8A70A83A6070A758F7F
:102A800023A0E70A8280B717004003A7470B498FAE
:102A900023AAE70A03A7070B1345F5FF45BFB7179E
:102AA000004083A6470B1347F5FF758F23AAE70A5B
:102AB00003A7070A598D4DB7B717004003A7470B67
:102AC000498FEDB7914763EEB702178701001307EF
:102AD00067A38A05BA959C41BA978287B7170040C9
:102AE00003A7470D1345F5FF698F23AAE70C03A73A
:102AF000070D698F23A8E70C03A7070C798D23A086
:102B0000A70C8280B717004083A6470D1347F5FF37
:102B1000F98E23AAD70C83A6070D558D23A8A70CE1
:102B200083A6070C758F23A0E70C8280B71700409F
:102B300003A7470D498F23AAE70C03A7070D1345E9
:102B4000F5FF45BFB717004083A6470D1347F5FFB4
:102B5000758F23AAE70C03A7070C598D4DB7B7173C
:102B6000004003A7470D498FEDB7B71700408847CE
:102B7000420541819377050491EB9377F501375531
:102B8000E801130505803345F50282809377050C33
:102B9000130700046397E7009377F50137459C1C02
:102BA000CDB72165130505D0828037E700E01C43CF
:102BB0005443A183E206D58F1CC1FD572320F7188B
:102BC0002322F718828013178500B7E700E023A0BF
:102BD000E710618123A2A7108280B7F700E0884741
:102BE000CC478280814737370040A14663C4C70085
:102BF000328582800345B740E38EA6FE3385F5001B
:102C00000345050085072304A740CDB7970700209B
:102C10009387476A9C43173700201307A7563E95B2
:102C2000636EE500174700201307C79D6368A70080
:102C3000170700202320A7683E858280FD57EDBF3F
:102C4000411122C406C62A840D372947B307E5027D
:102C5000B2408D83B3D7870222449507B3D7E702EA
:102C600037370040C207C1832316F7004101828035
:102C7000716541111305052006C6D937B7370040E5
:102C8000130770F82381E7000D47A381E7001307BE
:102C90000004A380E70005472387E700B240410115
:102CA000828037370040834727001A0593F7F703E0
:102CB000C98F93F7F70F2301F7008280B7370040E1
:102CC00003C7170019C9D98DA380B70003C7070030
:102CD000136787002380E700828093C5F5FFF98D95
:102CE000A380B7008280B73700402147B736004045
:102CF00091E1828003C6B700E30CC7FE05050346D9
:102D0000F5FFFD15C2052384C600C181D5B7411169
:102D100022C406C62A84913D2947B307E502B24082
:102D20008D83B3D7870222449507B3D7E70237379D
:102D30000040C207C1832316F740410182807165BC
:102D400041111305052006C6D937B73700401307D0
:102D500070F82381E7400D47A381E7401307000483
:102D6000A380E74005472387E740B24041018280C6
:102D7000CC41411106C6328503C6150083C5050046
:102D800022064D8E42068D654186138875A2630C1E
:102D90000611634BC804138845A26300060D634AFD
:102DA000C800938535A26301B60823900600294622
:102DB0004DA0138855A26305060D938565A2E31601
:102DC000B6FE8D451D4663E6E5081146198E63F390
:102DD000C7003E86B7E704002390C600FC479795DE
:102DE0000100938525349DA0138895A263030611E5
:102DF000634E060D1388A5A263000613938505A5EF
:102E0000E315B6FA99451D4663E5E504198E63F3AB
:102E1000C7003E86B7E704002390C600FC4797052D
:102E200000209385A5491DA09D451D4663E3E5024D
:102E30002146198E63F3C7003E86B7E70400FC47BE
:102E40002390C600970500209385C54ABA958297BE
:102E50000146B240328541018280AD451D46E3EA1C
:102E6000E5FE3146198E63F3C7003E86B7E70400DE
:102E70002390C600FC47977501009385A56BF9B7B1
:102E8000B1451D46E3E7E5FC3546198E63F3C700FF
:102E90003E86B7E704002390C600FC479775010003
:102EA0009385456A65B78D451D46E3E4E5FA11460D
:102EB000198E63F3C7003E86B7E704002390C6006F
:102EC000FC47979501009385A52649B78D451D467A
:102ED000E3E1E5F81146198E63F3C7003E86B7E7D4
:102EE00004002390C600FC479795010093850526B2
:102EF000B1BFA5451D46E3EEE5F42946198E63F3FF
:102F0000C7003E86B7E704002390C600FC479775CC
:102F10000100938565611DBFB5451D46E3EBE5F2F4
:102F20003946198E63F3C7003E86B7E70400239045
:102F3000C600FC47977501009385055E01BFB7E7A2
:102F4000040003A3071397060020938626D9414661
:102F5000A54517050020130565CF02832D4559EFC0
:102F600003C5050009476317E50803A8450041119B
:102F700006C6034718003285034608002207416849
:102F8000518F930828FE6308170363E9E8000518CA
:102F9000630307052390060029451DA8130648FE74
:102FA000630BC7021518E31707FF15463E87637BBF
:102FB000F602154705A83E8691C30546B7E704000B
:102FC000FC472390C6004206CC45418282970145CA
:102FD000B240410182801306700F3E876374F60091
:102FE0001307700FB7E704002390E600FC471316A1
:102FF0000701D9BF23900600054582808280416782
:1030000079176304E504411122C406C685472A8462
:10301000639FF500B7E7040022852244B24003A372
:103020008713970500209385A52D410102838947C9
:103030006399F500B7E7040083A7070B85458297DE
:1030400071D9B2402244410182808280797122D4B8
:1030500052CC2E842A8A977501009385E550177506
:1030600001001305255206D63AC626D24AD0B684A8
:1030700032894ECEEF507142A685177501001305B7
:103080006551EF5091412945EF50714583478400C8
:1030900093F70702E1E78349040089470545324772
:1030A0006396F908544083C7160083C60600A2073A
:1030B000D58FC166138616FE638CC7028D16638F8B
:1030C000D7068D669386269029456391D706B7E784
:1030D0000400A285225403A34714B250F249A686E5
:1030E0004A86925402595285624A85474561028355
:1030F0002D450DEF9307700F354563E99702B7E74C
:103100000400FC4748441306700FCA858297814922
:10311000970700209387871F9C43014581CB9C43E1
:1031200091C74E852686CA8582970145B2502254A2
:1031300092540259F249624A456182802D457DF7D9
:103140009307700F3545E3E397FEB7E70400FC47AC
:1031500048441306700FCA8582975DBF2145F9B7B1
:10316000411122C437E404008327841326C2AA84B1
:10317000416506C697050020938585187D158297C1
:103180008327C40A170500001305A5E785888297E1
:1031900095C0032304132244B240924497060020B2
:1031A000938686C54146C545170500201305C5B35E
:1031B00041010283B2402244924401454101828090
:1031C00019C59707002023A3A71401458280454510
:1031D00082801147636AA70A977601009386863733
:1031E0000A0536951841411106C63697AE87B28555
:1031F00002871307700F6145639DE700B7E704007E
:10320000FC471306700F170500201305E51682977B
:103210000145B2404101828005476145E39BE7FEDD
:10322000B7E70400FC470546170500201305050D08
:10323000F9BF1307700F6145E39DE7FCB7E7040092
:10324000FC471306700F1705002013056522C1B750
:103250001307700F6145E39EE7FAB7E70400FC47E8
:103260001306700F17050020130505304DB71547DD
:103270006145E390E7FAB7E70400FC4715461705F8
:1032800000201305250861B709458280411126C237
:10329000B7E4040083A7C41322C44AC006C62E8420
:1032A000970500209385C5052A898297058905C55C
:1032B00097070020938747A383D7A70BA28503A373
:1032C000440D2310F4002244B24092444A8502493E
:1032D000014641010283B2402244924402494945D9
:1032E000410182809707002023840702970700206E
:1032F00023A20702B717004003A7070CB706C0FFB9
:10330000FD16758F23A0E70C03A7070DB706400035
:10331000558F23A8E70C03A7070C3D9B23A0E70CC0
:1033200003A7070D1367070123A8E70C8280B717CF
:10333000004003A5470C83A7470C5981134515008E
:10334000C18B058999E3136525009707002083C782
:1033500027FC6380A70297070020238BA7FA11C9D7
:1033600097070020938707FB03A30700630303006D
:103370000283828011456FE0DFE0411193962500C2
:10338000AA852D4506C697F0FF1FE780C017B240FB
:10339000014541018280011122CC06CE3714004044
:1033A00026CA4AC84EC652C483447405034AB405AB
:1033B0008349840503499405EFE09FB78347A4053B
:1033C00093F4F40F137AFA0F93E71700230DF40424
:1033D00093F9F90F1379F90FB717004003C7A70541
:1033E000058B6DFF03D5C705A38D4705238C3705D6
:1033F000A38C2705A38B9704F2406244D244424930
:10340000B249224A0561828041119397050122C485
:1034100006C626C2C1872E8463DC0700B7E4040019
:10342000FC54829719C1BC5482972165218D3DA01F
:1034300093F7150013C5150095E393F7250085C78D
:10344000FD35B7E70400BC4F1306000A8945170590
:1034500000200345A5EC829713452400B240224486
:103460009244410182809397250163D50702B7E416
:10347000040083A7C41E8297F53DBC4C37F60200BA
:10348000130606E0896517050020034525E98297A4
:10349000096569BF939715010145E3D107FC1775CD
:1034A00001001305E515EF501114B7E70400BC4FF8
:1034B00013060064916517050020034525E68297F1
:1034C0001165ADB72D71232A9110FD74E98C232C61
:1034D000811023282111232631112A84AE893289B3
:1034E000930600100A86A6852D45232E111097F00D
:1034F000FF1FE780400113154401B7E70400FC47B4
:1035000051810A0513962900CA850A958297A685D6
:1035100085660146254597F0FF1FE780C0FE0A86B5
:10352000A68593060010294597F0FF1FE780A0FDB0
:103530008320C11103248111832441110329011126
:103540008329C11015618280B7F7070003C70701FF
:10355000411106C622C426C24AC0A547631AF70015
:103560009537B2402244924402490145410182808C
:1035700013942500AA843289A286AA85014625458E
:1035800097F0FF1FE78020F8A2864A86A685294586
:1035900097F0FF1FE78020F7E9B71D71A2CC37E451
:1035A00004005C5C485886CE4946977501009385B7
:1035B000A500829701E91775010013052501EF5059
:1035C000910201A0B7F600E0795798CAFD57DCCA0E
:1035D0000567B7E700E023A0E7101306F00290C2EA
:1035E00023A0E71801000100370700201847130641
:1035F000000481459706002023A0E6D24157A38A04
:10360000E7403C440808829797170020938787DE9D
:103610003EC8856713870760231AE1001D673ACC0F
:1036200037070105130707103ACE9387B7D313075F
:10363000B00F2310E1022312F102054797F7FFFFB5
:103640009387E7592301E1023ED8170700001307CB
:1036500007D397070000938747D4B7F50700BAC28E
:103660003EDC17070000130767EE970700009387FB
:10367000A7D081463000E1051945BAC43EDE97F077
:10368000FF1FE78040E818088147994630003E96C2
:103690000346060085070507A30BC700E398D7FE7E
:1036A000C24791C70357410185676373F70001A0C3
:1036B000B7E7040083A7470A08088297AA8501C9CB
:1036C000177501001305C5F1EF50215D01A0F6400B
:1036D000664425618280411126C2B7E4040083A7B5
:1036E000040806C622C417050000130525D28297D8
:1036F00017040020130484C22300A4003128DD36FF
:1037000003450400224403A38405B24092441306F7
:103710000032896541010283797106D622D41307EC
:103720008008F337078093F787083EC20100010045
:10373000B7170040930570052380B704130680FA7D
:103740002380C7040100010083C6F70293F6A60F89
:10375000A387D702238007049246F3A606800100C0
:10376000010073370780137787083AC4010001000E
:103770002380B7042380C7040100010003C7F702B8
:1037800013672700A387E70223800704A247F3A754
:103790000780010001000545EFE0CFFCE13E014755
:1037A00081468147054685451305407EEFE07F80D1
:1037B00037E404003C446800514681458297B707CE
:1037C000C0A83EC8B787E803938707D03ECA97F7DB
:1037D000FF1F9387C7BD3EC67C5868008297B250D2
:1037E00022544561828041119775010093850551EE
:1037F00017750100130505D906C6EF50014A177564
:1038000001001305256AEF504149B24029454101A5
:103810006F50E14C4111977501009385654F177505
:103820000100130525D606C6EF5021471775010084
:1038300013050566EF506146B240294541016F50BE
:10384000014A411122C406C6834705002A849DC34C
:10385000977501009385855117750100130585D271
:10386000EF50A1434C40177501001305E577EF5069
:10387000C1421DA058411DE7977501009385054F72
:1038800017750100130505D0EF5021411775010090
:1038900013050577EF5061402244B24029454101AC
:1038A0006F50E143A1679386D7036311D7029775E1
:1038B00001009385A54B177501001305A5CCEF50AA
:1038C000C13D177501001305A574E9B7ED0797759C
:1038D00001009385A549177501001305A5CA631951
:1038E000F700EF50813B177501001305A5735DB715
:1038F000EF50A13A4C40177501001305A57485BF20
:103900004111977501009385E54117750100130575
:1039100065C706C6EF506138B240294541016F5076
:10392000013C797122D426D24AD02E842A8981453D
:10393000B2844800714606D6EFE02FC397F7FF1F09
:103940009387076BDC4783D70700231421012313D8
:10395000F100EF2090029547A305F1009307401F67
:103960003EC6FD572305A100230AF100EF203013C6
:103970002686A2854800EF203003B250225492548C
:10398000025945618280970700202392079C970780
:103990000020238D079AB7E70400BC47411106C6F3
:1039A000414681451385413D8297EF107067EF10C6
:1039B00010450145EF30201503C7C1259307F00AD4
:1039C000631BF7009307F00889451385C125239EE3
:1039D000F124EF30A03FEF30804F814537050400E0
:1039E0009707002023A0079697070020239A0794A3
:1039F000970700202387079497070020239F0792AB
:103A000097070020239A079297070020239907928F
:103A100097070020239A0792EF20A0370145EF3047
:103A2000A041977501009385653217750100130554
:103A300065B5EF508126177501001305E566EF5057
:103A4000C125B240294541016F506129411122C46D
:103A500006C626C293F715002E84638D070C814697
:103A600017F6FF1F13064656854517050020035518
:103A7000658CEF80500A05C5977501009385C52DAB
:103A800017750100130505B0EF50212117750100CE
:103A9000130545CFEF5061202945EF50412497751C
:103AA00001009385652B177501001305A5ADEF5037
:103AB000C11E17750100130525CEEF50011E2945C3
:103AC000EF50E12117F5FF1F130585525C450547AF
:103AD0002390E700EFF0801A977501009385C527C2
:103AE00017750100130505AAEF50211B177501007A
:103AF0001305C5CBEF50611A2945EF50411E9307BE
:103B000010F8238EF1249707002083D76782A38EB5
:103B1000F1241385C125A1839145238FF124A38F1F
:103B20000124EF30A02A13451400B24022449244ED
:103B30004101828093F72500D1CB1707002003575E
:103B4000278051C397F6FF1F9386C67F94429777CD
:103B500001009387675717F6FF1F0346867E81454E
:103B60001385413DEF407008AA8431CD977501005F
:103B700093854525177501001305C5A0EF50E11188
:103B8000A685177501001305E5C3EF5001112945FE
:103B9000EF50E11497F7FF1F2394077A930710F86B
:103BA000238EF12497F7FF1F83D78778A38EF12404
:103BB000A183238FF12491458D471385C125A38FC0
:103BC000F124EF30A0201345240085B793F745007A
:103BD000B1CF977501009385E51E17750100130598
:103BE000659AEF50810B17750100130565BFEF5003
:103BF000C10A2945EF50A10E930720F8238EF12426
:103C000097F7FF1F83D76773A38EF124A183238FB8
:103C1000F1248547A38FF124EF2060681385C12527
:103C20009145EF30A01A1345440001B793F7850082
:103C30008DCF977501009385E51817750100130561
:103C40006594EF508105177501001305A5BAEF5073
:103C5000C1042945EF50A10897F7FF1F2392076E73
:103C6000EF40900513458400C9B593F70501A5C33E
:103C7000854517F5FF1F0355456CEF00514F9775AC
:103C8000010093852514177501001305A58FEF50CA
:103C9000C10017750100130525B7EF500100294534
:103CA000EF50E103930730F8238EF12497F7FF1FBD
:103CB00083D7A768A38EF1241385C125A1838D45E1
:103CC000238FF124EF30801013450401B9BD93F721
:103CD0000502B5C3977501009385C50E17750100E0
:103CE0001305458AEF40717B17750100130505B474
:103CF000EF40B17A2945EF40917E930740F8238E3B
:103D0000F12497F7FF1F83D72763A38EF124A183A4
:103D1000238FF1248547A38FF12497F7FF1F239D5D
:103D20000760EF20C0571385C1259145EF30000A89
:103D300013450402DDBB93F70504CDC79775010059
:103D400093854508177501001305C583EF40F1748D
:103D500017750100130505AFEF4031742945EF4099
:103D6000117883C7C1251307700A6388E704130716
:103D7000800A6386E7061307600A6397E7029307E2
:103D800060F8238EF12497F7FF1F83D7475BA38E3C
:103D9000F124A183238FF1248547A383F126B14524
:103DA0001385C125EF308002EF20604F13450404D6
:103DB00097F7FF1F239507588DBB930770F8238E45
:103DC000F12497F7FF1F83D78757A38EF124A18390
:103DD000238FF1248547A380F1269945D1B7930716
:103DE00080F8F1BF93F705080145E38007D4977584
:103DF0000100938525FD176501001305A578EF40A7
:103E0000D16917750100130565A5EF4011692945B2
:103E1000EF40F16C9307A0F8238EF12497F7FF1F72
:103E200083D78752A38EF124A183238FF124854762
:103E3000A38FF12497F7FF1F23980750EF20204608
:103E40001385C1259145EF20707813450408F1B919
:103E5000411122C497750100938585F22A84176564
:103E600001001305257206C6EF4031634C401775FB
:103E700001001305E514EF4051622945EF4031661A
:103E8000034704009307F00F6319F70297750100C9
:103E9000938505EF176501001305C56EEF40F15FCF
:103EA0004C40177501001305A512EF40115F224425
:103EB000B240294541016F409162B2402244410124
:103EC000828085CD411122C4176501001305856BE1
:103ED0002E84977501009385A5E506C6EF40F15B3A
:103EE000A285177501001305E519EF40115B224407
:103EF000B240294541016F40915E8280411122C448
:103F000026C22E84AA8497750100938525E3176540
:103F100001001305256706C6EF40315817750100EB
:103F200013050517EF4071572945EF40515B977511
:103F300001009385A5E097F7FF1F239D973E176526
:103F4000010013052564854497F7FF1F2392873EE0
:103F500097F7FF1F239F973C97F7FF1F2399873EF3
:103F6000EF40B15397F5FF1F83D5653E17750100EC
:103F700013058512EF4071522945EF40515697F7CE
:103F8000FF1F2385973CEF1080672285EF20B03715
:103F90000545EF20706A97F7FF1F93876705DC4799
:103FA00003D70700C167FD176312F7022244B7E782
:103FB0000400B240924403A3870517F5FF1F034591
:103FC00065361306000A854541010283B24022444A
:103FD000924441018280011122CC37E404005C5CF0
:103FE00006CE26CA3546977501009385E5EC177510
:103FF000010013052579829701E917650100130572
:10400000E55CEF40515E01A097F7FF1F938747657E
:104010003EC4B7F507008567938707C0814617F64A
:10402000FF1F13066630E10519453EC697E0FF1FE6
:10403000E780604D7C44194697F5FF1F9385C52E98
:10404000138581368297340017F6FF1F1306C62D9D
:10405000977501009385C530177501001305C531AB
:10406000EF402011AA8415C997750100938585D466
:104070001765010013050551EF403142A6851775FC
:104080000100130565E4EF4051412945EF403145FA
:10409000F2406244D24405618280EFA00028177587
:1040A0000100130565D9EF30602CEF704016EF006A
:1040B000D13417F5FF1F130565F0EF00B121177517
:1040C0000100130565D8EF001135AA84EF30100701
:1040D000EFC0205AEF207154EF403023EF3050668C
:1040E000EFE01037977501009385C5CC1765010087
:1040F0001305454989C8EF40513AA6851775010057
:104100001305C5DE49B7EF40513917750100130596
:1041100025E0EF4091382945EF40713CEFE0B019C0
:10412000EFB0E0436305050E854537050400EF1049
:104130005046977501009385E5C717650100130583
:104140006544EF409135177501001305E5DDEF403B
:10415000D1342945EF40B13897F7FF1F938787D9AE
:1041600083D7070017F7FF1F2313F71E854717F79D
:10417000FF1F230DF71CEF10A065EF10404817F547
:10418000FF1F0355C51CEF20101897F7FF1F83C7AB
:10419000D71BB9EFA303010083274417130671004F
:1041A000854513055030829797750100938585C02A
:1041B000176501001305053DEF40312E177501000D
:1041C0001305C5D8EF40712D2945EF405131977542
:1041D0000100938525BE176501001305A53AEF4040
:1041E000D12B17750100130565DCEF40112B71BD54
:1041F00097750100938505BC176501001305853887
:10420000EF40B129177501001305C5D765BF977534
:104210000100938525BA176501001305A536EF4007
:10422000D12717750100130525E8EF40112729450F
:10423000EF40F12A0145EF20304051BF411122C427
:1042400037E404008327041A06C68297EF2070140F
:104250008327040817F5FFFF1305857F829797F7DB
:10426000FF1F2381A70C17F5FF1F130565D8EF204B
:10427000E02F2244B2404101B9BB411122C4914612
:104280002A84138601349D652D4506C697E0FF1FDD
:10429000E7806027B7F7070003C70701A547631347
:1042A000F70001A09306001001469D65254597E0A3
:1042B000FF1FE7804025238081342244B24091468D
:1042C000138601349D652945410117E3FF1F6700EF
:1042D0008323B7E704001171FC47CED79389C1252A
:1042E000A2DDCAD986DFA6DB2E8432892E86AA8576
:1042F0004E85829783C70900130780029387E707DB
:1043000093F7F70F636AF774176701001307872F96
:104310008A07BA979C43BA9782878D4797750100A1
:10432000938585AB176501001305C525630BF40064
:10433000EF40B116176501001305C568EF40F11590
:10434000FDA2EF4091151765010013052569EF40A7
:10435000D1142945EF40B118930720F811469385F1
:10436000C1254A85238EF124A38F0124EFF06FDB52
:104370002A840DC597750100938505A61765010070
:1043800013054520EF407111A28517650100130543
:10439000A568EF4091102945EF4071149775010011
:1043A000938585A3176501001305C51DEF40F10E28
:1043B0001765010013058567EF40310E2945EF4071
:1043C00011124165930730FA05469385C1257D1585
:1043D000238EF124EFF0EFD42A840DC597750100E8
:1043E0009385859F176501001305C519EF40F10AF4
:1043F000A2851765010013052562EF40110A2945C2
:10440000EF40F10DB7E70400BC4F0566130606C880
:10441000A14517F5FF1F0345E5F08297FE506E5446
:10442000DE544E59BE591161828091476301F402F6
:10443000977501009385459A17650100130585144A
:10444000EF40B1051765010013058561C5BDB7E7EC
:104450000400FC4F914517F5FF1F0345A5EC82971B
:104460009775010093854597176501001305851120
:10447000EF40B1021765010013054560EF40F101FF
:104480002945EF40D105EF1090619145E1A28547A4
:104490006301F40297750100938505941765010087
:1044A0001305450EEF40617F176501001305855E1A
:1044B00071B597F7FF1F239227E9B7E70400056658
:1044C000BC4F130606C8C145A9B78D476301F40266
:1044D0009775010093854590176501001305850ABE
:1044E000EF40A17B176501001305855C81BD930733
:1044F00040F811469385C1254A85238EF124A38F68
:104500000124EFF00FC22A84E30A05F09775010039
:104510009385858C176501001305C506EF40E1778B
:10452000A285176501001305254FEF400177294546
:10453000EF40E17AE5B59147E31CF4F8B7E70400F2
:10454000FC4F9305000217F5FF1F0345A5DD829779
:10455000977501009385458817650100130585024D
:10456000EF40A173176501001305055601BF894788
:1045700063E1870297750100938505861765010041
:1045800013054500EF4061711765010013050555DE
:1045900075B383C4E12583C7D12597750100938541
:1045A000A583A204176501001305C5FDDD8CEF404E
:1045B000C16EA2851765010013058553EF40E16DBB
:1045C000C2042945EF40A171C1849305D4FF93969D
:1045D0000401C1824A8693F5F50F1385F125EF108A
:1045E000C07EE35D90E2930750F8238EF12483C7E9
:1045F000390022869385C12585074A85A38FF1243A
:10460000EFF02FB22A84E30B05E097650100938554
:10461000A57C176501001305E5F6EF400168A2854A
:1046200017750100130505A509B7894763E18702DE
:10463000976501009385457A17650100130585F498
:10464000EF40A165176501001305454CC5B9EF1092
:104650001045A2851385C125EF204077C1B38D4752
:104660006301F402976501009385057717650100E2
:10467000130545F1EF406162176501001305C54A56
:1046800075B9B76602000146B7750200054597E0A7
:10469000FF1FE78040E7930760F8238EF124A38F84
:1046A00001249307002623A0F126E57793870721AD
:1046B0002392F1263146A383A1269385C1254A85FD
:1046C00023830126EFF0EFA52A84E30905D497653B
:1046D000010093856570176501001305A5EAEF4099
:1046E000C15BA28517650100130585453DBDB14736
:1046F0006301F402976501009385056E176501005B
:10470000130545E8EF40615917650100130505459C
:1047100035B1B7E70400FC4F9305000417F5FF1F00
:10472000034545C08297EF109037B14525B79147B3
:1047300063E18702976501009385056A17650100AB
:10474000130545E4EF406155176501001305C542A7
:10475000F5B683C4012683C7F125A204DD8C8E043F
:10476000B77702006D14BE942286A68517650100F6
:104770001305C541EF406152B7E70400FC472286AC
:10478000938511262800829793160401C182300078
:10479000A685094597E0FF1FE780E0D62A8419C562
:1047A0001765010013054540EF40E163930770F87A
:1047B00019469385C1254A85238EF124A38081263D
:1047C000EFF02F962A84E30B05C4976501009385CB
:1047D000A560176501001305E5DAEF40014CA285DD
:1047E000176501001305453D89B399476301F4102E
:1047F000976501009385455E17650100130585D80F
:10480000EF40A149176501001305853C05BE91479E
:1048100063E18702976501009385055C17650100D8
:10482000130545D6EF406147176501001305C53BE9
:1048300031B683C4012683C7F125A204DD8C8E0422
:10484000B77702006D14BE942286A6851765010015
:104850001305C53AEF406144B7E70400FC472286E0
:10486000938511262800829793160401C182300097
:10487000A6850D4597E0FF1FE780E0C82A8419C58B
:104880001765010013054539EF40E155930780F89E
:1048900019469385C1254A85238EF124A38081265C
:1048A000EFF02F882A84E30B05B697650100938506
:1048B000A552176501001305E5CCEF40013EA28526
:1048C00017650100130585368DB199476301F40220
:1048D000976501009385455017650100130585CA4A
:1048E000EF40A13B176501001305C53581BCB7E753
:1048F0000400FC4F9305000417F5FF1F034585A234
:104900008297EF10D0199945B1B38D476301F40236
:10491000976501009385454C17650100130585C611
:10492000EF40A137176501001305453301BC17653A
:1049300001001305A533EF40014B1305C01297E0AA
:10494000FF1FE780409F0145EFE02FA60D45EFF0E8
:10495000DF92294597E0FF1FE780E09D97E0FF1F6A
:10496000E780008F65BC99476301F40297650100F9
:1049700093858546176501001305C5C0EF40E131F9
:10498000176501001305452F55BA03C7112683C7C4
:10499000012622075D8F9166BA96C2061166C18212
:1049A0001306F6EF8D476363D60297E7FF1F9387E1
:1049B00027649C4B03C6F1259386C70039C603D6EE
:1049C00007005DCA8907E39CD7FE89471307A0F853
:1049D00011469385C1254A85238EE124A38FF124B6
:1049E000EFE03FF42A84E30B05A29765010093856D
:1049F000A53E176501001305E5B8EF40012AA28521
:104A000017650100130585280DB603D6070063025C
:104A1000E60A8907E39BF6FE8D474DBF9147630287
:104A2000F402976501009385253B17650100130586
:104A300065B5EF408126176501001305A5266FF0C7
:104A4000FF8FB7E70400FC4F9305000817F5FF1F21
:104A50000345458D829705BC976501009385C53751
:104A600017650100130505B2EF402123176501000A
:104A70001305C5246FF09F8C2390E70017E5FF1FF7
:104A800013050557EFE02021976501009385C53494
:104A900017650100130505AFEF40212017650100E0
:104AA0001305C522EF40611F2945EF40412381478F
:104AB00031BF2390070017E5FF1F13056553EFE093
:104AC000801D976501009385253117650100130549
:104AD00065ABEF40811C176501001305A520D9B710
:104AE000411122C406C6834705002A849DC39765E9
:104AF00001009385252A176501001305A5A8EF403D
:104B0000C1194C40176501001305055DEF40E11820
:104B100075A05841B707CF009387777D6313F706D9
:104B2000976501009385052717650100130585A585
:104B3000EF40A1161C448356E4008355C40003C60D
:104B40000700176501001305A55AEF400115294517
:104B5000EF40E1180357E40097E7FF1F83D7277F53
:104B60006307F7008355C4000844EFE0CF9703566E
:104B7000E4008355C40008442244B24041016FF070
:104B80004FF5B707CC009387777D631FF7029765D2
:104B9000010093852520176501001305A59EEF40B0
:104BA000C10F1C448356E4008355C40003C60700AC
:104BB000176501001305C553EF40210E2244B24092
:104BC000294541016F40A111B707CE009387777D3A
:104BD0006302F702976501009385C51B1765010005
:104BE0001305459AEF40610B4C4017650100130512
:104BF000654529BFB2402244410182805171CAD12A
:104C000037E904008327C904A2D52E8686D7A6D308
:104C10002E84AA851385C125829783C7C1251307D2
:104C2000700A638DE70C636CF7001307600A6382F8
:104C3000E704BE502E549E540E596D6182801307B6
:104C4000800A6382E7121307900AE394E7FE8D4718
:104C5000630BF416976501009385C519176501006C
:104C600013054592EF406103176501001305C5AEBA
:104C700015A08D476306F40297650100938585179B
:104C80001765010013050590EF402101176501002C
:104C90001305C5A5EF4061002945EF40410451BF10
:104CA000854717650100130525A617E7FF1F230792
:104CB000F768EF404113B7750200B766020001467E
:104CC000054597E0FF1FE7800084930760F8238E77
:104CD000F124A38F01249307002623A0F126E57772
:104CE000938707212392F126B14523830126A383CD
:104CF000A1261385C125EF20600D25BF914763E1F3
:104D00008702976501009385E50E1765010013057D
:104D10006587EF309178176501001305E5A09DBF09
:104D200083C4012683C7F125A204DD8C8327C9042F
:104D30006D14228693851126280082978E0493167F
:104D40000401B7750200C1823000A695094597D0CD
:104D5000FF1FE780407B930770F8238EF12499456D
:104D6000A380A12679B7914763E187029765010087
:104D700093854508176501001305C580EF30F17173
:104D8000176501001305C59B31B783C4012683C78E
:104D9000F125A204DD8C8327C9046D142286938536
:104DA0001126280082978E0493160401B77502001D
:104DB000C1823000A6950D4597D0FF1FE780A074F3
:104DC000930780F859BF176501001305259AEF4036
:104DD00081011305C01297D0FF1FE780C055014520
:104DE000EFD0BFDC0D45EFF04FC9294597D0FF1F2D
:104DF000E780605497D0FF1FE78080451DBDB7E76F
:104E000004004111FC4726C29384C1252E8606C6A4
:104E100022C44AC02E842A89AA852685829797654E
:104E200001009385E5FE175501001305A575EF30C8
:104E3000D16683C5C125176501001305A5A3EF3011
:104E4000D1652945EF30B16983C704004147938795
:104E5000070693F7F70F6365F74817670100130715
:104E6000A7848A07BA979C43BA9782879D476303B2
:104E7000F402976501009385A5F917550100130504
:104E80006570EF309161176501001305259FEF30C4
:104E9000D160D1A283C7D125ADCF83D7012603D757
:104EA000E125C207D98F17E7FF1F232DF74883C7D6
:104EB0006400976501009385A5F51755010013055A
:104EC000656C17E7FF1F230EF746EF30115D97E77C
:104ED000FF1F938727478C4317E6FF1F034666464D
:104EE000176501001305459BEF30315B2945EF3015
:104EF000115FA38E01242244B240924402499307D9
:104F000000F8238EF1249D451385C12541016F10C2
:104F1000F06BEF300066239FA124935705012A848C
:104F20002380F126935785010145A380F126EF30B8
:104F300000652381A12697650100938565ED1755CE
:104F4000010013052564EF30515503C62126A285C3
:104F5000176501001305C59541BFCD476301F402F4
:104F6000976501009385C5EA175501001305856112
:104F7000EF30B152176501001305059509BF37E4FD
:104F800004007C4441469385D1251385413D829799
:104F90001385413DEF00207D9D2583C7E12603C792
:104FA000D126A20703238405D98F17E7FF1F2319F2
:104FB000F7381306000A89452244B2409244024958
:104FC00017E5FF1F03450536410102838D47630145
:104FD000F402976501009385A5E3175501001305B9
:104FE000655AEF30914B176501001305A59D45B536
:104FF00003C4E12583C7D12597650100938545E169
:105000002204175501001305E5575D8CEF30F14878
:10501000A285176501001305A58CEF3011482945BD
:10502000EF30F14B0D469385C1252285EFE07F8F50
:10503000AA8415C997650100938585DD1755010080
:1050400013054554EF307145A6851765010013051A
:10505000658AEF3091442244B24092440249294586
:1050600041016F30D14797E7FF1F2398872CB7E79F
:105070000400116603A38705130606E891452DBFBA
:105080008D476301F40297650100938565D8175534
:1050900001001305254FEF3051401765010013053E
:1050A00025A1F5B303C4E12583C7D1259765010088
:1050B000938505D62204175501001305A54C5D8C78
:1050C000EF30B13DA285176501001305E583EF3090
:1050D000D13C2945EF30B1400D469385C12522854D
:1050E000EFE03F84AA840DC197650100938545D206
:1050F0001755010013050549EF30313AA6851765AC
:1051000001001305A581B1B797E7FF1F23968722FA
:10511000B7E70400116603A38705130606E89305A5
:10512000000259BD894763E18702976501009385B5
:1051300025CE175501001305E544EF3011361765EC
:1051400001001305A599A1B383C4E12583C7D12527
:10515000976501009385C5CBA2041755010013057F
:105160006542DD8CEF307133A685175501001305BC
:10517000657CEF3091322945EF3071362286938578
:10518000C1252685EFE0EFF92A84630A05169765A5
:1051900001009385E5C7175501001305A53EEF30C3
:1051A000D12FA285175501001305057A5DB58547F6
:1051B00063F78714834519002244B24092440249A0
:1051C000B335B00097E7FF1F238AB71617550100C4
:1051D0001305C57841016F30512CA2852244B2409D
:1051E00092444A85024941016FF05FA199476301EA
:1051F000F402976501009385A5C1175501001305B9
:105200006538EF309129176501001305E5A641B116
:1052100003C4E12583C7D12597650100938545BF68
:105220002204175501001305E5355D8CEF30F1269A
:10523000A285175501001305E573EF3011262945A6
:10524000EF30F12919469385C1252285EFE06FEDF6
:10525000AA840DC197650100938585BB1755010090
:1052600013054532EF307123A6851755010013054C
:105270006571C5B397E7FF1F2398870CB7E7040054
:10528000116603A38705130606E8930500082DB3EE
:105290008547976501009385A5B71755010013054C
:1052A000652E6309F400EF30511F175501001305F7
:1052B000A56EF1BEEF30711E175501001305456F45
:1052C000EF30B11D2945EF3091212244B240924484
:1052D000024997E7FF1F2395070641016F30C01D64
:1052E000976501009385C5B21755010013058529FF
:1052F000EF30B11A176501001305459C49BEB24055
:1053000022449244024941018280411106C622C4CE
:10531000EFE02FE19377F50F95CB2A849765010095
:10532000938585B0175501001305C525EF30F1169B
:105330009375F40F176501001305C5D3EF30F11510
:105340002244B240294541016F307119B2402244D4
:105350004101828001114EC697E6FF1F83D626FFCA
:10536000B28917E6FF1F035666F726CA4AC806CE5B
:1053700022CCAA842E89152397E7FF1F83C707FD38
:10538000A9CB03C4440083C734001765010013058B
:1053900065DA22045D8CEF3051104A86A68522859D
:1053A000AD37638F090297E7FF1F83C707FA8DCBDD
:1053B0006308090297E7FF1F83C747F895E3624434
:1053C000F240B249CA8526854249D24405616F1030
:1053D000F01F17650100130565D6EF30D120D1B756
:1053E000F2406244D2444249B24905618280834717
:1053F00055008345450017650100130565D2A207D6
:10540000DD8D6F30910917650100130565D06F3090
:10541000911D8D4763F2B70A011126CA06CE22CC30
:105420000344350097E4FF1F83C434F297650100FD
:10543000938585D1B337800017E7FF1FA307F7F0E7
:1054400009C4976501009385E5D017650100130530
:10545000E5D0EF30910497E7FF1F83C717EF638311
:1054600097001D2C97E7FF1F83C737EE9DC3854725
:105470002306F100B7E7040083A7471770008545AE
:1054800013055030829717650100130525CEEF30C4
:1054900091159967938757EE2316F10068008547A9
:1054A0009145A30781002307F100EF103012F2406D
:1054B0006244D244056182808280894763F2B708E2
:1054C000011122CC06CE26CA8344250085472A84B2
:1054D0006398F404914763F0B7040345450083479C
:1054E000340022055D8D97E7FF1F2399A7DE15295C
:1054F0009967938767EE2314F100834734002305EF
:105500009100A305F1008347440095452800230638
:10551000F100EF10B00BF2406244D244056182808A
:10552000FDF89967938767EE2314F10097E7FF1F53
:1055300083D7C7DAA305F10023050100A183F1B7E2
:1055400082800111996722CCD51717E4FF1F13043D
:10555000E4DF2314F1008347040026CA97E4FF1F09
:105560009384E4DE2305F10083D7040028009545E9
:10557000A305F100A18306CE2306F100EF1010056C
:1055800003D604008345040017650100130585BF99
:10559000EF30A170F2406244D244056182809D6781
:1055A0007971D9172316F10097E7FF1F83C707DA30
:1055B00006D62307F1009DCBB7E70400FC47414620
:1055C0009385413D1305F10082976800CD45EF10AA
:1055D000E07F97E5FF1F83C565D7176501001305B9
:1055E00065BDEF30816BB25045618280B7E7040042
:1055F000BC47414681451305F1008297F9B7B7676B
:1056000002036971938757AA3EC4856785072316ED
:10561000F10097E7FF1F938767D383C70700232411
:105620008112A30701002307F10097E7FF1F93876B
:1056300007D283D7070037E404002326111223186A
:10564000F10097E7FF1F938767C983D7070041469B
:1056500048082319F1007C449385413D8297F14528
:105660002800E52A2312A1027C442C002810794648
:1056700082973C44130561041306900D814582977F
:1056800030109305700F0145EFD0BFB48320C112D5
:105690000324811255618280B7C7A55A01119387EF
:1056A000C7333EC497E7FF1F83C737CA3EC6B7F765
:1056B000070003C7070106CE22CCA5476313F700F6
:1056C00001A01164930504F09306001001462545DE
:1056D00097D0FF1FE78020E33000930504F0A14638
:1056E000294597D0FF1FE78000E297E5FF1F83C59C
:1056F000D5C5176501001305A5BCEF30015AF2406E
:1057000062440561828001119165A1463000938554
:1057100005F02D4506CE97D0FF1FE780C0DE22475B
:10572000B7C7A55A9387C7336312F702B245176507
:105730000100130525ACB335B00097E7FF1FA38622
:10574000B7C0EF308155F240056182808145176511
:105750000100130565AC97E7FF1FA38807BEEF3074
:10576000C1531D3FCDB7B7C7A55A79719387F73598
:105770003EC6B7E70400FC47AA8506D622D44146B8
:1057800008088297B7F7070003C70701A547631307
:10579000F70001A01164930504E893060010014688
:1057A000254597D0FF1FE78000D67000930504E8D9
:1057B000D146294597D0FF1FE780E0D41765010047
:1057C0001305C5B3EF302162B25022544561828087
:1057D00079719165D1467000938505E82D4506D60F
:1057E00097D0FF1FE78020D23247B7C7A55A9387CB
:1057F000F73517650100130525AA631EF700B7E703
:105800000400FC471385413D41460C08829717650B
:105810000100130565A6EF30015DB250456182803D
:10582000B7F7070003C70701A5476313F70001A0F7
:1058300091654111930600100146938505E82545C1
:1058400006C697D0FF1FE78000CCB2401765010065
:105850001305859841016F300159C167697681460A
:10586000FD1705061397060141836364B7003E8563
:1058700082803307D50003470700B98F214713F80B
:105880001700858363050800B18FC207C1837D17A8
:105890001377F70F6DF78506F1B749C1A54705479F
:1058A00063FFB70683471500034705003168A20769
:1058B000D98F13978700A183D98FC207C18313089B
:1058C000C8550547639D0705411106C622C426C277
:1058D00003442500914763FD8702930754006399B1
:1058E000F502A301C50021822302C5009304340000
:1058F00091C6A302D500A1822303D5002A84A685E0
:10590000A93F26942300A4002181A300A4000147FD
:10591000B240224492443A854101828005473A854B
:105920008280B7C7A55A01119387E7343EC42AC6BF
:10593000B7F7070003C7070106CE22CC26CAA54742
:105940006313F70001A091642A84938504EE930603
:1059500000100146254597D0FF1FE780C0BA3000F0
:10596000A146938504EE294597D0FF1FE780A0B993
:10597000A285176501001305A596EF300132EFF0FF
:105980001FC8F2406244D2440561828001119165D2
:10599000A1463000938505EE2D4506CE97D0FF1F1A
:1059A000E78060B62247B7C7A55A9387E7346314E8
:1059B000F702B245176501001305058897E7FF1F39
:1059C000239EB790C205C181EF30212DEFF03FC378
:1059D000F24005618280D147D1451765010013056A
:1059E000A58717E7FF1F231BF78EEF30012B17E565
:1059F000FF1F0355A58E3537E1BF011126CA06CE1C
:105A000022CC93F71500AE848DCBAD6737170040DD
:105A10009387A7AA1CC3B7E70400BC4F130600195D
:105A2000854517E5FF1F0345458B829713C5140075
:105A3000F2406244D2440561828093F7250063837B
:105A40000712976501009385658F2D464800EF305A
:105A5000611997E5FF1F83C5758F854793C424009F
:105A600063E1B70489CD97E7FF1F83C7078E85C31E
:105A70008545170500201305E5F7EF102035139530
:105A8000040197E7FF1FA383078C418155B7416548
:105A90000546970500209385E5F57D15EFF0FF8617
:105AA000F9BF170400200344E4F49707002083C7DC
:105AB00077F422045D8CAD679387B7556306F408CD
:105AC00063E68702A9679387A7556306F40897E7FB
:105AD000FF1F83C787878DE741652E867D15970554
:105AE0000020938525F1EFF05F82B9A0B16793871D
:105AF000C755630EF400B5679387D755E319F4FCD7
:105B000017050020130505EFEF10402C35A00546C2
:105B100017050020130505EEEFF0DF8397E7FF1F61
:105B200083C7C78291EB4800EF30213493150501FC
:105B3000C1814800EFD02F9BA285175501001305A6
:105B4000E57DEF30811525BF17050020130585EA97
:105B5000EFF0FF89D5B7170500201305A5E9EFF091
:105B60009F8AD9BF93F745000145E38307EC17559A
:105B700001001305E57BEF300127EF10003713C557
:105B800044007DB5411122C437E404005C5C06C6C4
:105B90003546975501009385253217650100130599
:105BA00065BE829701E9175501001305E579EF30CD
:105BB000812301A08327041C82972A840545EF8056
:105BC0002075EF10C168EF100147EF70B0292285F2
:105BD000B2402244410182801567B7170040130785
:105BE000575598C3D8439D66558FD8C3D843FD7683
:105BF000758FD8C3D8431367F70FD8C3356713071A
:105C0000C7CC98C3828041111305800406C622C404
:105C100026C24AC097C0FF1FE780604985457D5571
:105C2000EFC0FFDF85457D55EFC0DFE93714004049
:105C30008327840A8D451305002093E7072023243A
:105C4000F40AEFC0DFDDB7E40400EFD04F8FC8588F
:105C50001309840C1304C40CEF30E118176501001C
:105C6000130545B2EF3021188327C4FF8545414510
:105C700093E70708232EF4FEEFC0DFE48D451305FC
:105C80000008EFC03FE4EFC0BFFE0145EFD06F81D9
:105C900085450545894717D7FF1F230BF76AEFD0C6
:105CA000EF8137070004B7E700E023A0E710EFD04B
:105CB000DF8EEFD05FA2F935EFF0FFA4EFF01FCD3C
:105CC000EFE0CFD78D450D65EFC0DFDF1705002072
:105CD000130545E285671CC589672320250140C15E
:105CE0002326250100C95CC983A7841E829783A748
:105CF000040817050000130585D0829797D7FF1F6A
:105D0000238DA75CBC4C1306006485458297E9355A
:105D100097C0FF1FE780C06C01458280B7F707007E
:105D200003C70701A547AE866316F70093974501A1
:105D300091C301A0AA850146254517C3FF1F67002F
:105D4000837C4111B2862E86AA852D4506C697C052
:105D5000FF1FE780407BB2400145410182809307ED
:105D6000000463E6C7021D71A2CC2A84080886CE0F
:105D700032C6EF203167B2461008A285294597C088
:105D8000FF1FE7804078F6406644256182803955E0
:105D90008280411126C2AE848D4522C406C62A8463
:105DA000EFC05FD2B717004099C803A5C70C418D5B
:105DB00023A6A70CB240224492444101828003A54D
:105DC000870C418D23A4A70CF5B783470500034733
:105DD0001500A207D98FC2076177C1871307272053
:105DE0006397E70083452500370504005DB782808F
:105DF00097D7FF1F9387075618429C4383D64500C9
:105E00000345070083C5C700035646006396A500F7
:105E100083D5E700638DD502011106CE2386A70046
:105E20002397D700B705CF00DC4B9385757D050719
:105E30007D162EC2230001003AC42316C100231789
:105E4000D10099C30A858297F240056182808280E1
:105E5000DC4DDC4B81CFB7E70400904503A38705F9
:105E6000914517D5FF1F0345254F028382806D7131
:105E70003C083EC6B707E500232291103EC8AA841D
:105E80003C083285232611103ECA2324811023208A
:105E900021112E89EF2090672A8497550100938560
:105EA000E552174501001305E56DEF20115FA2854E
:105EB0001755010013058561EF20315E2945EF205C
:105EC0001162B705CB009385757D6800EF10A04384
:105ED000A2856800EF203059014781467000CA85CD
:105EE0002685EF10C06215C52A8497550100938559
:105EF000E54D174501001305E568EF20115AA2850D
:105F0000175501001305455DEF2031592945EF2054
:105F1000115D8320C11003248110832441100329C3
:105F200001105161828097D7FF1F9387A7421842C3
:105F30009C43797122D406D60348070083C8070121
:105F40002A8483D64500035546006396080183D80A
:105F50002701638DD8022388070105072399D700FD
:105F60003708CC00DC4B1308787D3ACC1307F5FFDB
:105F700042CA23080100231EE100231FD10099C754
:105F8000080832C62EC482973246A2452285C535FE
:105F9000B2502254456182806D713C083EC0B70703
:105FA000E5003EC23C083EC4232611102324811084
:105FB0002322911023170100231801002319010047
:105FC000231A0100231B010097D7FF1F83D7470621
:105FD00099E3C167FD172316F10097D7FF1F83D7F9
:105FE000470591EB97D7FF1F9387C7369C439C4388
:105FF000DC4783D7070017D4FF1F13046403584CF2
:106000002317F10083574400484B2318F10005ED96
:106010009755010093858542174501001305855664
:10602000EF20B1471755010013058542EF20F146D7
:106030002945EF20D14A8320C110032481108324F5
:1060400041105161828097D7FF1F83C7D7FE89EB2C
:10605000B7E70400BC5782975C4C23AA0700E1BF56
:10606000FD1797D6FF1FA388F6FC03560701834749
:1060700004014C470A85230BF100EF20F03C97D731
:10608000FF1F9387272D9C430147814688430A863B
:106090006C00EF10C047AA841DC997550100938575
:1060A000E539174501001305E54DEF20113FA685A1
:1060B000175501001305853AEF20313E2945EF20A1
:1060C0001142584CB7E70400BC57484B69B797D703
:1060D000FF1F83C757F6F5D7B7E70400BC4F10443E
:1060E000854517D5FF1F034525278297A9B75C4E25
:1060F000DC4BA9CBA1C9411122C4174501001305EE
:1061000065482E84975501009385853106C6EF209A
:10611000D138A2851755010013058536EF20F137D8
:106120002945EF20D13BB7E704002244B24003A346
:10613000870517D5FF1F0345252213064006914505
:10614000410102838280411122C417D4FF1F13042E
:1061500024EC1C4C06C689C7DC4399C34C48829783
:10616000584CB7E70400BC57484B82975C4CB24090
:10617000224423AA07004101828017D7FF1F13077B
:106180000716834707009306F00B850793F7F70F71
:1061900063E9F60097D6FF1F2383F6140345070033
:1061A0008280930700F8FDB7835745006386070E8A
:1061B00001114AC817D9FF1F130989E752C4032ADE
:1061C000C90106CE22CC03274A0126CA4EC656C2B2
:1061D000F15721EF1307D00DFD576368C704B7E9E6
:1061E000040083A709072A8413058600420541811C
:1061F000B284AE8A8297232AAA000325C9015C498A
:106200009DEF975501009385A51F174501001305C4
:106210006537EF209128175501001305A52EEF20B3
:10622000D1272945EF20B12BDD57F2406244D244FB
:106230004249B249224A924A3E850561828093874B
:106240004400B705CF002319F5009385757D31050E
:10625000EF10600B0325C901834564003105EF2071
:1062600090200325C9012686D6853105EF20D01D53
:106270007146A2854A85EF20F116504419CA83A7BA
:106280008905854517D5FF1F0345050D8297814771
:1062900069BFEFF07FD0E5BFFD573E858280411199
:1062A00026C297D4FF1F9384A4D8D84C22C437E4C5
:1062B00004003C54484B06C68297DC4C0323C405BB
:1062C0002244B240924423AA070017D5FF1F03457A
:1062D000A508854541010283411126C297D4FF1FBD
:1062E000938444079C4006C622C44AC0C9CBDC4301
:1062F000D9C75CC12300B5002A8497550100938556
:10630000650B174501001305E527EF2011192945F5
:10631000EF20F11C9C4023A4070023A2070097D77D
:10632000FF1F9387E7CEDC4FDC4B81C72955EFF089
:106330009FE197D7FF1F9387A7CFDC4FDC4B91C31B
:10634000B93F37E904008327C905894517D5FF1FE1
:106350000345850082978327C905914517D5FF1FFF
:10636000034585FF82979C4003A34701630903000F
:1063700022852244B2409244024941010283B24044
:10638000224492440249410182800111328506CEA5
:1063900022CC26CA2E84EF207017AA8497550100BC
:1063A00093858504174501001305C51DEF20F10EE7
:1063B000030784000356640083554400A6861755DE
:1063C00001001305E50DEF20510D2945EF20311196
:1063D00097D7FF1F83C727C4639897000145EFF045
:1063E0009FD681450A85CD3DF2406244D244056185
:1063F00082806D7123248110232611102322911095
:1064000093F745002E84638507123C083EC0B7070A
:10641000E5003EC23C083EC42317010023180100DA
:1064200023190100231A0100231B010097D7FF1F26
:1064300083D707BE99E3C167FD172316F10097D7ED
:10644000FF1F83D707BD91EB97D7FF1F938787F077
:106450009C439C43DC4783D7070017D7FF1F1307D4
:1064600027BB2317F100544F835747002318F1002F
:10647000DC4A95EF97550100938545FB17450100D0
:1064800013054510EF20710117550100130545FC58
:10649000EF20B1002945EF209104134544008320EB
:1064A000C11003248110832441105161828097D749
:1064B000FF1F83C757B62555ADCBFD1717D6FF1F56
:1064C000A30BF6B403D6060183470701CC460A8521
:1064D000230BF100EF20407797D7FF1F938787E7C3
:1064E0009C4317D7FF1F1307A7B297660100938637
:1064F000A6C888430A866C00EF106001AA8451DDAB
:1065000097550100938585F217450100130585070E
:10651000EF20A178A68517550100130525F4EF207B
:10652000C1772945EF20A17B2685EFF0DFC1B5B704
:1065300093F725009DC3B7E70400BC47414681455A
:10654000280882972555EFF01FC028089305F00F03
:10655000EFF09FD81345240099B793F71500014534
:106560009DDFEFF07FA31345140015BF5C4D411173
:1065700006C688C317D7FF1F232EF7DCB7E7040032
:1065800083A70708170500001305E5E68297B240C8
:1065900097D7FF1F2382A7DC0145410182800111AB
:1065A0009307700F2316F10006CE97D7FF1F83C7FE
:1065B00077DB8DE7B7E7040083A7870D17D6FF1FAA
:1065C000034646D26C0017D5FF1F0355E5D98297C5
:1065D0003335A00097D7FF1FA386A7D8F2400561E7
:1065E000828041119397050122C406C626C2C18745
:1065F0002E8463D40702B7E40400FC5417D5FF1FB0
:10660000034545CE829719C1BC5482972165218DDF
:10661000B240224492444101828093F715008DC715
:10662000B7E7040083A7471A17D6FF1F130646A231
:1066300097F5FF1F9385055117D5FF1F034585CAA1
:10664000829713451400E9B793F7250099CFB7E770
:106650000400BC4F13060064894517D5FF1F03458E
:1066600065C882971345240065B793F785009DC7D9
:10667000B7E7040003A8871A1307401F97D7FF1F27
:1066800083C747C6814613064006994517D5FF1FA5
:10669000035585CD0298134584009DBF93F74500AF
:1066A0000145BDD7B7E4040083A7041817D5FF1F21
:1066B000035585CB8297BC4C13060064914517D5D2
:1066C000FF1F034525C282971345440091B797D712
:1066D000FF1F83D767C96396A70217D7FF1F23162B
:1066E000B7C817D7FF1F2313C7C817D7FF1F23101B
:1066F000D7C82E8617550100130585F6BE856F2075
:10670000C15917550100130525F76F20C16D0357B7
:106710004500011106CE22CC97D7FF1F83D7C7C4EF
:1067200017550100130545F56310F706C167F91702
:1067300017D7FF1F232AF7C237E4040097D7FF1F9C
:1067400023A607C27C4C894517D5FF1F034585B991
:1067500082977C4C914517D5FF1F0345A5B88297BA
:1067600097D7FF1F83C777BE95C78547A307F1005B
:10677000832744171306F10085451305503082978F
:10678000175501001305C5E4EF20E165F2406244AE
:106790000561828097D7FF1F83C747BB175501004C
:1067A0001305C5E7F5F38547A307F10083274417D1
:1067B0001306F100854513055030829717550100E7
:1067C000130545E3D1B77D15954763E0A71A175721
:1067D00001001307A7DC0A053A951C41011122CCE0
:1067E00006CE26CABA972E84828717550100130554
:1067F00025E9EF20415F0DA203C725009947631DDE
:10680000F7002E85EFF0BFF08345640017550100B7
:10681000130505E8EF20614897D7FF1F238707B2CC
:1068200017550100130585E8E9B703C7250095470B
:106830006317F702C16717D7FF1F0357E7B2F917AE
:1068400003D5A5006307F702B7E7040083A7C717BE
:10685000829717550100130565E6EF20C15885475B
:1068600017D7FF1F2303F7AE17550100130585E760
:1068700049B797D7FF1F2399A7AE83D7E500B7E4A1
:106880000400096617D7FF1F2311F7AE83D7050150
:106890001306069017D5FF1F0345C5A417D7FF1F82
:1068A0002316F7AC83D72501A14517D7FF1F231067
:1068B000F7ACBC4C8297BC4C13060064914517D5CD
:1068C000FF1F034525A282970356E4008355A400C9
:1068D000175501001305C5DFEF20213C49B71755B7
:1068E00001001305E5E031B783C525009147639AA0
:1068F000F502854717550100130505E1A307F100CF
:10690000EF20614EB7E7040083A747171306F10095
:106910008545130550308297F2406244D2440561A8
:1069200082809947639EF5002285EFF05FDE834504
:106930006400175501001305A5D5EF200136E9BF06
:106940009547639FF5008347140017550100130511
:10695000A5DBE39007EA175501001305A5DC51BD3F
:1069600017550100130585DCC9BF82806D71232492
:1069700081102326111023229110328401CD8947E2
:106980006306F5028320C110032481108324411083
:106990005161828017550100130505DAAE84EF209E
:1069A0008144A2852685EFE08FC5E9BFB7E70400E3
:1069B000FC4728008297175501001305A5D8EF2042
:1069C00081428347810039C01307000B638EE700C3
:1069D0001387A7051377F70F8D4663E9E602A285B3
:1069E0002800EFE0AFA179BF8547E3FD87F8834535
:1069F000910017450100130565F6B335B00097D730
:106A0000FF1F238DB792EF204129ADBF03479100AF
:106A1000A207D98F35671307D755638DE7066366DD
:106A2000F7022D671307B7556381E7063167130730
:106A3000C7556386E70429671307A7556392E702E2
:106A4000A2852800EFE03F9C35BF39679306E765D4
:106A50006383D70663E9F6001307E7556388E70405
:106A6000A285280089B73D679306F755638AD70446
:106A70001307F766E396E7FEEFE07FB221B7014622
:106A8000A2852800EFE01F8DF5BDA2852800EFE06C
:106A90001F96CDBD8947E3F787EE9305E4FFC20556
:106AA000C1811305A100EFC00FA4E9BDA285280094
:106AB000EFE03F96C1BDA2852800EFE01FA0D9B549
:106AC000EFE03FA8C1B5411122C417C4FF1F130452
:106AD000E459AA86175601001306C6AD2285C145A2
:106AE00006C6EF2041310357440097C7FF1F938725
:106AF000E7582393E700035764002394E700B2406C
:106B0000224441018280011106CE22CC6D3F37E440
:106B100004008327841417C6FF1F13062655D54586
:106B200001458297832784179305F10013055030A0
:106B300082978347F100A1C7A30701008327441769
:106B40001306F100854513055030829783274417BB
:106B500017C6FF1F13068652CD4513057030829766
:106B60008547A307F100832744171306F1008545E5
:106B7000130550308297F24062440561828083277A
:106B8000441717C6FF1F1306664FCD451305703017
:106B9000D5B7130101DE232C812037E404008327BD
:106BA0000408232E1120232A912023282121232683
:106BB000312117050000130505A3829717C9FF1F90
:106BC00013094972994785442300A9002318F1004D
:106BD00097550100938505A79307400617450100C7
:106BE0001305459A2314F1102304910097C9FF1F40
:106BF0009389E975EF20610A83D5090017550100D3
:106C00001305059CEF2061092945EF20410D03D5AF
:106C10000900EFF05FEB832744173000854513052B
:106C2000503082978327441717C6FF1F1306064567
:106C3000CD451305703082978327441717C6FF1F71
:106C40001306C641B5451305603082978327441764
:106C500010088945130510318297832744173002A5
:106C60008945130520318297832744159305000534
:106C70000D4582978327441593050005114582979A
:106C8000A301910023029100230491002324011009
:106C900023080100832784163002914513057040B4
:106CA000829783278416130631008545130500401B
:106CB00082978327841650008545130510408297DC
:106CC0008327841610088545130520408297832763
:106CD000841630008545130550408297832704159C
:106CE0007D558297832744137D5582977D55EFC04C
:106CF0002FC78327440C8297EFC06FA48327841487
:106D000017C6FF1F13068636D5450145829789476A
:106D10001306700F814508082302F100EFB0EF84DD
:106D20008D471306700F814528022308F100EFB04C
:106D3000CF8391472304F11097C7FF1F9387075B09
:106D4000984383C747003AC42306F100EFE03F8B26
:106D5000500085450545EFC0CFC710089305700F5B
:106D60000945EFC00FC730029305700F0D45EFC006
:106D70004FC6300095451145EFC0AFC5C16717C775
:106D8000FF1F1307675EF9171CC32322070017C5EF
:106D9000FF1F1305E554EFC0AFC28327C41D17C5FD
:106DA000FF1F1305A55B82973C48034509008545F5
:106DB00082978320C1210324812183244121032937
:106DC00001218329C1201301012282800111C167A1
:106DD00026CA06CEAA8422CC17C5FF1F0355C55864
:106DE000F9176306F50437E40400832784122E861E
:106DF0002315B10001478146ED4582977C44035637
:106E0000A1002AC6A68582972C0017C5FF1F03552F
:106E1000A555EFC0AFC701CD1755010013058583F8
:106E2000EF10717C8327C412ED4528008297F24051
:106E30006244D24405618280011106CE22CC2DC964
:106E4000854717C7FF1FA300F72297C7FF1F238D92
:106E5000072037E40400832784179305F100130506
:106E6000503082978347F100A9CBA3070100832705
:106E700044171306F1008545130550308297832788
:106E8000441717C6FF1F1306661DB545130560306E
:106E900082978547A307F100832744171306F10063
:106EA0008545130550308297F24062440561828027
:106EB00097C7FF1FA389071A49BF8327441717C61F
:106EC000FF1F1306A619B54513056030E9BFC1675A
:106ED00017C5FF1F03554549F9176307F500B7E7C5
:106EE000040003A3C7170283828001118547A3070B
:106EF000010017C7FF1F2307F746B7E7040083A762
:106F0000471706CE1306F1008545130550308297CA
:106F1000F24005618280EFA2BFE02A8408452E89F5
:106F2000B28909C900C1970500009385C574610540
:106F3000EF00810181447D5AEF10C00963C3A404AE
:106F40008144EF10200A63C6A40497F7FF1F9387BC
:106F500027C09C43DC47B307F94091872302F40024
:106F6000638109048327C900B307F4409587A3020E
:106F7000F4001C4C89C79C4799C3228582976FA057
:106F80007FDD5C44139714008504BA972390470172
:106F900065B71C48139714008504BA97239007001F
:106FA0004DB7832789000547B307F4409587A302AF
:106FB000F40083570400638EE7028DC3094763849E
:106FC000E7040D47E397E7FA97570100938747CA0D
:106FD0001CCC975701009387A7CA11A897570100A7
:106FE000938787901CCC975701009387E7905CC8E4
:106FF00049B7974701009387277C1CCC974701002E
:107000009387877CEDB797570100938727CB1CCCDC
:1070100097570100938787CBD9BF85E1EFA2FFD1B6
:10702000004618448347940075839D8B6315F700D1
:10703000EF00501C48C46FA09FD28280EFA25FCEA9
:1070400013893500C16442094111AA890144F11430
:1070500013590901054A2EC6EF00D077B2456346A1
:10706000A400014541016FA0FFCE83A709001317BB
:107070001400BA9783D707006388B700639497001A
:1070800063742A010504C1BF0545E9BFEFA27FC8AB
:10709000AA892E89328BB6843A8ABE8AEF80204C28
:1070A00055C12685EF1030368D4763E5A7007D5525
:1070B0006FA0BFC983DB4400EF00D0772A84EF00C4
:1070C000B0789307740031443305850263C5A70285
:1070D000EF005076EF0010762A84EF00F0769307E9
:1070E000740031443305850263CDA702EF0090742C
:1070F0009307450019A8EF00307533058502130783
:10710000F0179307C017E357A7FC2D55E3C277FB91
:1071100063000B02D6865286A6854A85EFE010638F
:1071200041BFEF007072330585029307C5FFF1BFC1
:10713000832749001385C90083D52700EFF01FF08E
:1071400071F9B5B76955ADB797F7FF1F2394A7A09D
:1071500097F7FF1F9387C79F904381470C463307DC
:10716000F500420741836393B70082805446139829
:1071700047008507C2962390E600D5B797F7FF1F13
:107180009387079D9C4303C58700828017F5FF1FE7
:107190000355459C8280EFA25FBAC1671387D7FF72
:1071A0006307E5026368A700F117630EF500014568
:1071B0006FA0FFBA1387E7FF630EE500FD171D8D73
:1071C00013351500F5B7EF40003D7D15D5BFEF40F5
:1071D000801AE5BFEF40E018CDBFEFA21FB6411106
:1071E000AA8401442EC6EF00F05FB2456346A400B6
:1071F000014541016FA0BFB69C48131514003E9590
:1072000083570500E387B7FE0504E9BF034855002F
:10721000814693F7F60F63E5070181473E8582803B
:10722000584593975600BA9703D727006316B700BF
:1072300003D70700E304C7FE8506E1BF8346450088
:1072400001479377F70F63E4D700814711A81C45E6
:10725000131657000507B29703D60700E313B6FECF
:107260003E858280EFA2DFAB93170501C18797FAB5
:10727000FF1F938AEA8D6355F00883A70A00C04771
:107280009C4703570400198D420541816366F50050
:10729000014422856FA01FAC12052A94DDBFDC4794
:1072A00013944900014A3E94834744006341FA0223
:1072B000014A834754006347FA028509C20993D9FA
:1072C000090183A70A009847E3EBE9FCD1B71C4406
:1072D00013195A00A6853E994A85EFF01FF011ED6B
:1072E000050AD9B75C4413195A00A6853E994A8508
:1072F000EFF0BFEE19E1050A6DBFE30009FC51BFD5
:10730000AA8481497DBFEFA25FA31C452A8481E73F
:107310009307C5001CC51C44231204001CC093071E
:10732000F00F63E9B70093F5F50F2285EF10B01366
:107330006FA0FFA293940501C167C18063F7F500B8
:10734000A6852285EF10D015E5B7C18193F5F50F1D
:107350002285EF105011A6852285EF101012C9BFAB
:1073600097E7FF1F9387C77E884382801C4599C794
:1073700097E7FF1F23AEA77C014582807D55828061
:1073800097E7FF1F9387C77C98438347450048478B
:1073900092073E958280EFA25F9A617100451C18AA
:1073A0003EC6B70780013EC81C183ECA835744003A
:1073B00002CE02D002CC231EF100834784002A892A
:1073C00002D22301F1023C083ED402D6EFF05FFB6B
:1073D000835705002316F102EF30706B2307A102DB
:1073E0005C4003556400F18313F717008347F102F3
:1073F00052055181F99BD98FA307F102EFE0702666
:1074000039C5AA8403550500EF80401683D70400D0
:107410002AD26800231CF10083D72400231DF10029
:107420001C4803D647008C43EF1010028347B4007A
:10743000CA86174601001306A6318117A305F4007A
:107440006C004810EFE090305D616FA05F912155B6
:10745000E5BF1C45B1CF03C5A7008946135765009A
:10746000630BD7028D46630ED70285466300D702B1
:10747000130740063305E50203C7B700418B15CB60
:1074800083C7B700BD8B3355F54082801375F50374
:107490001307803EC5B709671375F5031307077116
:1074A000D1BF372709001375F5031307077CD9B738
:1074B00001458280EFA27F8803A985006305090446
:1074C0008347B900AE8493F7070E91CF0345990027
:1074D000930520030D810505B305B50288446105B8
:1074E000EFF0B0320DA02E85EFF0BFF62A8401CD6B
:1074F00011238325C900B307B54063F887002E9494
:10750000B305A440E1FD6FA09F858545C1BFEFA2F3
:10751000DF822A8403D50500011132C636C43AC27F
:107520002EC002CA02CC02CEEF80400482452ACA95
:1075300022852ECCEFF0DFE403570500231EE10087
:10754000EF30F054A24632469247230FA10036870F
:107550004C08B28622850146EFF05FB305616FA04B
:107560001F80EFA28FFD61711C183EC6B707800116
:107570003EC81C183ECA3C0800453ED4AA8402CC32
:1075800002CE02D002D202D6EFF09FDF8357050071
:1075900035592316F102EF30904F2307A10209C499
:1075A0008357440091E721594A855D616FA02FFB05
:1075B0000355640052055181EFE0B00A2A8965D570
:1075C0008347B40093F7070E89C713058401EFF0D2
:1075D000502583574400231EF10083478400230174
:1075E000F1025C4003550900D98313F7070883476C
:1075F0001102231CA10093F7F707D98FA300F10212
:1076000083572900231DF1005C40F18313F7170015
:107610008347F102F99BD98FA307F102EF70107530
:107620002AD251D1834794006800139757008347AB
:10763000B400FD8BD98FA305F4001C4803D6470086
:107640008C43EF106060A6871747010013074710AF
:10765000740005464C102685EFF05FA32A8929D5D2
:107660008347B400A685FD8BA305F400EFF09FE4EB
:1076700025BFEFA28FEC832485FE2A844111268545
:10768000EFF03FDD834734FF93F7070E9DC32AC613
:107690002685EFF05FD019C9834734FFB245FD8BD3
:1076A000A309F4FE81C52285EFF0301641016FA0D9
:1076B0000FEB6DDD8327C4FF2685829765F983472D
:1076C00034FF93F7070E81C72285EFF0901503254D
:1076D00084FEEFF01FE9D9BFEFA22FE39C414111D7
:1076E0002A8903C7070089472E8493566700638C55
:1076F000F6020D466382C6049307F0076302F702A1
:107700002E85EF10A060AA848149C16B130C49003B
:1077100097E7FF1F9387C7439C43984763ECE902B1
:1077200041016FA04FE203D745008547E3FAE7FE2A
:107730002E85EF108061C1BF03D74500E3F2E7FE5D
:107740002E85EF10A05CAA842285EF10805DC20414
:10775000C98C5DBFDC470355A900139A49003E9AC6
:1077600093170501C187635DF00083570A00639595
:10777000A70263E574038327CA00034D5A001DA0C6
:10778000A1672167A98F1307F7EFE374F7FE6395ED
:107790000900EFF05FA071FD85099DBF83278A0076
:1077A000034D4A00835DA90003576900216A138BCA
:1077B000C7003AC6814A33CA4D01631E5D0197E78F
:1077C000FF1F938767399C43E1DBA2866286814570
:1077D00026858297D1B7A1679387F7EF930C4BFF6C
:1077E00063F04703B2455A85EFF05F8519CD032753
:1077F0008B00104719CA10436380C4023107D5BFFC
:10780000EE856685EFF07F9D71FD93861A0093FAF1
:10781000F60F130B0B0255B7835644005C43E3EDA0
:10782000F6F622853AC6EF10603DA1679387D7042C
:107830002A8A035D4400324763E897008347D900F2
:1078400093E707F8A306F9001C4766852286E285C0
:107850008297C1670844FD17337AFA00529508C031
:107860002312A40115BF97E7FF1F9387672E984344
:10787000814715C31447814763FFD500939745009F
:107880004C47BE9519C903C7550081476375E6008B
:10789000DC451606B2973E85828003C745008147C6
:1078A000E37BE6FE16069C45F5B7EFA26FC7AA89F3
:1078B0002E8A814497EAFF1F938A8A2983A70A00A8
:1078C000984763E4E4006FA0EFC8DC4713944400DA
:1078D00001493E9413BB140083474400634BF900F5
:1078E000014913BB140083475400634FF90085041A
:1078F000F1B70844931759005287DA860146A285EA
:107900003E9582990509C9BF48449317590052878B
:10791000DA860546A2853E9582990509E9B7EFA268
:10792000CFC1814517F5FFFF1305255F97E7FF1FBF
:1079300023920722EFF07FF76FA06FC297E7FF1F38
:10794000938707219C4381CFEFA22FBF814517F575
:10795000FFFF1305855CEFF05FF56FA04FC08280DD
:10796000EFA20FBC37E404008327841241112315D2
:10797000E100AE893289368A3A8681460147ED4573
:10798000AA8482972AC621C50356A100D285EF108A
:1079900061258327C413CE8526858297058915C561
:1079A0008327440D2314210101462C00268582974C
:1079B0002A8401C9B7E7040083A7C712ED45280050
:1079C0008297228541016FA0EFB84944E5B765541D
:1079D000CDBF5C41FD175CC18280EFA20FB6B7E757
:1079E0000400FC5F829795473305F50281450D81C0
:1079F0006FA0EFB6EFA26FB4B7E70400FC5F829709
:107A000095473305F5020D816FA06FB5EFA2EFB278
:107A1000B7E7040083A7870B0355050082976FA083
:107A20000FB4EFA28FB1035505003287AE8617B6AB
:107A3000FF1F0356C66A97E5FF1F93852512EFF0D7
:107A40003FF26FA0CFB1EFA24FAFB7E7040083A71B
:107A5000C71782976FA0AFB0EFA22FAEB7E70400B1
:107A600083A7871397E5FF1F9385450F82970145ED
:107A70006FA0EFAEEFA26FACB7E7040083A7C71FFC
:107A8000814517B5FF1F0355856182976FA02FAD04
:107A9000EFA2AFAAB7E7040083A7871397E5FF1FFC
:107AA0009385C50C829701456FA06FABEFA2EFA83D
:107AB000B7E7040083A7C71F814517B5FF1F03550C
:107AC000056482976FA0AFA9EFA22FA72E85EF6064
:107AD0000055EF60900D6FA08FA8EFA20FA6EF608A
:107AE000D0176FA0CFA75C49E1175CC95CC583576D
:107AF0002501A1072319F50083570501A1072318C4
:107B0000F5008280F1473305F50297E7FF1F938761
:107B1000E7079C433E9582808D476317F60603D79F
:107B20004600854763F2E706EFA22FA1368536842B
:107B30002E89EF10A01D39C183574400931405010D
:107B4000C18063ED97022285EF10401CFD142312C3
:107B500094009307A002630EF5009307B00263013F
:107B6000F50293079002631BF5002285EFC0B07EFB
:107B700031A00146CA852285EF80000F6FA02F9E9D
:107B80002285EF001059DDBF828097E6FF1F9386A4
:107B900026009C42014599CF9843D44217E6FF1F27
:107BA0002328E6FE6396D70097E6FF1F23A4E6FE90
:107BB0001385C7FE8280EFA24F98E92671443305F2
:107BC00085029145EF70606201E565556FA02F99C0
:107BD00097E7FF1F23AAA7FA75263305850291456B
:107BE000EF70A0607DD197E7FF1F23A1A7FA592E60
:107BF00097E7FF1F2394A7F8712697E7FF1F2390AD
:107C0000A7F8974701009387E7B917E7FF1F232BD2
:107C1000F7F697070000938747ED17E7FF1F23212B
:107C2000F7F6014565B7EFA24F91AA8517E5FF1F4B
:107C30001305C5F4EF1060216FA06F92EFA2EF8FD4
:107C4000EFF07FFEEF10E02197E7FF1F938747F4E7
:107C50009C4381CF1387C7FE09CB83D5C7FF17E5A8
:107C6000FF1F130565F3EFF0403A6FA04F8FEFA2AF
:107C7000CF8CEFF09FF119C9834785002A8493F7D1
:107C8000070499E70355E500EFF05FFB6FA02F8D28
:107C90008347C5009304450117E9FF1F130949EF06
:107CA00085E3832709005CC997E7FF1F23A297EEAE
:107CB00083274900E1FF97E7FF1F23AD97ECF9B752
:107CC000FD172306F5006105EF60E07E8307840061
:107CD00063CB07048347840093E707F82304F40089
:107CE000B7E704009C5F82974205A947418133753D
:107CF000F5028347840093F707FCC98F2304F4003F
:107D00008347D4003E951C402318A40089CF984394
:107D100019CB8347C4005040814585073305F502E0
:107D2000420541810297832709005CC897E7FF1F3E
:107D300023A097E68327490089E797E7FF1F23AB36
:107D400097E48347C400B9D38355040117E5FF1FA7
:107D5000130585E4EFF0602B15BFEF921FFE97E748
:107D6000FF1F9387A7089C4701448583858B81EF7C
:107D7000AE84B2853A86EF1020142A8409C5EF102C
:107D8000200B829408CC22856F907FFDEF925FF9E3
:107D900041112E8932C6AA89712C32471306050279
:107DA000CA8697050000938525D617E5FF1F1305A2
:107DB000E5DCEFF09FFA2A8429CD9304C5006526FF
:107DC0001946AA852685EF00306885452685EF008F
:107DD0001065174501001305A59A4E9583450500CA
:107DE0002685EF0050685C4831468145A1075CC894
:107DF0005CC483572401E1172319F400835704015D
:107E0000E1172318F4001C4C3E85EF901FF6A304E5
:107E10002501228541016F90FFF3EF921FF241117E
:107E2000AA842EC632C4EF100003004DB24522468C
:107E3000834784000CC050C093F7F70393E707040F
:107E40002304F400231804002685EF00707E834786
:107E50009400A9462317A40013D73700050733075A
:107E6000D7029D8B85072306F400A306E40083C791
:107E70000401D8488507230FF7FE17E7FF1F1307F4
:107E800027D15843232A0400930744011DEB17E729
:107E9000FF1F2321F7D017E7FF1F232BF7CE17E48F
:107EA000FF1F130464CF2285EFF0A00B1C44858BC9
:107EB0005D8D09E581452285EFF0201541016F9028
:107EC0001FEA1CC317E7FF1F2326F7CCC9BFEF9299
:107ED000DFE697050000938565C40145EFF0DFBE3E
:107EE00001456F90DFE7EF925FE5EFF01FBF6F9006
:107EF0001FE78347C500A1E7EF923FE42A840355BB
:107F0000E500EFF05FD215C98347840093F7F7FBD4
:107F10002304F4001C4091C7DC4381C74C40014559
:107F20008297EFF09FC617E5FF1F1305E5C6EFF038
:107F3000400F0355E400EFF07FD06F905FE2828046
:107F4000EF92BFDF97E7FF1F938787C49705000075
:107F5000938525D217E5FF1F130505C423A007004D
:107F600023A20700EFE0507E6F907FDF1C4D91CB86
:107F7000DC4381CBEF927FDC8345070082976F90D3
:107F80001FDE828097E7FF1F938747C39C4303C58B
:107F90000700828097E7FF1F938747C29C4303C572
:107FA0001700828097E7FF1F938747C19C4303C553
:107FB0002700828097E7FF1F938747C09C4303C534
:107FC0004700828097E7FF1F938747BF9C4303C505
:107FD0003700828097E7FF1F938747BE9C4303C506
:107FE0005700828097E7FF1F938747BD9C4303C5D7
:107FF0006700828097E7FF1F938747BC9C4303C5B8
:108000007700828097E7FF1F938747BB9C4303C598
:108010008700828097E7FF1F938747BA9C4303C579
:108020009700828097E7FF1F938747B99C4303C55A
:10803000A700828097E7FF1F938747B89C4303C53B
:10804000B70011E11D45828097E7FF1F938707B7AF
:108050009C4303C5C700828097E7FF1F938707B63D
:108060009C4303C5D700828097E7FF1F938707B51E
:108070009C4303C5E700828097E7FF1F938707B4FF
:108080009C4303D50701828097E7FF1F938707B3BF
:108090009C4303C52701828097E7FF1F938707B2A0
:1080A0009C4303D54701828097E7FF1F938707B161
:1080B0009C4303D56701828097E7FF1F938707B032
:1080C0009C4303D58701828097E7FF1F938707AF03
:1080D0009C4303C5A701828097E7FF1F938707AEE4
:1080E0009C4303C5B701828097E7FF1F938707ADC5
:1080F0009C4303C5C701828097E7FF1F938707ACA6
:108100009C4303C5D701828097E7FF1F938707AB86
:108110009C438857828097E7FF1F938727AA9C4339
:1081200003D5C702828097E7FF1F938727A99C4347
:1081300003D5E70219E11305800C828097E7FF1F42
:108140009387C7A79C4303C50703828097E7FF1F58
:108150009387C7A69C43C85B828097E7FF1F9387DE
:1081600067A58843828097E7FF1F9387E7A488432A
:10817000828019E17D558280F5DE984265DFFDD968
:1081800017E7FF1F130787C61847AA877155058B86
:108190006319072203C507001547E37DA7FC03C742
:1081A00037001305F0057D171377F70FE364E5FC3F
:1081B00003C35700E30003FC83C86700E38C08FA9D
:1081C00003C77700494579171377F70FE364E5FA9A
:1081D00003C7A70011481305F7FF1375F50FE36BED
:1081E000A8F803CE97000D481305FEFF1375F50F91
:1081F000E362A8F803C8B70063090800651813789C
:10820000F80F1305600DE36705F703C5C70079484C
:1082100079151375F50FE36FA8F403C8D7000D4562
:108220007D181378F80FE36705F503D80701930E5F
:1082300040175118420813580801E3ED0EF303C824
:10824000E7007D181378F80FE36605F303C82701EC
:108250007D181378F80FE36F05F103C88700C54E4A
:1082600075181378F80FE3E70EF103D86701856EF0
:10827000938EBEE06D18420813580801E3EC0EEF30
:1082800003D847016D18420813580801E3E40EEFC4
:1082900003D887017918420813580801E36C05EDEB
:1082A00003C8A7017D181378F80FE36505ED03C532
:1082B000B7011D487D151375F50FE36DA8EA03C5D9
:1082C000D701714879151375F50FE365A8EA03D551
:1082D000E7011308E00F7D1542054181E36CA8E832
:1082E00003C50702494879151375F50FE364A8E83B
:1082F000C85301C937C834005915130858BFE36B78
:10830000A8E603A8870237C53400130555BF5918DE
:10831000E36205E717E5FF1F2320C58A03C60501B1
:1083200017E5FF1F232CF5880545E375C5E403D841
:108330002501D04933760603E31E06E203C6150184
:10834000E30A06E217E6FF1F2326B68683C5270049
:1083500001466387A50003C61700F1453306B60240
:1083600083C707039305C00272971A071307C7054F
:1083700016031A9796084697B387B70241553E975A
:10838000329742074183636EE802EF921F9B368566
:10839000EF60D06FEFD0B0212A84EF80B01D2A9417
:1083A000EFC090252A94EF7040072A94EFF0BF8029
:1083B0002A94EF2050632A94EF50406622956F90E4
:1083C0001F9A8280EF927F974111A307A100EF804F
:1083D000801E9305F10017050000130565B9EFF045
:1083E000CFCC014541016F909F97EF929F9217E488
:1083F000FF1F1304A49F0328840079599368180071
:1084000097E4FF1F23A8149F13781800631E080029
:10841000BA84BE89368B328A2E89AA8AEFE01FD6AB
:108420007D15269509E531594A856F901F92EFE039
:10843000FFD47D152695A167E357F5FE97E7FF1F4B
:108440009387C7D198433E8C814B11C70145EFC03C
:10845000B03E933B15004A85DA865686D285EF708A
:1084600070372A8911CD1C44F99B17E7FF1F23237E
:10847000F79883270C00CDDBE3880BFA82976DB762
:10848000268597E7FF1F23A50796EFE0FFCB414620
:10849000CE8517E5FF1F1305E59EEF00A174EFA041
:1084A00070080325040BEFA0700A0545EFA07010BB
:1084B0000545EFF03FF18DBF97E7FF1F93870793C7
:1084C0009C47858BD5C7EF925F8717E5FF1F130584
:1084D000A59997E7FF1F23AB079097E7FF1F23A9F5
:1084E000079097E7FF1F23A70790EFE09033EF4037
:1084F000C002EFE0F00AEFE0700F97E7FF1F9387ED
:10850000678D9C4381C70545EF60B03397D7FF1F48
:10851000938707769C4389C741657D15EF50A06B13
:10852000EFC0703AEFA0F00097E7FF1F938707A115
:108530009C431397170163540700EFC0A04597E7CA
:10854000FF1F23A1079497E7FF1F23AF079297E729
:10855000FF1F23AD079297E7FF1F23AB0792EFF0B2
:108560009F984923EFF0AFBBEFC080676F902FFF5C
:10857000828097E7FF1F9387678788438280EF9207
:10858000CFFBEF60B07EEF7080006F904FFDEF92F9
:108590002FF92A849304140201112E85B289A6852D
:1085A000214636C63A89EF0081611DE1B24638089E
:1085B0002686CE8513059404EF40604321462C089F
:1085C0004A85EF00C15F1335150005616F908FF884
:1085D0000145E5BFEF926FF69305450617D5FF1FDE
:1085E0001305055EEFE070226F906FF7EF92EFF4E6
:1085F00041112EC6EFF00FC0B24588C141016F9006
:108600000FF6EF92EFF1AA842E84EF605078AA89DA
:1086100085452285892D83C7E4011389940899E350
:1086200013890403CE8522853D2D21469305190229
:108630002285192D97D7FF1F9387477B8C4322856F
:10864000EF00E0682146938584022285F52B6F9028
:108650006FF0EF920FEC3971EFC0E04E93054006DA
:1086600045EDEF60D06F630E051097D7FF1F83C7EE
:10867000E75613B7170097D6FF1F2381E65601442C
:1086800089CFC16417D9FF1F130949769309400E9A
:10869000FD14EFF03F986348A408EFF0AFB54169CF
:1086A000B7290900096AFD7A2A8B81447D199389CB
:1086B000F97B130A0A71938A8AC7EFF0BF9563D5D5
:1086C000A4041304400EB387840217D7FF1F1307B7
:1086D000E7710324070B3E948357C401638627097F
:1086E00018403307EB4063EAE900834744008507FD
:1086F000B3874703D6976369F70601468145094565
:10870000EFF0CFE8AA8B29E1EF20105A8547631FCD
:10871000F50489659385057117D5FF1F1305454A33
:10872000EFE0B00EA1A8B30734030327090BBA97F3
:1087300003D7C7016308970003C75700A382070048
:108740002382E7000504B1B79305C5002285EFF049
:108750005FEB5E852286973501009385A503EFF0D8
:10876000CFEB5E85EF00E06F850481BF97D7FF1FD9
:108770009387C7679C478D83858BC1FF21616F906D
:10878000CFDC01468545094502D002D202D402D68B
:10879000EFF0CFDFAA847DD1EFC0203A1389C40067
:1087A0002A8481454A85C1210C4041464A85692970
:1087B00083294400638809084E8502D802DA02DC66
:1087C00002DEEF00816A2ACE141005462C08081834
:1087D0004ECCEF4060191375F50F2DE583558400DD
:1087E00093E525004A856D2911460C104A85A92973
:1087F000014697350100938565FA2685EFF0EFE194
:108800002685EF0000665C40B5DB014685450D45D9
:10881000EFF0CFD7AA843DD148401389C400EF00C0
:10882000C1642AC64A85C5263246636AC5004C40E3
:108830004A851929014681452685EFF00FDE2685F8
:108840000D252DBF8355840071BFEF920FCF97D7B1
:10885000FF1F9387A7599C4719CD93E7870017D52A
:10886000FF1F1305E53517D7FF1F2325F758EFE046
:1088700060786F90CFCEDD9B17D7FF1F232CF75664
:10888000EF2090427DF517D5FF1F13056533EFE00C
:108890004079C5B7EF92EFC74169AA892E8AB28A9B
:1088A000368BBA8B814417DCFF1F130C2C54930CAE
:1088B000400E7D19EFF00FF663C4A40001442DA013
:1088C0003384940383270C0B3E948357C401638045
:1088D00027055A87D6865286CE8513050403EFF006
:1088E0001FCB11C523800B0022856F900FC68347D5
:1088F000F40191CF5A87D6865286CE851305940807
:10890000EFF0FFC809C585472380FB00F1BF850450
:1089100055B783574500638D0716EF926FC001115D
:108920002A84ED2619C58547630AF50405616F9011
:108930006FC2EFC040217DF9835744004947ED9B4A
:10894000E396E7FEC14522854524AA842285F52EBB
:108950000357440002CE91472A896317F700228506
:1089600039293C082ACC3ECEEFC0201D5C55DDDF06
:1089700074084A86A685054582974DBF0357440073
:10898000D147E3F5E7FA032A0400C169014997DA00
:10899000FF1F938AAA45130B400EFD19EFF08FE7D6
:1089A0006344A90C2285032A04008D26A1452A8947
:1089B00022851D2CAA842285D92614402A86AA89BC
:1089C00078082685CA85EFF0FFECAA8425D103C775
:1089D000F40189476315F7008347C101A1DB5546C0
:1089E000D28513856400EF00E11F0145EF60103868
:1089F00001C583D7C401B1EB97D7FF1F9387073F0A
:108A00009C4793551900858913D73700058B11CBE7
:108A10008983858B6397B70001452EC6EFF0FFE28F
:108A2000B2454E85EF60703C0346C1012A849375C0
:108A300019002685EF70703131C92685EF607037D7
:108A4000268511C00145EF60D061EF20F0258547F4
:108A5000E31EF5EC83C754001307F00FE388E7EC3F
:108A60008507A382F400D9B5B304690383A70A0B71
:108A7000BE9483D7C401638937015546D2851385D7
:108A80006400EF00C11371D1050909BF5DDC5DBF52
:108A90008280EF92EFA8EF60902C11CDC164014469
:108AA00017D9FF1F130989349309400EFD14EFF005
:108AB0006FD6634AA40017D5FF1F13056510EFE0BA
:108AC00060536F902FA9330534038327090B3E951C
:108AD0008357C5016386970023120500EF60702D50
:108AE0000504F1B797D7FF1F938747309C478D83C5
:108AF000858B99EBEF926FA417D5FF1F1305450CDB
:108B0000EFE020526F90AFA58280EF920FA3970500
:108B10000000938545B417D5FF1F1305650AEFE0E4
:108B2000A0426F90CFA3EF924FA18841B7E7040016
:108B3000BC5B050542054181829709C58547230035
:108B4000F50005056F90AFA183C7F5FF2E8585075A
:108B5000A38FF5FE828083C7F5FFFD1793F7F70F0C
:108B6000A38FF5FE99EBEF924F9DB7E70400BC573A
:108B70001385F5FF82976F908F9E82801C4103576B
:108B800045008D8FBA951CC12312B5003E858280A9
:108B900093D78500A2051441DD8D835745001387C7
:108BA000E6FF18C189072312F50013D6850041118D
:108BB000238FB6FEA38FC6FE410182801841930722
:108BC000F7FF1CC18357450085072312F500A30F4B
:108BD000B7FE8280835745008D8F2312F5001C411C
:108BE000BE950CC12E858280AA8703D74700084115
:108BF0000D8FAA952392E7008CC382801841084507
:108C00003305A740828083574500035765001D8FB9
:108C10001C4108453385A7403305A7408280EF9269
:108C2000CF9141112EC62A84EFF0FFFDB245637348
:108C3000B50001A0835744000840BE952312B4003C
:108C40003E9541016F90AF91EF922F8F41112E848D
:108C5000B28532C6EFF0BFFC3246A285EFF09078C5
:108C600041016F90CF8FEF924F8D2E848545EFF0AD
:108C70001FFB230085006F908F8EEF920F8C4111A8
:108C80002317B1008945EFF09FF98347E1002300E6
:108C9000F5008347F100A300F50041016F902F8C90
:108CA000EF92AF8993D78500A2054111DD8D23177F
:108CB000B1008945EFF0BFF68347E1002300F500DE
:108CC0008347F100A300F50041016F904F89EF92B7
:108CD000CF861397850193D78501C166938606F0E9
:108CE000D98F13D78500758FD98FA2053707FF005D
:108CF000F98D4111DD8D2EC69145EFF05FF26C00CC
:108D00001146EFF0306E41016F906F85EF92EF8268
:108D10001C41854503C40700EFF0DFEB22856F900F
:108D20000F84EF928F811C414111894503C70700D1
:108D300083C717002307E100A307F100EFF09FE9C5
:108D40000355E10041016F908F81EF821FFF1C41AD
:108D50004111894503C7070083C717002307E100B6
:108D6000A307F100EFF01FE78357E100410113D59E
:108D70008700A2075D8D420541816F805FFEEF8213
:108D8000DFFB0C4141112A8411466800EFF0906529
:108D900091452285EFF01FE4B247C166938606F045
:108DA0001397870113D58701598D13D78700758FC6
:108DB000598DA2073707FF00F98F5D8D41016F8044
:108DC0001FFA1C45BE950CC18280AE87944391E684
:108DD000584101EF0CC15CC1828003C75700136783
:108DE0001700A382E700B687D5B70CC3EDB7AA87F3
:108DF000084119CD1841D44398C36313D500D8C393
:108E00002A87034657009376160081E62320070041
:108E10008280944381CA8C4203A847008CC3639329
:108E20000601CCC3799A14C3A302C7003687D1BF09
:108E30001C45DC471D8DB777DBB6938777DB09854B
:108E40003305F502420541818280F147B385F50281
:108E500048452E9582808347450085072302F5000B
:108E60008280EF829FED2A8419E06F805FEF834755
:108E70004400E5DFFD1793F7F70F2302F400F5F741
:108E80001C4403D7270005072391E700DC4399C35F
:108E9000228582974C4889CD83475400898B99E776
:108EA0001C4422859C479C439C478297232A0400AC
:108EB0000040232004004DBFEF823FE88357250088
:108EC00041112EC691E70144228541016F803FE99F
:108ED000035705008147F146E307F7FEB385D70244
:108EE000404585072E948345440008C4F5F5B247F4
:108EF000AA8481E7232A040009A81C456C00228566
:108F00009C439C43829748C85DDD85472312F4004B
:108F1000B24723200400231804002319F4005C48FE
:108F20005CC483D72400FD172391F40071BFEF8246
:108F3000DFE097D7FF1F9387A7CA88432326050042
:108F4000232405004105EFE0C00D6F805FE1EF8253
:108F5000DFDE17D4FF1F1304A4C81C40411189CFC2
:108F60009C472300B5002AC65CC1EFF05FFC1C40A3
:108F7000DC4399C33245829741016F805FDE03472E
:108F800045001DEB584DAA877D550DCBEF82FFDACA
:108F90001CC3DC4797D6FF1F23A4E6C4F156130574
:108FA00007012390D7009705000093858501EFD036
:108FB000B07901456F80BFDA7D5582808280EF8273
:108FC000DFD70111614681452800EF801FDA97D76E
:108FD000FF1F9387E7C09C4328009305F00FDC47F1
:108FE0003EC6EFF0DFF605616F807FD797D7FF1F92
:108FF000938707BF9C43D847A1679387C702631233
:10900000F70A397106DE22DC26DA80004AD84ED60D
:1090100052D456D23285B284EFF05FCFAA8926852A
:10902000EFF03FD02318A4FC2685EFF09FCF231943
:10903000A4FC2685EFF0FFCE83D744000A8A231ACA
:10904000A4FC858393F7F70F230EF4FC8607BD0776
:1090500093F7073F3301F1408A8A01498347C4FDF2
:109060006365F902CE85130584FC232C54FDEFF0D3
:109070001FEE5281130104FCF2506254D254425943
:10908000B259225A925A216182802685EFF07FC917
:1090900093171900D69705092390A7001379F90FA4
:1090A00075BF828097D7FF1F938787B39C43D847AC
:1090B000A1679387A7026310F70A397106DE22DCE5
:1090C00026DA80004AD84ED652D456D23285B2849F
:1090D000EFF0DFC3AA892685EFF0BFC4FD57231840
:1090E000A4FC26852319F4FCEFF0BFC383D744000A
:1090F0000A8A231AA4FC858393F7F70F230EF4FC46
:109100008607BD0793F7073F3301F1408A8A01497B
:109110008347C4FD6365F902CE85130584FC232CC7
:1091200054FDEFF0DFE25281130104FCF25062546F
:10913000D2544259B259225A925A216182802685CC
:10914000EFF03FBE93171900D69705092390A700AB
:109150001379F90F75BF828097D7FF1F938747A8B0
:109160009C43D847A16789076318F708397106DE61
:1091700022DC26DA80004AD84ED652D456D2328526
:109180003289EFF0BFB8AA894A85EFF09FB98357BB
:1091900049000A8A2318A4FC858393F7F70F230C50
:1091A000F4FC8607BD0793F7073F3301F1408A8A35
:1091B0008144834784FD63E5F402CE85130584FC76
:1091C000232A54FDEFF0BFD85281130104FCF25062
:1091D0006254D2544259B259225A925A2161828021
:1091E0004A85EFF01FB493971400D6978504239017
:1091F000A70093F4F40F75BF828097D7FF1F938762
:10920000279E9C43D847A1679387E7046312F70A18
:10921000397106DE22DC26DA80004AD84ED652D4D6
:1092200056D23285B284EFF07FAEAA892685EFF060
:109230005FAF2318A4FC2685EFF0BFAE231AA4FC71
:109240002685EFF01FAE83D744000A8A2319A4FCB9
:10925000858393F7F70F230EF4FC8607BD0793F77A
:10926000073F3301F1408A8A01498347C4FD6365A2
:10927000F902CE85130584FC232C54FDEFF03FCD7D
:109280005281130104FCF2506254D2544259B25933
:10929000225A925A216182802685EFF09FA8931767
:1092A0001900D69705092390A7001379F90F75BF08
:1092B000828097D7FF1F9387A7929C43D847A167C7
:1092C0009387C7046310F70A397106DE22DC26DAB9
:1092D00080004AD84ED652D456D23285B284EFF0AE
:1092E000FFA2AA892685EFF0DFA3FD572318A4FC6F
:1092F0002685231AF4FCEFF0DFA283D744000A8A04
:109300002319A4FC858393F7F70F230EF4FC86073B
:10931000BD0793F7073F3301F1408A8A014983472C
:10932000C4FD6365F902CE85130584FC232C54FD2E
:10933000EFF0FFC15281130104FCF2506254D25489
:109340004259B259225A925A216182802685EFF001
:109350005F9D93171900D69705092390A7001379ED
:10936000F90F75BF828097D7FF1F938767879C434C
:10937000D847A167DD07631BF702EF821F9C797155
:1093800032853284EFF09F982AC62285EFF07F99CC
:109390002311A1022285EFF07F97B2452300A1029D
:1093A0002808EFF0DFBA45616F807F9B828097D7F6
:1093B000FF1F9387E7829C43D847A1679387870461
:1093C000631BF702EF827F97797132853284EFF069
:1093D000FF932AC62285EFF0DF942311A102228594
:1093E000EFF0DF92B2452300A1022808EFF03FB66C
:1093F00045616F80DF96828097C7FF1F9387477E06
:109400009C43D847A1679387A704631CF700EF82AA
:10941000DF92011128008145EFF07FB305616F8075
:109420001F94828097C7FF1F9387877B9C43D847F1
:10943000A167938757026311F702EF821F90011112
:109440003285EFF0BF8C2308A10081452800EFF0A2
:109450001FB005616F80BF90828097C7FF1F938701
:1094600027789C43D847A1679387E702631FF702D9
:10947000EF82BF8C011132853284EFF09F8AAA847B
:109480002285EFF01F8A854719E52285EFF01F88B6
:109490004205B337A00028008145231891003ECA39
:1094A000EFF0FFAA05616F809F8B828097C7FF1F37
:1094B000938707739C43D8479947631FF704EF824C
:1094C000DF87797132853284EFF05F842AC6228586
:1094D000EFF03F852310A1022285EFF03F832301A7
:1094E000A1022285EFF09F82A301A1022285EFF065
:1094F000FF812302A1022285EFF05F812313A102E5
:109500002285EFF0BF80B2452314A1022808EFF0B6
:109510001FA445616F80BF84828097C7FF1F938718
:10952000276C9C43D847A1679387C703631FF70441
:10953000EF82BF80797132853284EFF02FFD2AC629
:109540002285EFF00FFE2310A1022285EFF06FFDC0
:109550002311A1022285EFF06FFB2302A1022285D5
:10956000EFF0CFFAA302A1022285EFF02FFA230336
:10957000A1022285EFF08FF9B245A303A1022808CA
:10958000EFF0FF9C45616F808FFD8280EF82EFFAE4
:1095900001112A84EFF08FF7AA842285EFF06FF88B
:1095A0002285EFF00FF8035744008D4763F5E7007D
:1095B0002285EFF00FF72285EFF0AFF62800A685A1
:1095C000EFF0FF9805616F808FF997C7FF1F9387B2
:1095D00027619C43D847A167FD076319F700EF8215
:1095E000CFF53285EFF09FFA6F806FF7828097C7D3
:1095F000FF1F9387E75E9C43D847A167E507631188
:10960000F706EF828FF3797132853284EFF00FF035
:109610002AC62285EFF0EFF02285EFF08FF02310BD
:10962000A1022285EFF0EFEF520551812311A10233
:10963000228523020102EFF06FEDA302A102228531
:10964000EFF0CFEC2303A1022285EFF02FECB2451F
:10965000A303A1022808EFF09F8F45616F802FF0D0
:10966000828097C7FF1F9387A7579C43D847A1675E
:109670009387E7036319F700EF822FEC3285EFF051
:10968000FFF06F80CFED828097C7FF1F938747550C
:109690009C43D847A167938747046314F702EF827E
:1096A000CFE9797132853284EFF04FE62AC6228500
:1096B000EFF02FE7B2452808EFF07F8945616F8012
:1096C0000FEA828097C7FF1F938787519C43D84733
:1096D000A167938787026316F702EF820FE679711D
:1096E00032853284EFF08FE22AC62285EFF00FE256
:1096F000B2452300A1022808EFF07F8545616F8005
:109700000FE68280EF826FE30111EFF02FE0AA8570
:109710002800EFF0DF8305616F806FE497C7FF1FBC
:109720009387074C9C43D847A167D1076319F7007B
:10973000EF82AFE03285EFF0FFFC6F804FE2828076
:1097400097C7FF1F9387C7499C43D847A167C507A1
:109750006319F700EF826FDE3285EFF0BFFA6F809A
:109760000FE0828097C7FF1F938787479C43D847A6
:10977000A167B9076319F700EF822FDC3285EFF09C
:109780007FF86F80CFDD828097C7FF1F93874745A3
:109790009C43D847A167AD076319F700EF82EFD963
:1097A0003285EFF03FF66F808FDB828097C7FF1F17
:1097B000938707439C43D84789476310F702EF829A
:1097C000CFD70111328532C8EFF04FD4AA852800D7
:1097D000EFF0EFF705616F808FD8828097C7FF1F8A
:1097E000938707409C43D847A1678D076317F7020B
:1097F000EF82AFD4011132853284EFF02FD11306FE
:109800006100AA844C002285EF20D00C2800A68598
:10981000EFF0EFF305616F808FD4828097C7FF1F51
:109820009387473C9C4381CBDC4391C7EF82EFD0C9
:1098300082976F80CFD28280EF822FD079713C08DF
:10984000AE843ED2A165B7070A002A843ED44810F0
:109850003C08DD053ED636C432C63AC2EFD0BFAAB8
:1098600012474810BA85EFF00FC032464810B28553
:10987000EFF0AFC0A2464810B685EFF0CFBE501053
:1098800001478146A6852285EFD07FC845616F805C
:109890000FCDEF828FCA01117C000329C501AE8470
:1098A0003ECAA165B70707002A843ECC48087C0061
:1098B000C5053ECEEFD03FA58345D9004808EFF05F
:1098C0008FBA500801478146A6852285EFD03FC454
:1098D00005616F80CFC8EF824FC683C7950093F7AD
:1098E000F707A384F500EFF0DFFA6F804FC7EF8230
:1098F000CFC479713C08AE843ED2A165B707090098
:109900002A843ED448103C08938545043ED632C68E
:1099100036C4EFD05F9FA2464810B685EFF0AFB4D3
:1099200032464810B285EFF04FB5501001478146DE
:10993000A6852285EFD0BFBD45616F804FC2EF8203
:10994000CFBF83C7950041112A8493F7F707A384FB
:10995000F50032852EC6EFF0CFBC85672AC4637C44
:10996000F500EF50B0402246B24509E91147814663
:109970002285EFF07FEC41016F806FBE0147834687
:10998000F501FDB7EF82CFB901113C003ECAB70720
:109990000A003ECC3C003ECE83C79500AA893285A2
:1099A00093F7F707A384F5002E84EFF08FB7856750
:1099B0006371F504A165AA84938585044808EFD0F6
:1099C0009F942685EF50903A2A891DE591454808D5
:1099D000EFF06FA9A6854808EFF02FAACA854808BE
:1099E000EFF06FA8014781465008A2854E85EFD061
:1099F0001FB205616F800FB681454808EFF0AFA632
:109A000003490902C1BFEF82AFB179711C103ECA90
:109A1000B7070F003ECC404D1C10AA84AE89480801
:109A2000994532C636893ECEEFD0FF8D3246480882
:109A3000B285EFF04FA363040902A5454808EFF093
:109A40000F9E2546CA85EFF0E01950080147814670
:109A5000CE852685EFD0BFAB45616F80AFAF835514
:109A6000C4024808EFF06FA10355E402814515C117
:109A700085478545630FF500C167FD179305F00F16
:109A80006309F5007D15EF5020749305150093F5DB
:109A9000F50F4808EFF02F9D834504034808EFF0C9
:109AA0008F9C834514034808EFF0EF9B83552403F4
:109AB0004808EFF08F9C835544034808EFF0EF9B74
:109AC00069B7EF828FA783C795008146014693F758
:109AD000F707A384F500EFF01FF36F804FA8EF8224
:109AE000CFA579713E841C103ECA2E89B7070F009E
:109AF000A1653ECCFD051C10AA84480842C03AC2AC
:109B00003ECE36C432C6EFD01F8032464808B285FA
:109B1000EFF06F95A2464808B685EFF00F96124712
:109B20004808BA85EFF06F95024863040802914532
:109B30004808EFF0CF8E1146A285EFF0A00A50083A
:109B400001478146CA852685EFD07F9C45616F809D
:109B50000FA189454808EFF08F8C8347040023004C
:109B6000F50083471400A300F500D1BFEF824F9B9F
:109B700083C7950001112A8A93F7F707A384F5009C
:109B80003285AE8432C6EFF0CF9932462A893285CB
:109B9000EFF0CF978567637FF900AA894A85EF5078
:109BA000F01C2A8419E9114781464A86A685528508
:109BB000EFF09FC805616F80EF999387E9FF93F7F6
:109BC000F70F0547E368F7FE8347F50195E78947F7
:109BD000E382F9FE8346F401528501474A86A68551
:109BE000EFF09FC5A167D90748083ECC230A0100C2
:109BF00002CEEFF0BFC27DBF639CE7008947639C44
:109C0000F90093071020231FF500EF50901AD9B7E1
:109C10000947E391E7FC8D47E39EF9FA2285EF506F
:109C2000D03B97C7FF1F9387E71A9C4399E797C7D5
:109C3000FF1F9387E7039C4389C703D50400EF60A8
:109C4000300C231F04002285C9B7EF820F8F01114A
:109C50003C003ECAB7070B003ECC3C003ECE83C75B
:109C600095002A89328593F7F707A384F500AE841F
:109C7000EFF02F8B93170501C187635EF004A16598
:109C80002A849385E5024808EFD0EFE7A2854808CB
:109C9000EFE0BFFE97C7FF1F938787FD9C439DEFB3
:109CA00001449375F40F4808EFE0FFFB935584409F
:109CB00093F5F50F4808EFE01FFB9355044193F52A
:109CC000F50F4808EFE03FFA014781465008A685A6
:109CD0004A85EFD0DF8305616F806F8841658546D7
:109CE0000546A2857D15EF3070675DD95105EFD02F
:109CF0004027130440063344850265B7EF82EF83A3
:109D00000111B70706003EC683C7950021642A8962
:109D100093F7F707A384F500AE8428009305A40405
:109D20000AC40AC8EFD02FDE300001478146A6855D
:109D30004A85EFD0CFFDEFE02FF8130494044808D4
:109D400022CC230A010002CEEFF05FAD05616F80E7
:109D50000F81EF72FFFCC1642A89014497C9FF1F7C
:109D60009389C908130A8002FD14EFE0AFAB634585
:109D7000A40001456F701FFEB307440303A7C90A7F
:109D8000BA9703D707006306970083D72700638439
:109D900027010504D9BF0545F1BFEF727FF82A8A74
:109DA0002E8999C123A005008149814497CAFF1FCC
:109DB000938A8AE3614BEFE02FAD63C5A4004E8523
:109DC0006F705FF93384640383A70A003E9483575E
:109DD000040099E763040900232089008504E1BF9A
:109DE0004146D28513054400EFE0705D65F9A28914
:109DF000F5B7EF72FFF239717C083ED4B7070A005D
:109E00003ED67C083ED883C795002A8A328593F7D0
:109E1000F707A384F5002E8932C6EFE09FF085672F
:109E20006373F5063246AA843285EFE03FEE85473C
:109E3000AA8963EAA704A165938585042810EFD059
:109E40008FCC2685EF5080722A8429E19145281015
:109E5000EFE07FE1A6852810EFE03FE2CE852810F5
:109E6000EFE07FE0014781463010CA855285EFD090
:109E70000FEAA1679387770448183EDC230A0102A2
:109E800002DEEFF0BF9921616F70DFEC8145281091
:109E9000EFE07FDDA6852810EFE03FDE97C7FF1FCC
:109EA0009387872B9C4391C7228563870900EFB076
:109EB000600C8345040265B7EFB0200BDDBFEF7285
:109EC0003FE683C795004111AA8993F7F707A3845A
:109ED000F5003285AE84328AEFE0BFE48567637BAC
:109EE000F5022A89EF5080682A84914621C1834770
:109EF000F50105476383E70291C70D47636EF702DB
:109F0000AD462DA09305050303250A004146EFE069
:109F1000104B1DE141016F70FFE393059508032588
:109F20000A004146EFE0B049814679F94A86A685A4
:109F30004E85EFF0DF9BF9BF83250A0013059408D7
:109F4000EF60600119C1C146D5B797C7FF1F93875E
:109F500067E89C4399E797C7FF1F938767D19C43A6
:109F600089C72285EF60A05479FD8547A30FF400CF
:109F70002285EF80B05D2285EF50A0634E8581463B
:109F80004A86A685EFF0BF96A167938757044800DD
:109F90003EC42302010002C6EFF05F88A5BFEF7246
:109FA0005FD783C795004111AA8993F7F707A38468
:109FB000F50032852E89B28AEFE0BFD685676370DF
:109FC000F50CAA84EF50805A2A841DE9416B014A9E
:109FD00097CBFF1F938B8BE1130C400E7D1B19A8B1
:109FE00033048A0383A70B0B3E948357C401638D0C
:109FF0006703050AEFE00F82E344AAFE954639A8FD
:10A000008357C501639297029305050303A50A00D0
:10A010004146EFE0D03A994611E181462686CA854D
:10A020004E85EFF0DF8CA1A883A50A001305040379
:10A03000EF507072C1467DF12285231E9400EF809F
:10A04000F0502285EF50E05697C7FF1F9387C71047
:10A050009C438DCB230004022285EFA090614E85A6
:10A0600081462686CA85EFF09F88A16793870704FB
:10A0700048003EC42302010002C6EFF02FFA41015E
:10A080006F70BFCC89472300F402D1BF397106DE5F
:10A0900022DC4AD8800052D456D25AD026DA4ED684
:10A0A0005ECE2E8A32892A8BEFD0DFF3060571054A
:10A0B00041998A8A3301A140232224FC231404FC01
:10A0C000EFD05FF283479A000605350593F7F7074F
:10A0D0002315A4FCA304FA004A85232624FCEFE000
:10A0E0005FC493170501C1876340F00256811301D5
:10A0F00004FCF2506254D2544259B259225A925A34
:10A10000025BF24B21618280AA844A85EFE07FC125
:10A11000AA894A85EFE0FFC0A1659385C5022A8917
:10A12000130544FCEFD02F9E2685EFD0AF938545D5
:10A1300001C94A86CE85EFD06F8DAA8B15ED894572
:10A14000130544FCEFE03FB2A685130544FCEFE0A5
:10A15000DFB2CE85130544FCEFE03FB2CA8513059C
:10A1600044FCEFE09FB101478146130644FCD285D1
:10A170005A85EFD0CFB99DBF8145130544FCEFE070
:10A180009FAEA685130544FCEFE03FAFCE851305D7
:10A1900044FCEFE09FAECA85130544FCEFE0FFAD41
:10A1A0008144EFD03FE4E3D0A4FC83A70B011397D5
:10A1B0001400BA9783D5070089C5130544FCEFE066
:10A1C000DFAB8504F9BF797106D622D44AD00018D6
:10A1D0004ECE52CC56CA26D25AC8AE893289AA8AE5
:10A1E000EFD05FE00605690541990A8A3301A14075
:10A1F000232A24FC231C04FCEFD0DFDE83C7990054
:10A2000006052D0593F7F707231DA4FCA384F90089
:10A210004A85232E24FCEFE0DFB093170501C187A8
:10A22000634FF0005281130104FDB2502254925446
:10A230000259F249624AD24A424B45618280AA845D
:10A240004A85EFE01FAEA1659385A5022A89130513
:10A2500044FDEFD04F8B2685EFD0CF80854519C5C3
:10A26000CA85EFC0BFFD2A8B0DE98945130544FD62
:10A27000EFE07F9FA685130544FDEFE01FA0CA8590
:10A28000130544FDEFE07F9F01478146130644FD1F
:10A29000CE855685EFD0AFA771B78145130544FD34
:10A2A000EFE07F9CA685130544FDEFE01F9DCA8566
:10A2B000130544FDEFE07F9C8144EFD0BFD2E3D58E
:10A2C000A4FC83270B0113971400BA9783D50700CA
:10A2D00089C5130544FDEFE05F9A8504F9BFEF726D
:10A2E000DFA583474500404DD5E7FD574DC0834668
:10A2F00094000947636DD7080346B400854663E8B8
:10A30000C6088306E40063C406085C45F95623903A
:10A31000D70097C7FF1F83C7678D99E3A304E400A5
:10A3200097C7FF1F9387C7949C4381E78947A3067C
:10A33000F40097C7FF1F938727E29C4381E7894773
:10A340002306F4009705000093854505AA841305AC
:10A350000401EFC0703FFD57231AF40281471CDC53
:10A36000014897C7FF1F23AF878697C7FF1F9387B3
:10A37000A787232E040304C08043EFD0FFD061469B
:10A380003306C50281452285EF703F9E81473E8599
:10A390006F70FF9CFD57E5BFEF723F9A2A8403550B
:10A3A0004502EF50A01C09E5231E04006F703F9B7F
:10A3B0008357E401E5DF930504FF1715010013053A
:10A3C000A577EFB01063DDB7EF723F972E89A165D7
:10A3D00041119385E5032A8436C432C6BE843AC24D
:10A3E000EFC07FF212472285BA85EFE0DF87324661
:10A3F0002285B285EFE07F88A2462285B685EFE010
:10A40000DF87630D090091452285EFE05F811146EA
:10A41000A685EFE0207D41016F707F9489452285FC
:10A42000EFE0EFFF83C704002300F50083C71400AB
:10A43000A300F500CDB7EF725F9083C79500444D40
:10A44000054793F7F707A384F5001C42411183C722
:10A450000700636DF7042E842A8985CC03C7D400D6
:10A460006309F70217C7FF1F13078780184301CF3F
:10A47000A386F400EF80902B83C7D40089E7416561
:10A480007D15EF30407583D72403918B99C3EFB0CE
:10A49000B0624A85A285EFF0CFBFA167C10748002F
:10A4A0003EC42302010002C6EFF04FB741016F70B6
:10A4B0001F8BEF729F8803D745008D47AA844111F7
:10A4C0002E8432892E8563EDE700EFE09F85AA8513
:10A4D000230009002685EFC07FD641016F703F88B9
:10A4E000EFE03F842AC62285EFE0BF83B24585476F
:10A4F0002A862300F9002685EFC05FD1F9BF3971A4
:10A5000006DE22DC26DA80004ED652D456D24AD855
:10A510005AD05ECEAE89B284AA8AEFD0BFAB060510
:10A520001305250241990A8A3301A140232224FC04
:10A53000231404FCEFD01FAA83C7990006054D051C
:10A5400093F7F7072315A4FCA384F9002685232697
:10A5500024FCEFE00FFD93170501C1876340F00273
:10A560005281130104FCF2506254D2544259B25940
:10A57000225A925A025BF24B21618280AA8B03AB72
:10A580000400EFC03FCE35E983D74400014985443C
:10A59000F11793B71700A301F4FC834734FCA165BE
:10A5A000BDC79385E504130544FCEFC0DFD5A68540
:10A5B000130544FCEFE02FEBDE85130544FCEFE0D0
:10A5C000CFEB834734FC114691E30946DA85130546
:10A5D00044FCEFE06FE7814463080900416B7D1B99
:10A5E000EFD05F9F63C8A40201478146130644FC75
:10A5F000CE855685EFC0BFF1A5B7A685130634FCFE
:10A60000EFF03FEB933415002A89860479B79385E0
:10A61000C50451BF8327C90013971400BA9783D587
:10A62000070063866501130544FCEFE00FE5850430
:10A6300045BFEF720FEE79711C103EC4B7070F00D3
:10A640003EC61C103EC883C79500AA8A328593F780
:10A65000F707A384F500AE893284EFE08FEC9317FF
:10A660000501C1876350F0062A8A2285EFE06FEB6F
:10A670002A895285032B0400EFC0DFBE39E58357DA
:10A68000440081440544F11793B71700A303F10078
:10A6900083457100DA872287CA8652862800EFF048
:10A6A000BFD2014781463000CE855685EFC03FE6D8
:10A6B000A1679387D70348083ECC230A810026CEA2
:10A6C000EFF0CF9545616F704FE8A28513067100DA
:10A6D000EFF03FDEAA84094445DD3544E30A55FB2B
:10A6E0004A85EFF00FE70D4445D50144EFD09F8E2A
:10A6F000634BA400C16B0144FD1BEFD0BF8D634EC3
:10A70000A400154471B7DC4413171400BA9783D71B
:10A710000700638127030504D1BFD84493171400B1
:10A72000BA9703D70700631977012390270126857D
:10A73000EF80C0540144A9BF0504C1B7EF724FDEDA
:10A7400083C7950041112A8A93F7F707A384F50080
:10A7500032852E893284EFE0CFDC93170501C18763
:10A76000635BF004AA892285EFE0AFDB2311A1002F
:10A770004E85832A0400EFC0FFAE29E183574400D1
:10A7800085440144F11793B71700A300F100034873
:10A79000110003572100D6875285CE862686CA85AA
:10A7A000EFF0EFB3A167F10748003EC42302910028
:10A7B00022C6EFF0AF8641016F70CFD9A285130694
:10A7C0001100EFF01FCF2A84894471D183572100F3
:10A7D00011678544BA97C2071167C1831307F7EF62
:10A7E000E367F7FA97B7FF1F9387C75E9C4391C74C
:10A7F000854513052100EF40300E83552100228549
:10A800008144EFC09F9D41D5231005002285EF8034
:10A810008048B5BFEF72EFCF83C7950041112A8BF7
:10A8200093F7F707A384F50032852E8A3284EFE090
:10A830004FCF93170501C1876359F004AA8A228577
:10A84000EFE02FCE2A895685832B0400EFC09FA10D
:10A8500021E18357440081440544F11793B7170061
:10A86000A301F10003483100DE875A854A87D68666
:10A870002286D285EFF0AFA6A167ED0748003EC45F
:10A880002302810026C6EFE07FF941016F70EFCB14
:10A89000A28513063100EFF0DFC1AA84094479D103
:10A8A0009167CA97C2071167C1831307F7EF054481
:10A8B000E36AF7FACA85EFC05F92014445F5814922
:10A8C000EFD04FF263DBA900984893971900BA972D
:10A8D00003D7070015E723902701EFD0AFF0154409
:10A8E000E382A9F82685EF80003B97B7FF1F938787
:10A8F000674E9C430144BDD74A85EF4040769DB7E3
:10A9000085097DBFEF72CFC179713E847C083EC856
:10A910002E8AB7071400A1653ECAE5057C08AA89FE
:10A92000080836C4428932C6BA8AC6843ECCEFC013
:10A930009F9DCA850808EFE00FB332460808B2852C
:10A94000EFE0AFB3A246630E09029D450808EFE0B1
:10A950000FAD1D468145EF704FC163870A069145D3
:10A960000808EFE0CFAB1146A685EFE0A02710085E
:10A9700001478146D2854E85EFC07FB945616F7032
:10A980006FBDB6850808EFE04FAF1C400808D843FC
:10A990009355C701858912075183B205D98DEFE020
:10A9A000CFAD1C40080883C58700EFE0CFAB1C404B
:10A9B000080883C5A700EFE00FAB1C40080883C55B
:10A9C0009700EFE04FAA51BF89450808EFE02FA597
:10A9D00083C704002300F50083C71400A300F5001B
:10A9E00079B7EF72EFB383C795004111AA8993F746
:10A9F000F707A384F5003285AE843284EFE06FB2AE
:10AA000093170501C1876357F0042A89032A0400BC
:10AA1000EFC05F8519E9835744000548F11793B7E4
:10AA20001700A307F100814621A81306F100A285B3
:10AA3000EFF03FA81DC11C459DC383D647000148C8
:10AA40000347F10093078500D2884A86A6854E8584
:10AA5000EFF05FEB41016F70EFAF0948E9B71D48B8
:10AA6000D9B7EF72EFAB65715C083EC4B7077B01E5
:10AA70003EC65C083EC883C795002A8A328593F794
:10AA8000F707A384F500AE89EFE04FA88357E100F4
:10AA9000C5C389452800EFC01F8781452800EFE026
:10AAA0008F9CEFC0FF8B97B7FF1F9387E76A9C438C
:10AAB00017B4FF1F03448413AA843334800099C35E
:10AAC0001364240097B7FF1F9387871A9C4399C389
:10AAD0001364440097B7FF1F9387C72F9C4399C304
:10AAE0001364840083D5040028000149EFE0EF9847
:10AAF00083D524002800EFE04F9883D54400280038
:10AB0000EFE0AF97EFD00FC993150501C181280081
:10AB1000EFE0AF96A2852800EFE02F969C44636C8F
:10AB2000F900014781463000CE855285EFC03F9E37
:10AB300059616F702FA2DC441314490028003E9421
:10AB4000EFE06F8C834744000347540089070607F2
:10AB5000BA978607E36EF5FC835524002800814AE6
:10AB6000EFE0AF91834544002800EFE0CF8F8345AD
:10AB700054002800EFE02F8F8347440063C9FA0098
:10AB8000814A8347540063CFFA00050941BF1C4442
:10AB900013975A002800BA9783D50700850AEFE07B
:10ABA000CF8DD9BF032BC40093975A0028003E9B3A
:10ABB00083552B00850AEFE04F8C83550B0028004E
:10ABC000EFE0AF8B7DBFEF724F975C4993E71700C3
:10ABD0005CC9EF8020336F708F98EF720F962E84D0
:10ABE0008145EFF08F9B05C183570500FD172310AA
:10ABF000F50009C4835725002310F400EFF0BFFCD3
:10AC000001456F70CF9531456DDC23100400D5BF31
:10AC1000EF720F9183C7950041112A8A93F7F707C6
:10AC2000A384F50032852E893284EFE08F8F93174D
:10AC30000501C187635EF004AA89C1452285EFD072
:10AC4000BFFA2A8B4E85832A0400EFC0AFE121E5CD
:10AC500083574400231101000544F11793B71700EF
:10AC6000A300F10081440348110003572100D68757
:10AC70005285CE862286CA85EFE07FE6A16793875C
:10AC8000170248003EC42302810026C6EFE01FB928
:10AC900041016F702F8C13061100A285EFF07F81A8
:10ACA000AA8409E523110100094475BF9305210019
:10ACB0005A85EFF09FF2835721002A84CDD797B7AA
:10ACC000FF1F938727119C4391C7854513052100DA
:10ACD000EF4080408355210026853144EFC0EFCFFF
:10ACE00059D1231005002685EF70F07A0144A5BFE5
:10ACF000EF72AF8441112E896C00AA8402C6EFF076
:10AD0000CF8909CD0357050005072310E500EFF0B3
:10AD10009FEB81473E8541016F706F8432479547B5
:10AD200075DBCA852685EF20D008C147E34405FEC0
:10AD30003244854741462310F40083570900A68515
:10AD4000130544002311F400EFD0D0692285C1B768
:10AD5000EF621FFD83C795004111AA8A93F7F70799
:10AD6000A384F5003285AE893284EFD09FFB931720
:10AD70000501C187635EF0042A8AC1452285EFD0B0
:10AD8000BFE6AA845285032B0400EFC0AFCD21E5B6
:10AD900083574400231101008544F11793B717002E
:10ADA000A300F10001440348110003572100DA8792
:10ADB0005685D2862686CE85EFE07FD2A16793871F
:10ADC000070248003EC42302910022C6EFE01FA5FF
:10ADD00041016F603FF8A28513061100EFF06FED9F
:10ADE0002A8409E523110100894475BF268593054E
:10ADF0002100EFF0FFEFAA845DF583552100228545
:10AE0000EFC0AFBD4DF10149EFD0CF9D635DA9000B
:10AE1000184893171900BA9703D707001DE703577F
:10AE200021002390E700EFD0EF9B6302250397B743
:10AE3000FF1F938727FA9C4389C703552100EF40E2
:10AE400000222285EF703065B9BF050975BF9544B2
:10AE500099BF05C19307F00F630FF500C547630C59
:10AE6000F5009307F5FF05453315F50042054181CF
:10AE700082800145828041657D158280B9E1EF6263
:10AE8000DFEB034506033284EFF0BFFC9305803E01
:10AE9000B305B502C205C18191C90357E4028547D4
:10AEA00063F6E70013050401EFC020168357E402A0
:10AEB00041677D176385E700FD172317F4026F6074
:10AEC0001FEA8280EF62FFE4004283C79500444D91
:10AED0000349140093F7F707A384F50083470400A0
:10AEE000220911673369F900A167B347F9004111DD
:10AEF0002A8BAE8A63ECE70C834724001307C00E4D
:10AF0000B91793F7F70F6371F70E03473400C14782
:10AF100063ECE70C834744001307E00793C7070877
:10AF20006373F70A8349840083477400A209B3E975
:10AF3000F900856763F9F908034A64008347540000
:10AF40004E85220A336AFA00EF40406245C12396DB
:10AF50002403834B3400137AFA00239A34032388A2
:10AF600074032399440393890401631A090023A6F7
:10AF70000402239804024E85EFC0A00A1DA00349D5
:10AF800024004A85EFF0FFEC2397A4028347440096
:10AF90004E85A388F402E3810BFEE30F09FCEFC0AA
:10AFA0006005EF70907981460146D6855A85EFE0BD
:10AFB0009FA5A167938797033EC423020100480021
:10AFC00002C6EFE0BF8541016F603FD88544A2868D
:10AFD0002686D6855A85EFE01FA3A167938797033E
:10AFE0003EC423029100E1BFBD44D5B79144C5B72B
:10AFF000EF621FD301111C08404D3EC2B7070F007E
:10B000003EC41C083EC62A89AE89EFC01F9D585C0D
:10B010001C5C634CB70A6394E50063E8A70A3385B8
:10B02000A740B3B7A700B305B7401306803E8146DB
:10B030009D8DEFD0407B93140501C180A165938560
:10B04000C5034800EFC02FAC81454800EFD0BFC119
:10B05000835504044800EFD05FC2835524044800A0
:10B06000EFD0BFC1814599C8C167FD179305F00FA7
:10B070006386F4002685EF402015AA854800EFD0AE
:10B080009FBE03554404814511C9C167FD1793054F
:10B09000F00F6305F500EF402013AA854800EFD0BC
:10B0A0009FBC834564044800EFD0FFBB8345740414
:10B0B0004800EFD05FBB500001478146CE854A85EE
:10B0C000EFC0EFC405616F60FFC8814485BFEF62C8
:10B0D000DFC683C7950093F7F707A384F500EFF069
:10B0E0003FF16F60DFC7EF62BFC383C795004111B7
:10B0F000404D93F7F707A384F5002A8A3285B2847E
:10B10000AE89EFD01FC22A8B2685EFD09FC12A8936
:10B110002685EFD0BFBF93170B0163CA0702E17703
:10B12000CA97C207C183116763E3E7029307091057
:10B13000C207C1831307B00F637BF70093170901A0
:10B14000C187AA8A6348F000C54763FA57014101E5
:10B150006F605FC0EFC08F83E31B25FFF5B7630609
:10B160000B0263040902814463870A02B7077F0068
:10B1700023106405231124057CC05685EFF07FCD94
:10B180009304803EB304950239A0B7077F002320C3
:10B1900004047CC0814403552404EFB0101095CC06
:10B1A000EFC0BF83269593D7F44133379500AE9710
:10B1B000BA9708DC5CDCCE855285EFF07FE399E03E
:10B1C00023220404A1679387B70348003EC42302E7
:10B1D000010002C6EFE08FE49DBF814701481CDCFF
:10B1E000232E0403C9BFEF625FB5EFC0FFE9E1475B
:10B1F0003305F5029145EF30507FE55711C597B7FC
:10B20000FF1F23A3A79E81473E856F605FB58547DB
:10B2100017B7FF1F230CF79C8280EF621FB297B70E
:10B22000FF1F9387279C80432DC083570404639E90
:10B23000A70483572404639AB7043689B284EFC005
:10B24000CFF95C5C63C3B7046395B7001C5C63EE25
:10B25000A7028347640463F3F400A6872303F4047E
:10B260008347740463F39700A687A303F40483570A
:10B27000440441677D176385E70085072312F404C2
:10B280003C4481C7CA85268582976F605FAD97B7BA
:10B29000FF1F938727959C43014599C303C58700EA
:10B2A0008280EF629FA90111B70707003EC683C7DE
:10B2B0009500584D0AC493F7F7070AC8A384F50010
:10B2C0002A89AE8401CB1C4283C707002304F70000
:10B2D000EF70D0452164930554022800EFC0AF827F
:10B2E000EFF0FFFAAA852800EFD0FF973000014762
:10B2F0008146A6854A85EFC08FA113044402480801
:10B3000022CC230A010002CEEFE04FD105616F602D
:10B310001FA5EF629FA201117C003ECAB70707007C
:10B320003ECC7C003ECE83C795002E84AA8493F742
:10B33000F707A384F500A165938555024808EFB08F
:10B340009FFCEFF0DFF4AA854808EFD0DF915008AA
:10B3500001478146A2852685EFC06F9B05616F601E
:10B360001FA097B7FF1F9387E7879C43094599C3A1
:10B3700003C59700828097B7FF1F9387A7869C43DA
:10B38000094599C303C5D700828097B7FF1F9387EC
:10B3900067859C43014599C303C5A7008280EF627E
:10B3A0003F980111B70708003EC683C79500404D7E
:10B3B0000AC493F7F7070AC8A384F5002A89AE8464
:10B3C00029C01442854703C7060063EEE70683479A
:10B3D000940009468149638EC700B307F740A30470
:10B3E000E400B339F00083C716002305F400EF70C2
:10B3F000F03303572403058B09C763840900EFA0CA
:10B40000B06B2164930584022800EFB0DFEFEFF00A
:10B410005FF5AA852800EFD01F85EFF01FF7AA85FA
:10B420002800EFD05F84014781463000A6854A8519
:10B43000EFC0EF8D13047402480822CC230A0100E8
:10B4400002CEEFE0AFBD05616F60DF90EF62FF8E6F
:10B4500001117C003ECAB70708003ECC7C003ECEFE
:10B4600083C795002E84AA8493F7F707A384F50079
:10B47000A165938585024808EFB0FFE8EFF07FEE05
:10B48000AA854808EFD02FFEEFF03FF0AA854808C4
:10B49000EFD06FFD500801478146A2852685EFC099
:10B4A0000F8705616F60BF8B97A7FF1F9387877317
:10B4B0009C43014599C303C5B7008280EF62FF87B3
:10B4C0000111B70707003EC683C79500404D0AC467
:10B4D00093F7F7070AC8A384F5002A89AE8405C448
:10B4E0001C42054783C70700636AF7040347B4009B
:10B4F000630BF700A305F400EF7050238347B400FB
:10B50000A9C3EFD00FD921649305B4002800EFB090
:10B510009FDFEFF07FF9AA852800EFD0CFF4014735
:10B5200081463000A6854A85EFB07FFE2904480891
:10B5300022CC230A010002CEEFE04FAE05616F601E
:10B540001F82EFD02FDAC1B7EF622FFF01117C000D
:10B550003ECAB70707003ECC7C003ECE83C79500AD
:10B560002E84AA8493F7F707A384F500A165AD059F
:10B570004808EFB05FD9EFF03FF3AA854808EFD055
:10B580008FEE500801478146A2852685EFB03FF82F
:10B5900005616F60CFFC97A7FF1F9387A7649C434B
:10B5A000094599C303C5C7008280EF620FF90111F5
:10B5B0007C00AE843ECAA165B70707002A843ECC52
:10B5C000D1057C0048083ECEEFB0FFD3EFF0BFFCC2
:10B5D000AA854808EFD02FE9500801478146A68583
:10B5E0002285EFB0DFF205616F606FF7EF62EFF475
:10B5F00083C7950093F7F707A384F500EFF0FFFAF0
:10B600006F60EFF5EF62CFF183C795000329C501A5
:10B61000411193F7F707A384F5001C4283C9070083
:10B62000854763EC370597B7FF1F9387E7B29C43C5
:10B630002E84AA8495C7EFF01FF689476302F502AE
:10B64000630009028347C900638C3701230639016F
:10B65000EF70D00D83572903898B99C3EFA0D04594
:10B660002685A285EFF07FF4A167CD0748003EC490
:10B670002302010002C6EFE06F9A41016F608FED77
:10B6800097A7FF1F938707569C431D4599C303C582
:10B69000E7008280EF626FEA0111B70707003EC63C
:10B6A00083C79500584D0AC493F7F7070AC8A384C7
:10B6B000F5002A89AE8405C71C4283C7070093960C
:10B6C0008701E18663C8060485466385D7048346FF
:10B6D000E7006386F6002307F700EF70300521646A
:10B6E0009305E4002800EFB01FC2EFF07FF9AA85B0
:10B6F0002800EFD04FD7014781463000A6854A8504
:10B70000EFB0FFE03504480822CC230A010002CE46
:10B71000EFE0CF9005616F608FE4EF620FE20111FF
:10B720007C003ECAB70707003ECC7C003ECE83C7F4
:10B7300095002E84AA8493F7F707A384F500A165EA
:10B74000B9054808EFB03FBCEFF09FF3AA85480861
:10B75000EFD06FD1500801478146A2852685EFB012
:10B760001FDB05616F60AFDFEF628FDBAA840144EE
:10B7700017A9FF1F13094947E149EFC0FF90634430
:10B78000A400014519A833053403832709003E9519
:10B79000835725006395970011056F60AFDB0504A3
:10B7A000E9BF032E850063040E1017A3FF1F1303C8
:10B7B000636203230300631503002943639A060EA3
:10B7C00003234E01631503001D436393070EEF62CD
:10B7D0004FD4C689428A3E89BA8AB684328BAE8BF0
:10B7E0002A84A1E903554E0009E501431A856F60DB
:10B7F000CFD5A167A98F116763F7E700EFF0DFF6F8
:10B800008145EFF08FBD0844B70700E05841F98F3C
:10B8100018455CC1B707001FF98F1CC55C4981C77B
:10B820006105EFB01000E38209FC2285EF70606EC5
:10B830006DBF3285EFA0E0620D434DD91C44116706
:10B8400003D54700A167A98F63F7E700EFF0DFF1A9
:10B850008145EFF08FB80323840093164B01D1820A
:10B860008347B300035663008588FD8BA305F3006F
:10B87000FD777D8E558EFD76FD16B204F18E832701
:10B880004301C58E231273012313D30023045301F4
:10B8900023052301A3044301D9D72285EFB07FBB41
:10B8A000AA850844B5DD6105EFB02076ADBF1D4324
:10B8B0001A858280EF62CFC60569AA84AE89328A72
:10B8C0000144FD5A7D19EFC0EFF06345A400014526
:10B8D0006F604FC8D84493171400BA9703D7070076
:10B8E000631B37032390570163050A002685EF7019
:10B8F000E0389C448DC383D76700B3F72701639C6E
:10B900003701D28801488147014781460146814578
:10B910002685EFF01FE905047DB7EF626FC07971EE
:10B920001C103EC4B7070F003EC61C103EC883C79C
:10B930009500AA8A328593F7F707A384F5002E892C
:10B940003284EFD00FBE93170501C1876350F00614
:10B95000AA892285EFD0EFBC2A8A4E85032B0400EA
:10B96000EFB05F9039E58357440081440544F117F7
:10B9700093B71700A303F10083457100DA8722878C
:10B98000D2864E862800EFE03FA401478146300072
:10B99000CA855685EFB0BFB7A1679387F7034808FC
:10B9A0003ECC230A810026CEEFD05FE745616F6071
:10B9B0006FBAA28513067100EFE0BFAFAA840944F5
:10B9C00045DD5285EFE0EFB80D445DD50546D285E3
:10B9D0002685EFF03FEE2A8445B7EF620FB6835518
:10B9E00007000346270041112A842E8532C62EC443
:10B9F000EFE02FB611C53246A2452285EFF09FEB4E
:10BA000041016F60CFB5EF62CFB083C795004111A0
:10BA1000AA8A93F7F707A384F5003285AE893284AA
:10BA2000EFD02FB093170501C1876357F008C145C8
:10BA30002A8A2285EFD04F9B2A8D2285EFD06FAEC8
:10BA40002A892285EFD08FAC930705F893F7F70F7B
:10BA50001307E007AA8B6371F7062285EFD00FABBF
:10BA60002A8C2285EFD08FAAAA8C5285032B040042
:10BA7000EFB04FFF29E583574400231101008144B3
:10BA8000F11793B71700A300F10005440347110015
:10BA900083562100938784005685DA88228852864F
:10BAA000CE85EFE03FE6A167E90748003EC42302E8
:10BAB000810026C6EFD09FD641016F600FA9130603
:10BAC0001100A285EFE0FF9EAA8409E52311010081
:10BAD00009446DBF930521006A85EFF06FA12A84A8
:10BAE00055F5835521009356C90013164901854821
:10BAF0006688E2875E87858A51822685EFF07FCA55
:10BB00002A8469B7EF62EFA083C7950041112A8BA1
:10BB100093F7F707A384F5003285AE893284EFD01E
:10BB20004FA093170501C1876352F0082A8A228526
:10BB3000EFD02F9FAA8A2285EFD0AF9E2A89228537
:10BB4000EFD0CF9C930705F893F7F70F1307E007A3
:10BB50002A8C637DF7042285EFD04F9BAA8C228527
:10BB6000EFD0CF9A2A8D5285832B0400EFB08FEF50
:10BB700029E18357440085440144F11793B7170026
:10BB8000A301F10003473100930784005A85DE8842
:10BB90002688D6865286CE85EFE0DFD68D474800D0
:10BBA0003EC42302910022C6EFD05FC741016F60FF
:10BBB000CF99A28513063100EFE0BF8F2A84894414
:10BBC00071D19356C9001316490185486A88E687E2
:10BBD0006287858A5182D685EFF0BFBCAA845DB7A3
:10BBE000EF620F942A8981440144617A916A17AB0C
:10BBF000FF1F130B2B1EEFC0EFBE63C5A4002285F1
:10BC00006F604F958327090093991400CE9703D551
:10BC1000070033074501420741836362570311CD93
:10BC200003270B0009C785453E85EF30E04A83278F
:10BC300009000504CE972390070085046DBFEFF03F
:10BC4000BFB2832709000504CE972390070075D55E
:10BC50008145EFE09FF8D5B7EF628F8C83C79500E1
:10BC600041112A8A93F7F707A384F50032852E89BC
:10BC70003284EFD00F8B93170501C1876354F00412
:10BC8000AA89832A0400EFB0EFDD21E18357440045
:10BC900085440144F11793B71700A301F10003484D
:10BCA0003100D68752850147CE862686CA85EFD0D9
:10BCB0001FE3A167F50748003EC42302910022C696
:10BCC000EFD0DFB541016F60EF88A2851306310028
:10BCD000EFE02FFE2A84894479D197A7FF1F93872D
:10BCE000670F9C4381CB0449EFC0CFAFAA8526855F
:10BCF000EF30803E13050401EFF09FEE2285EF60E8
:10BD00009079814469BFEF62CF8083C7950041116C
:10BD1000AA8A93F7F707A384F5003285AE893284A7
:10BD200023110100EFC0FFFF93170501C187635C7A
:10BD3000F0042A8AC1452285EFC01FEBAA8B5285E9
:10BD4000032B0400EFB00FD231E183574400854448
:10BD50000144F11793B71700A300F1000348110045
:10BD600003572100DA875685D2862686CE85EFD006
:10BD70001FD7A1679387270248003EC42302910082
:10BD800022C6EFD0BFA941016F503FFCA285130628
:10BD90001100EFE00FF22A84894469D197A7FF1FB1
:10BDA0009387470398433E8901CB0449EFC08FA393
:10BDB000AA852685EF30403213050401EFF05FE2DB
:10BDC000EFC04FA2954459D9930521005E85EFE05D
:10BDD0003FF2AA8441F51C48035721002285239095
:10BDE000E700EF60506B83270900ADDB03552100AE
:10BDF000EF30E026A5B7EF52DFF183C79500411180
:10BE0000AA8A93F7F707A384F5003285AE893284B6
:10BE1000EFC03FF193170501C1876359F0042A8AE7
:10BE20002285EFC01FF02A895285032B0400EFB052
:10BE30006FC321E18357440085440144F11793B750
:10BE40001700A301F10003483100DA8756854A87BD
:10BE5000D2862686CE85EFD09FC8A167F907480015
:10BE60003EC42302910022C6EFD05F9B41016F5078
:10BE7000DFEDA28513063100EFE0AFE32A848944A9
:10BE800079D19167CA97C2071167C1831307F7EF8A
:10BE90008544E36AF7FA97A7FF1F9387A7F39843B0
:10BEA000BE8B01CB0449EFC0EF93AA852685EF3006
:10BEB000A02213050401EFF0BFD2EFC0AF9295446A
:10BEC00059D11C482285814423902701EF60B05C42
:10BED00083A70B00ADDB4A85EF306018ADB7EF529A
:10BEE000DFE52A844105B284EFF09FCF01C52285AA
:10BEF000EF60705A81460146A6852285EF70C00B1F
:10BF00001C4C89C7DC4799C3228582976F503FE557
:10BF100097A7FF1F938707CD9C43014599C31385BE
:10BF20000701828097A7FF1F9387C7CB8843828032
:10BF3000EF52BFE09317C600DD8DC2054111C181EC
:10BF40002A8432C6EFC07FD3324622851182937590
:10BF5000F60FEFC05FD141016F507FE0EF525FDC21
:10BF600079713C083ED2B7070C003ED43C083ED65F
:10BF700083C79500AE842A8993F7F707A384F50059
:10BF8000A165938535044810EFB0EFB7C165FD1585
:10BF9000014417AAFF1F130A6AE5930A400EAE89EF
:10BFA0002E8B2EC6EFC00F874205931704014181E7
:10BFB000C183B24563E3A702C167FD176385F5003E
:10BFC0004810EFC09FCB501001478146A6854A8597
:10BFD000EFB0EFD345616F50FFD73307540383278A
:10BFE0000A0BBA9703D6C701630836016388350187
:10BFF0004810EFF0FFF3DA85050465B7B285EDBFB1
:10C00000EF523FD179717C083EC8B70711003ECA94
:10C010007C083ECC83C79500AA89328593F7F70741
:10C02000A384F5002E89EFC0DFCF8567637EF5021C
:10C03000A165AA8489050808EFB0EFAC2685EF302A
:10C04000E052133415000A04A2850808EFC0BFC1EE
:10C05000A6850808EFC07FC235C001478146100899
:10C06000CA854E85EFB0AFCA45616F501FCEB3078A
:10C0700054030327CA0ABA9703D70700631A970025
:10C0800003D62700638A65030808EFF07FEADE85A0
:10C0900005042EC6EFB01FF9420593170401418134
:10C0A000C183B245E3E5A7FCC167FD17E387F5FA55
:10C0B0000808EFC09FBC55B7B285D9BFC165FD1553
:10C0C000014417AAFF1F130A6AD2930A80022E8B1B
:10C0D000AE8BC1B7EF527FC6184183471700834626
:10C0E0000700A207D58FD207D1832390F50083479D
:10C0F0002700034717008D45A207D98F918323108E
:10C10000F600EFC03FAD6F509FC5EF527FC1C164D5
:10C11000014417A9FF1F130969CD93098002FD147B
:10C12000EFB05FF06345A40001456F50BFC2330517
:10C1300034038327C90A3E9583570500E38797FE9A
:10C140000504F9BFEF52DFBD2A8AAE89B284B68AF0
:10C15000EF30C04109E591473E856F50BFBF2A8946
:10C160004E85EF9010502A84638A0A048D476DD55E
:10C1700003570500C547E31147FF0347F90185460B
:10C18000AD47E31BD7FC8347450091CB4146A685CD
:10C190005D05EFC0D022814761D1AD4775BF13095E
:10C1A00065012302E500CA852685EF10202D15CDF7
:10C1B000A547E3830AFA2302040079BF11CD835710
:10C1C0000500E39A47F94146A6851905EFC0301FDF
:10C1D000814759D1994749B74E85EFF01FF32A841B
:10C1E00095473DD9130955007DBF4146A6852310CB
:10C1F00044012311340113051900EFC0B01E22853C
:10C20000EF60B03C814789BFEF523FB379717C004A
:10C210003ECCB7070A003ECE7C003ED083C79500D7
:10C22000B2842E8493F7F707A384F5001306A100C8
:10C230002A892C002685EFF0FFE9A16528088D05E5
:10C24000EFB06F8C90408355A10003558100854667
:10C25000EFF05FEFAA84AA852808EFC0DFA003569D
:10C26000A100835581002808EFF09FCC30080147DA
:10C270008146A2854A85EFB08FA9854748103ED4F4
:10C280002302910202D6EFD06FD945616F503FADC6
:10C29000EF52BFAA79717C003ECCB7070A003ECEB0
:10C2A0007C003ED083C79500B2842E8493F7F707B5
:10C2B000A384F5001306A1002A892C002685EFF03F
:10C2C0007FE1A16528088D05EFB0EF83904083558D
:10C2D000A100035581008146EFF0DFE6AA84AA851C
:10C2E0002808EFC05F980356A100835581002808F5
:10C2F000EFF01FC4300801478146A2854A85EFB0A0
:10C300000FA148102302910202D402D6EFD00FD120
:10C3100045616F50DFA4EF525FA2EFF0BFE26F50B4
:10C320001FA497A7FF1F9387278C88438280EF5213
:10C33000DFA0835725004111AE842A842307B10072
:10C3400017F5FFFF1305A5696C002316F100EFB088
:10C35000CFD581C42285EF60B02DFD572310F400A6
:10C3600013062002814513055400EF501FA0410120
:10C370006F50FF9EEF52DF9A79717C003ECCB70779
:10C380000A003ECE7C003ED083C79500AA89AE84C9
:10C3900093F7F7073285A384F5001306A1002C005C
:10C3A000EFF05FD3035581001144EF30201C15C11D
:10C3B0000355A1000144EF90D02A01CD0357050099
:10C3C0008357810045446316F7008545EFF03FF63B
:10C3D00001442169930539002808EFA0DFF2A28506
:10C3E0002808EFC05F880356A10083558100280804
:10C3F000EFF01FB4300801478146A6854E85EFB0A7
:10C400000F9148104AD42302810202D6EFD00FC107
:10C4100045616F503F94EF52BF909797FF1F9387EE
:10C42000677C2A8488432E8915C1035745038357A7
:10C43000C401631DF70023260502231805024105E8
:10C44000EFA0303E63040900EF60302F814497A9CC
:10C45000FF1F9389A999130A8002EFB0BFBC63CC78
:10C46000A40297A7FF1F9387A7809C4389C7035502
:10C47000C401EF104076630509002285EF60500388
:10C480001306400E81452285EF503F8EFD57231E37
:10C49000F4006F503F8C3385440383A7C90A3E954F
:10C4A000035705008357C4016315F700CA85EFF0F1
:10C4B0001FE885045DB7EF52BF8683C79500411121
:10C4C000AA8993F7F707A384F5003285AE84EFC0FD
:10C4D0005F8585676370F5042A89EF302009014480
:10C4E00011C983D704003144638627018545EFF0E5
:10C4F0009FF201444E85A2864A86A685EFD02FBFC3
:10C50000A1679387170448003EC42302810002C636
:10C51000EFD0CFB041016F50FF83EF527F809797EC
:10C52000FF1F9387276C80431DCC0145EFA0E05689
:10C5300081470148C1641CDC232E0403232004042A
:10C5400017A9FF1F1309898A01449309400EFD149E
:10C55000EFB05FAC634BA4008145170500001305E5
:10C560004598EFB08FB46F50EFFE33053403832747
:10C57000090B3E958357C501638597008545EFF00C
:10C580009FE90504F1B79357050113D78700A380EE
:10C59000F50093170501C183A1832380E500238162
:10C5A000F500A381A5008280EF522FF9230005003A
:10C5B00083C71500A300F50083C725002301F500FC
:10C5C00083C73500A301F50083C745002302F500AA
:10C5D00083C75500A302F50083C765009305950046
:10C5E000A30305002303F500230405003285EFF0C3
:10C5F0009FF96F50CFF6EF52AFF24111E9541DC9C8
:10C6000095C993F9C5FF2E842A89AA84338AA90083
:10C61000B7EA040063149A020D88854401CCB7E799
:10C6200004009C5F82972AC622866C00330539017C
:10C63000EFC0405B268541016F50CFF183A78A038D
:10C640009104829793170501C183A183A38EF4FE01
:10C6500093570501238FF4FEA183238EA4FEA38F9D
:10C66000F4FE4DBF63E0D502EF522FEDB2874111CA
:10C670003686BE8536C6EFC0E056B24641013685E5
:10C680006F50EFED814636858280838705001387E2
:10C69000F5003D05FD8793F77708834607007D1574
:10C6A0008606B58FA300F5006307B7007D178347A3
:10C6B00017009D83DDB78280EF522FE8B7E70400B3
:10C6C00083A7070932872A863A8582971335150092
:10C6D0006F50EFE801CD814799C9EF520FE641460F
:10C6E000EFC0405085473E856F506FE781473E85DC
:10C6F00082801DC5EF526FE4414681452A84EF5088
:10C70000CFE64146814513050403EF500FE601478C
:10C71000C1672322040438C87CC805456F502FE444
:10C7200001458280814729CDA1CDEF520FE1B2842E
:10C730002E891306800581452A84EF500FE3CA85B0
:10C7400024C42685EFF01FF9414681452285EF502C
:10C75000CFE13044A2852285EFF01FF69304040157
:10C76000A2852685EFF07FF2A68513050402EFF07F
:10C77000DFF12285EFF0FFF785473E856F502FDE12
:10C780003E858280EF52CFD94111E9541DC995C928
:10C7900093F9C5FF2E842A89AA84338AA900B7EAAF
:10C7A0000400639444030D88814401CCB7E704007E
:10C7B0009C5F82972AC622866C0033053901EFC040
:10C7C0006042268541016F50EFD883A78A03910408
:10C7D000829793170501C183A183A38EF4FE93571B
:10C7E0000501238FF4FEA183238EA4FEA38FF4FE04
:10C7F0004DBF71CDEF52CFD2B28401E605456F50E7
:10C800006FD52A842E890145FDD93C487848B3E686
:10C81000E700F5D69386F7FFB3B7F6007D17032A36
:10C820004404BA9734C87CC8630F0A04C14913058D
:10C830000A03B38949412295637B3601B2862E866D
:10C84000A685EFF03FE27C40BE9464C045BFCE8633
:10C850002E86CE85EFF01FE1C114D2944E9923228B
:10C860000404A2879306040103C7070003C6070355
:10C870008507318FA38FE7FEE398F6FE3044A2854B
:10C880002285EFF07FE32699C1493306994063EA98
:10C890009900ADD4A686A68513050403EFF09FDCAE
:10C8A0006DB78147B306F4003307F600034707006E
:10C8B00083C5060085072D8F2380E600E39437FFAC
:10C8C0003044A2852285EFF03FDFC1147DBF0145D2
:10C8D000828019C9EF526FC6130680058145EF505B
:10C8E000CFC805456F50AFC70145828081473DC91C
:10C8F000B5C9EF528FC4FC4141462E84AA8463938C
:10C90000C70413860501A2878146C14503C70700F6
:10C9100003C507038507298F3305D60003450500A6
:10C920008506298FA38FE7FEE392B6FE3044A285E9
:10C930002685EFF07FD82285EFF0BFF985473E8549
:10C940006F50EFC1138507031D8E81452295EF506F
:10C95000CFC17C40130700F813060402A297238876
:10C96000E70255B73E858280EF522FBD6D712E8450
:10C97000B284AA85901028003689EFF0BFDA19E951
:10C98000D55705A050400C402800EFF09FE66DD928
:10C99000FD142104E5F82C004A85EFF03FF58147AE
:10C9A00065D13E8551616F508FBBEF520FB9411178
:10C9B0002EC432C62C000546EFF01FFB41016F501C
:10C9C0000FBAEF528FB701112A842EC602C802CACD
:10C9D00002CC02CEEFC06049B2462A86A285080882
:10C9E000EFF0BFFC1375F50F05616F504FB7EF52B5
:10C9F000CFB47971B2872A8421462308B100130588
:10CA00001101BE853AC436C6EFC0C01DB2469305BB
:10CA100091013685EFF03FB72285141035460C089A
:10CA2000EFF0BFF82A84224711E521460C103A8521
:10CA3000EFC0401B228545616F506FB2EF52EFAFE0
:10CA40007171AE84AA850A853284EFF0BFC801C92E
:10CA50000A86A6852285EFF03FC6814711E1C547CA
:10CA60003E854D616F50AFAFEF522FAA1D712A8ADC
:10CA7000B289BE8435468547130511012E8CB68ACE
:10CA80003A8BC28C468D2308F100EFC0A015101020
:10CA90000C085285231F0100EFF05FFA2A842DE96C
:10CAA000A147631BFD069307900591E0E5473546D6
:10CAB000E2851305110113990A012308F1001359A6
:10CAC0000901EFC020121357890093978A00D98F6C
:10CAD00090080C085285231FF100EFF03FF62A84DE
:10CAE00005E9A1E09387FA0091831379F9003EC626
:10CAF000631309004149668B8144C14B854DB247A0
:10CB00006397970C6A868C0033855C01EFC0800DBB
:10CB1000228525616F502FA393079004C9F8A5477C
:10CB200079B7834701050947C14B2308F1008347C3
:10CB30001105A58FA308F10093872400814463EFBA
:10CB4000FB02014714083386E6008C08B386E40034
:10CB5000BA95DA9683C6060083C505000507AD8E33
:10CB60002300D600E390E7FE41476398E70490086E
:10CB70000C085285EFF09FEC35D535A8B3069B0025
:10CB8000BA871008B305F60090083E9603C5060064
:10CB90000346060085078506298E2380C500E3929B
:10CBA00077FF998F90080C085285BE94EFF01FE92B
:10CBB0008947014749D52A84A1BF90083E9603467C
:10CBC00006001408BE962380C600850779BFB247C9
:10CBD0008504638B971281471808B306F7009808FD
:10CBE0003E973386F9000347070003460600850792
:10CBF000318F2380E600E39177FF90080C0852857F
:10CC0000EFF0DFE34DF93546E28513051101230806
:10CC1000B101EFB0307D13970401418393978400F5
:10CC20002183D98F10180C085285231FF100EFF0D3
:10CC3000FFE051F1814710183387F9003E96034712
:10CC4000070003460600B306FB008507318F2380EB
:10CC5000E600E39277FF75A01808B306F70098087E
:10CC60003E973386F9000347070003460600850711
:10CC7000318F2380E600E3E127FFCA8763987709B5
:10CC800090080C085285EFF07FDB15F5814798007E
:10CC9000B306F700900818103E973E96034707002A
:10CCA000034606008507318F2380E600E39177FF76
:10CCB0003546E285130511012308B101EFB09072EA
:10CCC000139704014183939784002183D98F10180F
:10CCD0000C085285231FF100EFF05FD6E31D05EC31
:10CCE000814710183387F9003E9603470700034633
:10CCF0000600B306FB008507318F2380E600E3E2E0
:10CD000027FFC109410BE5BB8147B5B79408BE9623
:10CD100083C6060018083E972300D7008507B9BFD1
:10CD2000638E062CEF427FFE59712A84BE89B28B36
:10CD300085473546130511022E8B468C4289BA8AE7
:10CD4000368A2300F102EFB0F06910180C1022852A
:10CD500023170102EFF09FCE631E0510A147631950
:10CD6000FC069307900563930900E5473546DA858D
:10CD70001305110293140A012300F102C180EFB0E0
:10CD8000706693178A0013D78400D98F90080C100F
:10CD900022852317F102EFF07FCA69ED6390090441
:10CDA0009307FA00BD88918391E0C144C207C18313
:10CDB000DE8C814A3EC6414DB24763EAFA0C628678
:10CDC000B3854B018810EFB0905F4DC53D555DA018
:10CDD00093079004E39C09F8A54749BF83470105E1
:10CDE0000947C14C2300F10283471105B3C7F9007D
:10CDF000A300F10293872900814963EFFC02814679
:10CE000018103306D7008C083387D900B69556978B
:10CE10000347070083C5050085062D8F2300E60024
:10CE2000E390D7FE4147639AE70490080C102285EF
:10CE3000EFF0DFC035D53DA8B3863A01BA871010B0
:10CE4000B305F60090083E9603C5060003460600AB
:10CE500085078506298E2380C500E39297FF3387D7
:10CE6000EC4090080C102285BA99EFF03FBD89473D
:10CE7000014741D565616F401FED90083E9603461E
:10CE800006001410BE962380C600850769BFB2470E
:10CE9000850A93990A01939D8A0093D909016399A0
:10CEA000570D85473546DA85130511022300F10237
:10CEB00093D98900EFB01053B3ED3D0190000C10F1
:10CEC00022852317B103EFF07FB74DF58147A6897F
:10CED00063E6970626860C084A85EFB0B050814776
:10CEE0001810B306F700100898083E973E960347BF
:10CEF0000700034606008507318F2380E600E3E143
:10CF000097FE639DA90590080C102285EFF01FB3D2
:10CF100035F181479810B306F700900818183E972E
:10CF20003E9603470700034606008507318F23809E
:10CF3000E600E391A7FF4109C10CBDBD18089000B0
:10CF4000B306F7003E963387FC000347070003460D
:10CF500006008507318F2380E60095BF98084E971D
:10CF6000034707001C10CE972380E700850951BFB7
:10CF700085473546DA85130511022300F10293D95E
:10CF80008900EFB03046B3ED3D0190000C102285D2
:10CF90002317B103EFF09FAAE31E05EC81471808A1
:10CFA0009000B306F7003E963387FC000347070066
:10CFB000034606008507318F2380E600E391A7FF33
:10CFC00041460C084A85EFB0F04181471810B3067E
:10CFD000F700100898083E973E960347070003465F
:10CFE00006008507318F2380E600E391A7FF9008B4
:10CFF0000C102285EFF09FA41DDDADBD7D55828014
:10D00000EF42BFD301112A842E8593055100328946
:10D0100002C002C202C402C693047400EFF0AFD68D
:10D020001D46A68513059100EFB0D03B10088A85F8
:10D030004A85EFF0BFA019ED93071400180883C6C6
:10D0400007000346070085070507B18EA38FD7FEAB
:10D05000E397F4FE05616F409FD0EF427FCC2E84B2
:10D060008C414111AA89838715003289914463D389
:10D070000700A1449797FF1F9387070E9C43B1C3F6
:10D08000B5CE8D472310F10083C725004A852301C3
:10D09000F10083C73500A301F10083C745002302D7
:10D0A000F10083C75500A302F10083C76500930513
:10D0B0009100A30301002303F10023040100EFF01A
:10D0C0008FCC0C404A860A85EFF00FCE032804006F
:10D0D00083564400A6881D0881470147E51642860D
:10D0E0008A854E85EFF05F982A8909E5A685228515
:10D0F000EFB0FFB24A8541016F40DFC54A860A851D
:10D10000EFF08FCA7DBFEF42BFC12E848C41411129
:10D11000AA89838715003289914463D30700A1440B
:10D120009797FF1F938747039C43B1C3A5CE8D47B5
:10D130002310F10083C725004A852301F10083C72E
:10D140003500A301F10083C745002302F10083C726
:10D150005500A302F10083C7650093059100A30366
:10D1600001002303F10023040100EFF0CFC10C40C4
:10D170004A860A85EFF04FC3835644000328040013
:10D180008A85858EC2061D08C1822312D400A68816
:10D1900081470147E51642864E85EFF07FB8410191
:10D1A0006F405FBB4A860A85EFF00FC0C9B7EF42F8
:10D1B000DFB8B335B000011185052A891315F601D2
:10D1C000336515012308B1009305110136843AC671
:10D1D00032C03EC442C2EFF00FBBA24712484255D4
:10D1E00093D68700230BF100930591019357880094
:10D1F000A30AD100A30BF100230C0101EFF0AFB89B
:10D200003247024603280400B337E0008356440047
:10D210009207914411C2A1444A85A68842860C080F
:10D22000EFF09F842A8909E5A6852285EFB03F9F0C
:10D230004A8505616F40BFB2EF429FAE01113EC605
:10D240008647B335B0008505AA891315F6015D8DB3
:10D250002308B1009305110136843A89B28442C48F
:10D2600046C2EFF04FB222489248164593578800C5
:10D27000A30AF1009305910193D78800230B0101C4
:10D28000A30BF100230C1101EFF0EFAF3247104078
:10D2900083564400B337E000920703280900914801
:10D2A00091C0A1480C084E85EFF09FA7AA8411E514
:10D2B000835544004A85EFB09F96268505616F40EF
:10D2C0007FA9AA959307F00F17F700001307478A65
:10D2D0006317B50013C5F7FF1375F50F82800505B9
:10D2E0008346F5FFB58FBA9783C70700D5B70357B5
:10D2F000450014419307F00F17F600001306468708
:10D30000369742074183139506014181631BE5006F
:10D31000AD8FB29703C50700130515F3133515003C
:10D320008280850603C5F6FFA98FB29783C70700E1
:10D33000D9BFEF429FA0B28736842E86BA86AA85CF
:10D340003E85BA84EFF06FE6634B05002285EFB0AF
:10D35000D0312A86A686A2852685EFF00FE56F409C
:10D360001FA0EF42FF9B5D712A8BAE8A17E500007C
:10D370001305857D2C00B284368ABA893E89EFF088
:10D380004FE42A8459E534104146DA852800EFF04D
:10D39000CFE12A843DED8547A303F100A6C29307A0
:10D3A00071002408BEC4A68685470D462C18281097
:10D3B00002DC02DED6C0BEC6EFF00FDB2A8431E904
:10D3C00083477102A6860D4693F7F7072300FA00FC
:10D3D000C1473EDE2C188947281026DCA303F10044
:10D3E000EFF08FD82A8415E54146A6854E85EFB02B
:10D3F000607F8D47A6860D462C182810A303F100E8
:10D40000EFF08FD62A8411E54146A6854A85EFB014
:10D41000607D228561616F40FF93EF421F9297D735
:10D4200000009387270C984383C7470079712A89A6
:10D43000AE8417E500001305A5710C083AC4230655
:10D44000F100EFF00FD82A8415E514104146CA8583
:10D450000808EFF08FD52A8411ED140815462C002A
:10D460000810EFF08FD42A8411E521462C08268578
:10D47000EFB04077228545616F407F8EEF42FF8B92
:10D4800097D70000938707069C477971AA842E845A
:10D4900017E500001305456C0C083EC6EFF06FD28F
:10D4A0000DE514104146A6850808EFF00FD011EDE8
:10D4B000140811466C000810EFF02FCF19E58347D0
:10D4C000F10193F7F7032300F40045616F403F89B2
:10D4D000EF42BF863688A14881470147E546EFF015
:10D4E000AFD86F40DF87EF425F853688A14881471C
:10D4F0000147E546EFF0DF826F407F86EF42FF8312
:10D5000001112A842E850C0832C6EFF08FCB19E961
:10D51000324797E600009386A6621008C14522852F
:10D52000EFF03FE105616F409F83EF421F814111A2
:10D53000C1472EC032C48A8509463EC23EC6EFF0BE
:10D54000AFC241016F40BF81EF422FFF4111AE8654
:10D5500013061009AA850A8502C002C202C402C6C7
:10D56000EFF0AFC441016F408FFFEF420FFD3287F4
:10D5700097E600009386C65E2E8693050002EFF0C4
:10D580005FDB6F40CFFDEF424FFB7971C1472ACC83
:10D590002ED032D42C080D4628003ECE3ED23ED6A8
:10D5A00002C402C602C802CAEFF00FBC45616F4058
:10D5B0000FFBEF428FF80111AA842E8417E50000BB
:10D5C0001305855A8A85EFF0CFBF05E5140841465B
:10D5D000A6850A85EFF06FBD09ED8347E10103479A
:10D5E000F101A207D98FCA07C9836177D98F2310A8
:10D5F000F40005616F40AFF605C9EF420FF497875D
:10D60000FF1F9387E76290439785FF1F938585628D
:10D610001785FF1F1305C55DEFB080091785FF1F34
:10D620001305055D6F40AFF31785FF1F1305455CBC
:10D6300082809DC5EF426FF09787FF1F9387475FFA
:10D64000944301112E840A869785FF1F9385855E7A
:10D65000EFB0800A0A850294014505616F402FF002
:10D660007D558280EF426FEDEFB080149787FF1FEA
:10D6700023A0A75C17F5FFFF130525F8EF90D04016
:10D680006F40EFED1787FF1F1307C75C9317150057
:10D6900008433E95FD572310F5008280EF42EFE9E5
:10D6A0002A84084019E16F408FEB1C4158401CC090
:10D6B0006313E5005CC08347550023200500F99BF8
:10D6C000A302F500EFB0EFF9E9BFEF426FE59787EE
:10D6D000FF1F9387275A98432A8411CB834735002D
:10D6E00093F7070289C7035505008945029713057B
:10D6F0004401EF901013835504000355E400EF201C
:10D70000701B485809C5EFB0CFF5232A0402130552
:10D710008403EFF0BFF88144B149EFA0FF9A63C5DD
:10D72000A402834734002320040493F727FCA301B9
:10D73000F4000048EFA05F9A13161500814522857A
:10D74000EF40AFE26F400FE1B387340303290403D6
:10D7500085043E994A85EFF07FF42304090075BFE4
:10D760008347350093F7070299E301458280835789
:10D77000E500E39CB7FEC167FD176316F60005459B
:10D7800082800545B9A0EF424FDB93170601C187A0
:10D79000B2842A8401496359F002835705008DCB76
:10D7A00001456367F600034584003E953325A600D6
:10D7B0001375F50F39A81C4813171900BA9783D7AA
:10D7C0000700E38097FC0509EFA01F91E345A9FE40
:10D7D00001456F40CFD8EF42AFD4AE89AA84EFA005
:10D7E0007F852A84EFD0BFAAAA8601471306840149
:10D7F00097050000938545E91785FF1F1305C5456B
:10D80000EFA0AFD52A8921CD8C441304C500228511
:10D810009E0593F50508EFB00FC5CC4083877400D3
:10D82000E18163D1070493E505082285EFB0AFC31A
:10D830000D46938544002285EFB00FC183D50400C7
:10D840002285EFB0EFC583D524002285EFB04FC508
:10D8500003D6490083A509002285EFB0EFBE4A85B3
:10D860006F404FCF93F5F507C9B7EF420FCD0111C8
:10D870002A84328532C6EFB06FB4EF903F91835760
:10D8800004001787FF1F130767563246231BF1005A
:10D89000930700F8A30DF1001C471843231AA100B9
:10D8A0008983858BB307F740B28548083ECE231C99
:10D8B0000100230D0100EFF01FF205616F402FCA38
:10D8C000EF420FC60041014529CC9304C4002685D0
:10D8D0003289AE89EFB08FB295452A8A2685035BDF
:10D8E0000401EFB02FAF2685EFB02FC68D45AA8A71
:10D8F0002685EFB02FAE2685EFB02FC55C48420AD3
:10D90000135A0A01D2975CC42318640181476398B3
:10D910003A0146054D81330625419337160013F52C
:10D92000F70F6F402FC3EF42CFBE89692A8BAE8BB2
:10D93000328AB68A81440144314CFD19EFA0CFF8F8
:10D9400063C9A400EFA04FFB018D33B5AA006F405F
:10D95000CFBF3389840383270B003E9963170A00E6
:10D960008347890085043E94D1BF03560A00DE85B3
:10D970004A8533F6C900EFF0BFF47DD10545C1BF3C
:10D98000EF42AFBB01112A847C000355E5003ECA7B
:10D99000B70707003ECC7C003ECEEF10303D2A8911
:10D9A00085454808EFB0EFC199454808EFB02FA76B
:10D9B000AA844A85EF10B03D2380A4009787FF1FFB
:10D9C0009387C7429C434166130606F093968701EE
:10D9D00013D78701558F93D68700F18E558FA207F5
:10D9E000B706FF00F58FD98F11462C001385140060
:10D9F0003EC4EFB0201F5008A38204008945228551
:10DA0000EFF0BFE609C9AA8513058403EFB0EFBBA9
:10DA10003C4085073CC005616F406FB4EF42EFB1F9
:10DA2000EFA08FED2A840504EFA00FEC3305A402CC
:10DA3000F14791453305F502EF10207B01E565556F
:10DA40006F40EFB19787FF1F23AEA720EFA0CFEA6B
:10DA50002A840504EFA04FE93305A4028945060591
:10DA6000EF10A07869DD9787FF1F23A5A71EEFA001
:10DA7000AFE82A840504EFA02FE73304A4029787B8
:10DA8000FF1F239B871CEFA02FE72A84EFA0CFE581
:10DA9000930714003385A7029787FF1F239FA71AB8
:10DAA00097E70000938707D01787FF1F232AF71AED
:10DAB000014579B7EF42CFA6AA842E890144978900
:10DAC000FF1F9389A932130A8006EFA0EFE1634597
:10DAD000A40001456F400FA83305440383A7090242
:10DAE0004A86A6853E95EFF0BFC719E10504F1BF50
:10DAF0000545CDB7EF42EFA1AA8A2E8BB28B368CAB
:10DB00003A8A814401448149978CFF1F938C0C2EE3
:10DB1000130D8006EFA04FDD63C7A40011E0854917
:10DB20004E856F408FA23389A40383A70C025E86C3
:10DB3000D6853E994A85EFF0BFC219CDEFA0CFDB65
:10DB40000544636B4501D2866286DA8513050903B5
:10DB5000EFF07FDD11C1854985046DBFEF424F9C19
:10DB6000C16441112A8901449789FF1F93890928BB
:10DB7000130A8006FD1436C632C42EC2EFA0CFD6DB
:10DB800092452246B2466346A400014541016F40DA
:10DB90006F9C3305440383A709023E9509C683475A
:10DBA0003500C18B9DC791C68347350093F70702A7
:10DBB0008DC3630699008357E500639C27010357D3
:10DBC000050001CB63E7E50083478500BA97E3CF03
:10DBD000F5FA05044DB7EF42AF94C1642A890144B8
:10DBE0009789FF1F93898920130A8006FD14EFA0EF
:10DBF000AFCF6344A4006F40EF953305440383A780
:10DC000009023E958357E5006388970063049900F5
:10DC100063942701EFF07FAB0504D1BFEF42EF8E95
:10DC200089692A8AAE8A328BB68B8144178CFF1F92
:10DC3000130CCC1B930C8006314DFD19EFA0CFCAFD
:10DC400063C4A4006F402F903389940383270C0290
:10DC50008355CA015A863E994A85EFF07FB005CDBB
:10DC6000814D05A03384AD038327090303D60B0040
:10DC7000D68533F6C9003E942285EFF07FC419E5BE
:10DC8000850DEFA06FC4E3CFADFC31A02285EFF08E
:10DC9000FFA023040400850455B7EF428F87416934
:10DCA000AA8A014A178BFF1F130B4B147D19C14B16
:10DCB000054CEFA06FC36344AA006F400F8993091E
:10DCC0008006B3073A0383290B02BE9983D7E90084
:10DCD000638C270163842A016398570103A4890395
:10DCE00011E44E85EFF0DFC9050AE1B7835704015F
:10DCF000639977079304C4002685EFA03FF085451C
:10DD00002A8D2685835C0401EFA0DFEC2685EFA039
:10DD1000FFFF62056185635F05028D452685EFA0E3
:10DD20007FEB89452685EFA0FFEA89452685EFA090
:10DD30007FEA85452685EFA03FEB8347050009472D
:10DD400093F7F7076398E70099452685EFA0DFE989
:10DD5000A30285014848337D2D01231894016A955B
:10DD600048C40040B5BFEF325FFD37E404008327AD
:10DD7000041D82979787FF1F83C747F41755FF1F1E
:10DD80001305453DA300F5008327441C8297832794
:10DD9000841C81461306F00F8145014582976F3040
:10DDA0001FFC1787FF1F130767E118439785FF1FA5
:10DDB00083C5C5F09787FF1F9387C7EE8346870308
:10DDC000034697036397D5009787FF1F2388C7EE05
:10DDD000828083C587010347A7036317B60097872F
:10DDE000FF1F238DE7EC828003C687016317C700FE
:10DDF0009787FF1F2384D7EC828083C68701130790
:10DE000050026319D700930760021787FF1F23078B
:10DE1000F7EA828083C68701130660026315D60085
:10DE200093077002DDB783C7870155BF9787FF1F30
:10DE3000938747E7D44B09476385E608EF32FFEF46
:10DE40001789FF1F130949E33E8483470900918B1B
:10DE50009DCFB7E4040083A7041D829783A7441CC9
:10DE60001785FF1F1305C5E1829783A7841C814690
:10DE70001786FF1F0346C6E281450145829721C1EF
:10DE800083470900ED9B1787FF1F2307F7DE8347B2
:10DE9000040093F7F70F85C791471787FF1F232DBE
:10DEA000F7E0EFF05FECEFF0DFEFB7E70400BC4F17
:10DEB000414691451785FF1F034545DF82976F3027
:10DEC0001FEA8280EF327FE78D4741116304F5043A
:10DED000C5476306F50285476310F5029787FF1F64
:10DEE0002380A7DEB7E70400BC4B9305001017851D
:10DEF000FF1F0345A5DB829741016F305FE6854731
:10DF00001787FF1F230EF7DAB7E70400BC4B930512
:10DF10000020F1BF9787FF1F9387C7D8D44B1147C5
:10DF2000638DE600B7E7040083A7071D8297B7E774
:10DF30000400BC4B930500045DBF05491787FF1F14
:10DF4000232C27D783C7070032C62E8493F7F70FF9
:10DF5000C5D7B7E4040083A7041D7D141374F40F20
:10DF60008297E37689FCB245994703C61500E3F032
:10DF7000C7FCFC4409061785FF1F1305A5D482972B
:10DF8000BC48930500081785FF1F034525D28297DB
:10DF900079BFEF329FDA1787FF1F1307A7D04047DB
:10DFA000184B1C409786FF1F23A4F6D06316E4008D
:10DFB0001787FF1F2320F7D0130584FEEF907FF310
:10DFC000035564FFEF903FC6EFA0BFE96F303FD924
:10DFD000EF32BFD69787FF1F9387C7CCD84BDC475C
:10DFE00099C3EFF01FFB85471787FF1F2326F7CC48
:10DFF0009787FF1F938787BC9C4393050002178573
:10E00000FF1F0345A5CA83C787031787FF1F230781
:10E01000F7CAB7E70400BC4B82976F305FD497878D
:10E02000FF1F23A3A7C88280EF329FCF37E40400ED
:10E030007C4CA1451785FF1F034545C782977C4847
:10E04000A1451785FF1F034565C69784FF1F93846D
:10E0500064C58297DC4489E7EFF05FDD6F309FCFC6
:10E0600003D567FFEF903FBCAA897DD5D84891477B
:10E070006310F7027C4C91451785FF1F034505C3CC
:10E0800082977C4891451785FF1F034525C28297DB
:10E0900003A9490103D409018947B7E90400178797
:10E0A000FF1F232BF7C083A7091D21044204829779
:10E0B00083C784011755FF1F1305C5096119175739
:10E0C000FF1FA309F70883A7491C41808297978700
:10E0D000FF1F238707BE83A7C91C81460946937586
:10E0E000F40F4A85829711E99787FF1F83C787CD71
:10E0F00089C79740FF1FE780A077B7E70400BC4FB0
:10E100002146A1451785FF1F034545BA8297B9B738
:10E11000EF32BFC293F7052001112E8481CBEFF0BF
:10E120003FEB1345042005616F307FC393F7051063
:10E13000A9CB9784FF1F9384E4B6DC48EFF07FC639
:10E140001787FF1F130787A7184383C78401034757
:10E1500087036316F700DC4499C3EFF09FE385471C
:10E160001787FF1F232AF7B4B7E70400BC4B9305BA
:10E1700000021785FF1F034565B3829713450410FE
:10E180005DB793F70508ADC79787FF1F83C797B3A0
:10E19000E91719469785FF1F9385E5B21305D1004E
:10E1A00093F4F70F1789FF1F0349C9B1EFA090231C
:10E1B00093970401C1831787FF1F130727B1231DFE
:10E1C000F100231CF1009787FF1F9387A7AD3ACE7C
:10E1D0003ACAD8432306010009CBDC4393158901D1
:10E1E00054080D46E185680082971345040825BF51
:10E1F00093F72500B1CF9787FF1F9387A7AAD84B26
:10E2000089476306F7029787FF1F83C7E7A613F7BF
:10E21000270011EF918B99CFB7E70400BC4F13068D
:10E22000000A89451785FF1F034545A882971345B6
:10E230002400D5BD9787FF1F938747989C4383C7CA
:10E2400087031787FF1F230BF7A6EFF0FFDDC5B786
:10E2500093F7050291C7EFF03FDD13450402E1B5E6
:10E2600093F7850091C7EFF0BFD61345840065BDD5
:10E2700093F7150091C7EFF07FBB1345140065B508
:10E2800093F7450091C7EFF07FBA1345440061BD95
:10E2900093F7050485C39787FF1F83C7A7A081CB8A
:10E2A000EFF07FAC91471787FF1F2327F7A0134597
:10E2B000040495BD93F705010145E38607E69787BA
:10E2C000FF1F9387279ED84B91476310F7049787CA
:10E2D000FF1F9387679A9C4313D727008583D98FA5
:10E2E000858B91E7B7E7040083A7071D8297B7E7FF
:10E2F0000400FC4F91451785FF1F0345259B82971E
:10E3000085471787FF1F2329F79A1345040121BD6D
:10E310009787FF1F2388A7AA8280EF321FA29787C3
:10E32000FF1F23A707989787FF1F23A507988547F7
:10E330001784FF1F130484881787FF1F232EF79667
:10E340001C4083C787031787FF1F2309F796EF90A9
:10E35000FFDF39C19757FF1F23A2A7E01C40170515
:10E360000000130525DB83C787031787FF1F2307DB
:10E37000F7941757FF1FA30FF7DC9787FF1FA3839F
:10E380000792B7E7040083A7070882979787FF1FC4
:10E39000238EA7906F30BF9CB7C7898E938767ED98
:10E3A0001757FF1F232CF7DA55BF1787FF1F0347A7
:10E3B000678F795555E39787FF1F9387A78E03C70C
:10E3C000170005079786FF1FA38EE68C03C717006B
:10E3D0008D463377D7029786FF1FA385E68C83C6C9
:10E3E00017001777FF1F1307677D184393F6F60F83
:10E3F000A9EA834787031787FF1F2301F78C854707
:10E400001787FF1F2300F78A9787FF1F9387C78609
:10E410009C430145998BA9E3EF323F9237E4040016
:10E420007C48C1451785FF1F0345458882973C48B6
:10E4300085451785FF1F03456587829701456F3026
:10E440001F9283C7170085466395F600834797039D
:10E450005DB78347A70345B782809787FF1F83C7B0
:10E460006784A1CBEF327F8D37E404009787FF1FCD
:10E47000238A07827C4885451785FF1F034505834E
:10E4800082977C4C91451785FF1F03452582829713
:10E490007C4891451785FF1F0345458182973C487D
:10E4A000C1451785FF1F03456580829701456F3081
:10E4B0001F8B79558280EF325F882A84035565FF70
:10E4C000EF906FF69777FF1F9387C77DD847BE847D
:10E4D0001DEBEFA05F989C48232004008DEB9777FD
:10E4E000FF1F23A9877C9777FF1F23A3877CB7E7AC
:10E4F0000400BC4B89451775FF1F0345257B829798
:10E5000001456F30DF85630A87001843D1B780C3A8
:10E510009777FF1F23A0877AD9BF7955DDB7EF32F0
:10E52000DF819787FF1F9387278A8843232605006B
:10E53000232405005105EF80D02E6F305F82EF322B
:10E54000CFFF1784FF1F130424881C40411189CF7B
:10E550009C472302B5002AC61CC1EFF05FFC1C409B
:10E560009C4B99C33245829741016F304FFFEF3288
:10E57000CFFC4111444D328532842EC6EFA00FF9F5
:10E580002AC42285EFA0EFF903A84400630C080019
:10E59000B245835744001840224683D54500AA86D9
:10E5A0002685029841016F308FFBEF320FF9404D05
:10E5B0001DC408C0970500009385E50213054401BA
:10E5C000EF8090189787FF1F938707809C43014532
:10E5D00089E79777FF1F23A9877E6F304FF87D5516
:10E5E000EDBFEF328FF5011168009305F00F02C601
:10E5F00002C802CA02CC02CEEFF07FF405616F3090
:10E600000FF69777FF1F9387277C9C43D847A16716
:10E610009D076311F702EF324FF201113285EFA02F
:10E62000EFEE230AA10081456800EFF05FF105617C
:10E630006F30EFF282809777FF1F9387E7789C43D4
:10E64000D847A167938777036311F702EF32EFEEA4
:10E6500001113285EFA08FEB230AA10081456800EC
:10E66000EFF0FFED05616F308FEF82809777FF1F2E
:10E67000938787759C43D8479547631CF702EF3211
:10E68000CFEB011132853284EFA04FE8230AA100BD
:10E690002285EFA00FE983574400231BA100814589
:10E6A0003ECC1C4068003ECEEFF07FE905616F3044
:10E6B0000FEB8280930785FF89CF8327C5FF91CB1E
:10E6C000DC4B81CBEF326FE7032585FF82976F30FC
:10E6D0000FE98280EF326FE62A843285EFA00FE3E4
:10E6E000BD4763EBA70018449377F5000345B700D7
:10E6F00041995D8DA305A7006F306FE6EF32EFE320
:10E7000001117C003ECAB70707003ECC7C003ECE1C
:10E710005C4D8DCF2A8413858700AE84EF80700412
:10E72000A1652A899D054808EF80FFBD9305803EBD
:10E73000B345B902480893F5F50FEFA0CFD20147D2
:10E7400081465008A6852285EF807FDC05616F3009
:10E750000FE1EF328FDEEFF07FFA6F304FE0EF32F4
:10E76000CFDD01117C00AE843ECAA165B70707006A
:10E770002A843ECC48087C00938575033ECEEF800A
:10E780009FB81C44480883C5B700BD89EFA0AFCD32
:10E79000500801478146A6852285EF805FD7056135
:10E7A0006F30EFDBEF326FD92A84AE84EFF09FF247
:10E7B000A6852285EFF0BFFA6F306FDAEF32EFD720
:10E7C000EFF0FFF96F30AFD9EF322FD70329C50132
:10E7D0004111630409022A843285B284EFA00FD369
:10E7E0002AC62685EFA0EFD3832749002A8691C742
:10E7F000DC4781C7B2452285829741016F302FD611
:10E80000EF32AFD3444D81CC2A843285EFA06FD153
:10E81000DC40AA8589C79C4799C3228582976F30BF
:10E820000FD4EF32EFCF032AC501411163030A066B
:10E830002E89AA84954532853284EF80DFAC8545E8
:10E840002285EFA0CFBDAA89CA852285EFA0EFC29D
:10E8500083274A009DC7DC438DC72285EFA0AFBA4E
:10E8600083274A00104083564400DC437115A307F8
:10E87000A100B2961307F1004E86CA8526858297BD
:10E8800001C52380090031A08345F1002285EFA056
:10E890000FB941016F300FCCEF322FCA65711C08E0
:10E8A0003EC2B70780013EC41C0832893EC62A8496
:10E8B000AE84EFF07FF14A85EFA0AFC68357A10089
:10E8C00089CFAA8550002285EFF0BFF50147814628
:10E8D0005000A6852285EF809FC359616F302FC8F5
:10E8E000EF320FC465711C088329C5013EC2B7070A
:10E8F00080013EC41C082A84AE8432893EC6EFF0F3
:10E900003FF0638409024A85EFA0AFC18357A1009D
:10E91000AA8581CF50002285EFF0BFF001478146E4
:10E920005000A6852285EF809FBE59616F308FC24F
:10E93000EF32AFC065711C083EC2B70780013EC40C
:10E940002A841C0832853EC6AE84EFA08FBD835753
:10E95000A10089CFAA8550002285EFF09FEC0147E6
:10E9600081465000A6852285EF807FBA59616F30BD
:10E970000FBFEF328FBC444D91E88347450093B7FA
:10E980001700B307F0403E856F306FBD1845FD5747
:10E990007DDB97070000938707032A845CCB9705EC
:10E9A0000000938565D113858400EF80E05980C015
:10E9B00003474400814761FB1777FF1F23289740D7
:10E9C000D9B7EF32EFB58329C5014111032985007D
:10E9D0008147638B09080324090191452A8A22850E
:10E9E000EF807F9285452285EFA06FA38945AA8A93
:10E9F0002285EFA0CFA2AA84EF809F9683A749002B
:10EA00002A8B9DC79C438DC72285EFA0CF9F83A7EC
:10EA10004900A306A1001040835644009C431307FD
:10EA2000D100B296D6851306E1005285829709CDB2
:10EA300083570B002380F400A183A380F40023807C
:10EA40000A00A306010029A88357E100228523803C
:10EA5000F4008345D100A183A380F400EFA02F9C94
:10EA60008347D100B337F0000347B900920701454F
:10EA70003D9BD98FA305F90041016F30AFADEF3257
:10EA8000CFAB41111DE99777FF1F93872734804350
:10EA900005C80440130984009DC55C4099C79C4B80
:10EAA00089C726852EC68297B2459307803EB385D7
:10EAB000F5024A85EF80605521A0404DAA8479F87F
:10EAC00041016F30CFA94A85EF80A0555C40EDDB56
:10EAD000DC4BFDD726858297E5B7EF320FA62A8457
:10EAE0003285EFA0AFA2AA852285EFF05FF96F30E3
:10EAF0000FA7EF328FA42A84AE84EFF01FFEA68505
:10EB00002285EFF0BFBF6F308FA508413355B500A8
:10EB100005898280EF326FA21774FF1F1304042D42
:10EB20001C5C0111231701008D83858BA303F10069
:10EB30008327040B231801002319010003D7C70101
:10EB40003ECA3C002314E1007D572315E100035722
:10EB5000C4023ECC02CE2316E100EF802FE38357A0
:10EB6000E101231EA10093F707E093E71710231F8D
:10EB7000F1009777FF1F83C7072A85C30547014523
:10EB8000638AE7008347840393E727001777FF1F13
:10EB9000230AF72805616F308F9C814717D7000043
:10EBA0001307471C85461306710085454808EF701A
:10EBB000E04B6DF183478403F59B1777FF1F230319
:10EBC000F72685471777FF1F2307F724E1B7EF32B2
:10EBD000CF93977DFF1F938D6D2103A6CD063971CD
:10EBE0002A8981478144930600023357F600058B3A
:10EBF00001C7850493F4F40F8507E398D7FE83A734
:10EC00000D0B231701022318010203D7C7013EDAB7
:10EC10003C102314E1027D572315E10203D7CD02F6
:10EC20003EDC231901022316E10202DEEF800FD63B
:10EC30008357E103231EA102014593F707E093E701
:10EC40001710231FF1029777FF1F83C7C71CA9EF77
:10EC50009777FF1F83C7171D3EC69779FF1F9389BC
:10EC6000E9180144014D9D4A054B954B177CFF1F48
:10EC7000130C0C1F977CFF1F938C0C1E03DAC90525
:10EC800063090A00EA85631459036685EFF0FFE71C
:10EC90001DC1050DA1478909E312FDFE2DE09777FF
:10ECA000FF1F23AD071A014521616F30CF896285AF
:10ECB000EFF0BFE579DD3247B3878400E3F0E7FE8C
:10ECC0009C001306140006043E9413178A00935701
:10ECD0008A00D98FC207C183A30EF4FCA183230F3E
:10ECE000F4FC03A70D07B317AB01D98F1777FF1FEC
:10ECF0002326F71663047601328461BF15449777A3
:10ED0000FF1F83C72711138717009776FF1F2383E1
:10ED1000E61093161400230EF10017D70000130716
:10ED20006704814785067008CA854818EF7000346B
:10ED3000E34705F68347C10105451777FF1FA30B7E
:10ED4000F70C9777FF1F2388270DB9BFEF225FFDD0
:10ED50000111AA892E84EFD0EF9C2A899774FF1F96
:10ED60009384C4086399090A9C5C414793F707039D
:10ED70006393E70A1777FF1F0347370A894763EC56
:10ED8000E70883A7040B231701002318010003D70A
:10ED9000C7013ECA3C002314E1007D572315E10062
:10EDA00003D7C4023ECC231901002316E10002CE92
:10EDB000EF80CFBD231EA100EFC06FCD8357C101EF
:10EDC000230FA100914613D78700A207D98F2312E2
:10EDD000F1009777FF1F83D7070513D78700A20796
:10EDE000D98F2313F10017D70000130727F78147A6
:10EDF000500095454808EF70602705889317240058
:10EE000003C484036D985D8C9777FF1F238C870064
:10EE100005616F203FF4EF70B0781775FF1F130581
:10EE2000E500EF80002083A7040B9775FF1F83D5B3
:10EE3000A5FE03D5C701EF10E0279777FF1F83C713
:10EE400067FE93F60702014789E61777FF1F03570E
:10EE5000A7FC9776FF1F2399E6FC1777FF1F130780
:10EE6000A7F7184309CBC18B99C789451775FF1FB1
:10EE7000035585FA02979777FF1F23AF07F8977717
:10EE8000FF1F238A07F89777FF1F23A707FC9777B1
:10EE9000FF1F23A507FC9777FF1F23A307FC83D73A
:10EEA000840393F7270C93E717001777FF1F231BA3
:10EEB000F7F683572903A18B99C3EF70E03F11C484
:10EEC0009777FF1F23A607F4A1B78D471777FF1F7A
:10EED0002320F7F4EF902FA59305803EB305B502EC
:10EEE0001775FF1F130585F4EF80201215B797776C
:10EEF000FF1F9387A7EFD85325C791C99777FF1FA7
:10EF0000238B07F09777FF1F23AA07F48280EF2255
:10EF1000DFE283C7F70241112EC685071777FF1F6F
:10EF2000A30DF7EE9777FF1F2391A7F09D47177763
:10EF3000FF1F232FF7ECEF900F9E2A84EF90AF9DD9
:10EF4000B24501E5EF902F9DAA85B305B440177532
:10EF5000FF1F1305A5EDEF80400B41016F203FE03F
:10EF600082809777FF1F938767E8D85331C7EF22D6
:10EF7000DFDC03C7F70205079776FF1FA38FE6E8DC
:10EF800011CD8C5F0D470145898185899776FF1FDB
:10EF900023A0E6E8EFF09FDB6F207FDC8547930539
:10EFA000C0441775FF1F130565E81777FF1F23215E
:10EFB000F7E6EF808005CDB78280EF221FD8177764
:10EFC000FF1F034747E58547631EF7009777FF1F3D
:10EFD0009387C7E183C7870393C787001777FF1F0E
:10EFE0002302F7E41775FF1F130545E4EF80600364
:10EFF000EF807FEF99471777FF1F232BF7E0977775
:10F00000FF1FA38C07E09777FF1F238607E0EF9091
:10F01000AF8F930740063305F5029777FF1F23AFA5
:10F02000A7DE6F20DFD39777FF1F83C7A7DFC18BD2
:10F0300099C7EF229FD0EFF0FFAD6F205FD26955E7
:10F0400082809777FF1F938767DADC5381CBEF22AB
:10F05000DFCE8545EFF09FCF6F207FD0828017777E
:10F06000FF1F1307A7D801468146BA852148631EB2
:10F0700006019DCA2390A60083C7850393E7170066
:10F080001777FF1F2300F7DA05A08357C705631D15
:10F09000F502F8598547B397C70093C7F7FFF98F73
:10F0A0001777FF1F232EF7DA9C5D9183858B85C729
:10F0B0009777FF1F83C727D699EFEF221FC81D45FB
:10F0C000EFF0FFB06F20BFC981E699E39306C70553
:10F0D0000506090769BF8280EF22BFC38605AA849F
:10F0E000B309B500977AFF1F938A0AD7054B977B20
:10F0F000FF1F938BABD6214C639434039777FF1F8C
:10F100009387C7CE9C5F9183858B89CB9777FF1FB1
:10F1100083C767D081E72145EFF07FAB6F20FFC247
:10F1200003DA0400630B0A041779FF1F130909CCE3
:10F130000144CA8C8357C905639D4703A285568540
:10F14000EFF0BF9C11E5A2855E85EFF01F9C05C91D
:10F1500003A74C07B3178B00D98F1777FF1F232105
:10F16000F7D083C78C0393E717001777FF1F230B94
:10F17000F7CA05040909E31F84FB8904B5BF231EF0
:10F180000904C5BF1777FF1F0347E7C88547631A00
:10F19000F700EF229FBAEFF05FE2EFF0BF976F202A
:10F1A0001FBC8280814785451306000293861700A5
:10F1B000B397F500E98F13F7F60F89E7B687E39762
:10F1C000C6FE01473A858280FD4785457D56B39648
:10F1D000F50013871700E98E1377F70F89E6FD17FF
:10F1E000E397C7FE01473A85828089E901473A855E
:10F1F000828001473A8541016F207FB6EF22FFB33D
:10F2000041112AC62E852EC4EFF0DFF9A2457D15E7
:10F210008547B397A700E39EF5FC32469377360007
:10F2200099C3719A11069777FF1F9387E7BB9443A1
:10F230003E871778FF1F130868BA89EA83270800FA
:10F240009107F19B9776FF1F23A0F6BA032588004C
:10F250001843B307A700B3F7B702B387F540FD150E
:10F26000FD8D83274800AA95B306B600E3F3F6F8B0
:10F27000E371D5F82E979777FF1F23A5D7B63DDB0F
:10F280003A858145EF207FAE2A87ADB71841977741
:10F29000FF1F9387A7B423A4070098C35841D8C37E
:10F2A0009777FF1F23A207B48280EF227FA7AA844B
:10F2B00001441779FF1F130969B39309400EEF80CA
:10F2C0007FD56345A40001456F20DFA833053403D3
:10F2D0008327090B3E958357C501E38797FE0504F5
:10F2E000F9BFEF221FA39779FF1F938929B03E84AE
:10F2F000BA848347060003A7090041119D83058B4B
:10F300003D8F83C74401AE8A2A89F99BD98F238A0E
:10F31000F4001C44B685231204001CC02285328AE6
:10F3200036C6EF90DF8FB246D2853686EF90900BCF
:10F33000DC4883A509000840858B56869D8DEFD05B
:10F340003FCC61E918407D5583475700034767006C
:10F35000A207D98FC207C1872394F4006358F00A2B
:10F3600083C7440193F70703B5CBD04893771600C2
:10F3700003A609001D8E9777FF1F9387E7DD9C4347
:10F38000ADEB814641A003A70B0093172A00BA9763
:10F3900018409443834757008345670033F656016E
:10F3A000A207CD8F6311F60283473700034647005B
:10F3B00003472700A207D18F4207D98FBD82B3F739
:10F3C0006701638AF604050AEF80DFC342059317DD
:10F3D0000A014181C183E3E8A7FA41BFA16A370B63
:10F3E0000200014A977BFF1F938B0BAEFD1A7D1B1A
:10F3F000E1BF83C7440113070003854693F7070362
:10F40000E391E7F8A2854A85EFD0FFCF41016F2055
:10F41000DF936155E5BF7955D5BFEF227F90977493
:10F42000FF1F9384E4849C40D9EF9777FF1F938755
:10F43000679A9C436399070CEF80DFBE93078002B5
:10F440003305F5028945EFF05FDA41C99777FF1F71
:10F4500023A4A7A4EF801FBC9307400E3305F50239
:10F460009145EFF09FD835C99777FF1F23A8A7A232
:10F47000EF805FB201CDEF80FFB191450E05EFF057
:10F48000DFD621CD9777FF1F23ACA7A0EF801FCB3E
:10F4900011CDEF80BFCAD9473305F5028945EFF09A
:10F4A000DFD405CD9777FF1F23A6A79EEF809FB5DA
:10F4B00091450A05EFF07FD30DC19777FF1F23A574
:10F4C000A7A0014521A8EF803FC29307800633051E
:10F4D000F5029145EFF07FD101E565556F209F87DB
:10F4E0009777FF1F23A4A7920144130A8006177978
:10F4F000FF1F1309A98FB14AEF801FBF6364A402E5
:10F500009C40E38407F2EF803FBE9307A0043305DD
:10F51000F5028945EFF07FCD69D19777FF1F23A9C9
:10F52000A79A19BFEF805FBB89450605EFF0FFCBB7
:10F530004DD5B3094403032709024E9708CBEF804A
:10F54000BFB8330555039145EFF03FCA59D583271E
:10F55000090205041374F40FCE9788DB71BF977707
:10F56000FF1F9387A788884705898280C167FD1799
:10F570006319F5009777FF1F9387478703A5070B4C
:10F580008280EF228FFBEFF05FD26F204FFD81472B
:10F5900009C58347E501B337F0001777FF1F13074D
:10F5A000E78418470983058B19C393E727003E8535
:10F5B0008280EF228FF82A84EFF07FFD8347E401F9
:10F5C000AA851305940899E3130504039776FF1F92
:10F5D0009386C6819442130615021307840213050D
:10F5E0009504EFD0CFC06F208FF7EF226FF39764B1
:10F5F000FF1F9384A47F98442A892E840983058B56
:10F600009C4019C76314F5006380050E014401A2F4
:10F61000E3FEA7FE1387A702E36AA7FE850763FC44
:10F62000A70883A9440BEF80FF9613163500814588
:10F630004E85EF208FF39767FF1F23A9277B9767DE
:10F64000FF1F23A7077A49CC9C4493E7470017671D
:10F65000FF1F2321F77A9777FF1F23850780630F0A
:10F66000040C9767FF1F23A3277901440549EF8006
:10F670007F926341A40AEF80FF9493050006B3C50F
:10F68000A502B7F73600938707E81765FF1F130534
:10F69000A57D416901449309400E7D19B385F502AA
:10F6A000EF70B016EF801F97634FA4080145EF304D
:10F6B00040700544A9A86398A7029DE583A9440B5F
:10F6C000EF805F8D1316350081454E85EF20EFE901
:10F6D0009767FF1F23AC27719767FF1F23AA077047
:10F6E0009C44ED9BADB785C51767FF1F0347877720
:10F6F0009307F005E3FCE7F021F8EF60F03C6DD1F3
:10F700009C4493E707021767FF1F2325F76E2285A6
:10F710006F204FE483A7440B131534003E958357A5
:10F72000050081CB8347250099C721468145EF20FD
:10F73000CFE305042DBF23012501E5BF9767FF1F18
:10F7400023A8076A0DBF3305340383A7040B3E9536
:10F750008357C50163842701EFF0BFE5050499B71E
:10F76000EF22AFDDEF801F86130400063345A402AD
:10F770009764FF1F9384846783C784073E9513753E
:10F78000F50F9767FF1F238FA76C9307F00563E7BB
:10F79000A7020545EF30E061EF80DF823345A40228
:10F7A000B7F53600938505E8B305B5021765FF1F69
:10F7B0001305856BEF7070056F206FDA9C4405456B
:10F7C0008983858B81CBEF904F8888408145EFF00E
:10F7D000DFE1DDB7EF30E05DC5B7EF226FD4130492
:10F7E00095082A8913069005A28513050503EF9055
:10F7F000603F1306900581452285EF200FD74A858B
:10F80000EF30C0548144176AFF1F130A2A5E930A1F
:10F810008002EF803F8163C4A4006F20AFD33384A4
:10F8200054038327CA0A3E94035704008357C9012F
:10F830006317F702834744009DC39309640145465B
:10F84000CE8513055400EF90E039454681454E853D
:10F85000EF20AFD1228523020400EF30005785044A
:10F860004DBFEF228FCD9767FF1F938767409C4363
:10F870002A8491C70DC50355C501EFE00FC29777E4
:10F88000FF1F9387678D9C4389CBEFB0DFD08547FF
:10F890006315F5002285EF50C05D6F204FCC4165A8
:10F8A0007D15E1BFEF226FC91764FF1F13040454D5
:10F8B0004440938714001767FF1F232BF752EF3044
:10F8C000605E1C448983858B9DE75840B7E7B00094
:10F8D0009387075063F1E7020145EFF01F9D01CDCB
:10F8E0000545EF809FF6084085450505EFF0FFCF01
:10F8F0000145EFF01FF726856F206FC6EF224FC23C
:10F90000A1642A8901449769FF1F9389E95BFD146B
:10F91000338AA500EF800FEF6344A4006F208FC3EC
:10F9200003A7090093172400BA979843658F4207ED
:10F930004183634C2701635A470123800700A3805A
:10F94000070023810700A38107000504E1B7EF2228
:10F95000CFBB83594500C547411163F53731044199
:10F96000C1E533853401834785FF034795FF03488D
:10F97000B5FFA207D98F0347A5FFC2072207336748
:10F980000701D98F0347C5FF0348D5FF2207336717
:10F9900007010348E5FF0345F5FF420722083365E9
:10F9A000A800498FB98F1767FF1F1307A74F176864
:10F9B000FF1F130828513A85832807006384172BFB
:10F9C0001107E31B07FF1767FF1F1307A74F184314
:10F9D0001318270042951CC10507A1473367F7029A
:10F9E0009767FF1F23A0E74E93F735001397470053
:10F9F00083474601C16B368993F7F7FCD98F328470
:10FA00002E8A230AF600814A176CFF1F130C0C3E46
:10FA1000FD1B976CFF1F938CAC25176DFF1F130DFB
:10FA20002D4BEF802FDF63C7AA00E15426854101EB
:10FA30006F206FB11308400EB3870A0303280C0B25
:10FA4000B30DF800638E0D2083D7CD01638A772133
:10FA500083A70C00014B639707169767FF1F9387D7
:10FA600067379C436390071683C7040003C70D04E0
:10FA700093F7F707631BF71ACA872287CE86268675
:10FA800093859D0613851D04EFF0BF85631F051840
:10FA900083D7CD01032709002320B4012312F400EA
:10FAA000FD572313F4008347170093F6F7078347A6
:10FAB000D40093F707F8D58FA306F40093F7F70760
:10FAC000B337F000B307F0402307F4008347170073
:10FAD0009D839396370083474401DD9BD58F230A8E
:10FAE000F4008347370083464700A207D58F83463B
:10FAF0002700C206D58F1CC88347770003478700BD
:10FB0000A207D98F2315F4000D476304EA00BD5402
:10FB100091DF93870710C207C1831307B00FBD544D
:10FB2000E376F7F0EF800FC98144E31105F09766A3
:10FB3000FF1F83C6A639938716001767FF1F230789
:10FB4000F7381767FF1F13072738231BD400939735
:10FB50002600144303578400E175BE96A1671386FF
:10FB6000F7FFB377C70098426D8FD98F9CC21848B2
:10FB7000F18F3E07D98F9CC2EF80CFC89767FF1FD8
:10FB800083C7C73433F5A7029767FF1F2380A734C5
:10FB900071BD9307A004B308FB0283270D00BE9834
:10FBA00003D7080083D7CD01631DF70083C7040086
:10FBB00003C7880093F7F707630BF70083C7FD01BE
:10FBC0009DEB050BEF804FD2E345ABFC71BD9385F8
:10FBD000980113859800CA872287CE86268646C656
:10FBE000EFF02FF0B24879F98347440193E74700DB
:10FBF000230AF40071BD83C7040003C7980293F77A
:10FC0000F707E310F7FCCA872287CE8626869385FE
:10FC1000A8031385A802EFF0CFEC45F58347440114
:10FC200093E72700230AF400C1B783C7FD018DCBFA
:10FC300083C7040003C79D0993F7F7076312F70210
:10FC4000CA872287CE86268693852D0C1385AD091B
:10FC5000EFF02FE911E58347440193E7270049BFFF
:10FC6000850AC1B3FD54D9B3EF22AF8A79718354A9
:10FC70004500AA8B2E84B28AEF80CFBB5905634919
:10FC80009504B7E4040003A90407EF80AFBA59054F
:10FC90004205418102992A8905CD2AC6231801000F
:10FCA000EF804FB959052319A10061468145280805
:10FCB0009769FF1F938989134ACAEF200F8B23028C
:10FCC000810203A48900058819E4BC544A858297FF
:10FCD00045616F208F8774003008D6855E85EFF010
:10FCE0001FC765F56800EF807FF1176AFF1F130AD1
:10FCF000AA4683270A00AA84035B010189CB8947AE
:10FD00006397FA00835501025E85EF50203003555A
:10FD10002102EF704FC819E503552102EF708FD40F
:10FD20003334A000931764000344C1022C08680018
:10FD30001374F4FB5D8C23068102EF60B056E95723
:10FD40006314F5028356E1029767FF1F9387C71775
:10FD50009C43139726006176BA979843718F98C396
:10FD60009767FF1F2384D716831721026345F0008E
:10FD700085476396FA00B25793F7070C95E7D24789
:10FD8000C2040347C102C180BE9426C62318610184
:10FD900013770703C147631DF700834751020547E7
:10FDA00093F7F7076390E704B7E70400BC5739BF40
:10FDB00092570544A18393F7F707E377F4FE15C73D
:10FDC0008347C1021307000293F707036397E70015
:10FDD000EFB06FFC8547E319F5FC8347C10293F749
:10FDE000070389CFEFB0AFCA21A8EFB08FD7E309DF
:10FDF00085FCEFB04FFAE31985FAD9B7EFB0EFD829
:10FE0000AA8501460545EF707FF82A8451DD8347B6
:10FE1000C102414793F707036384E70232478347F0
:10FE2000170093F707F8A300F7003247925783466D
:10FE30001700A18393F7F707FD17D58FA300F700ED
:10FE400003560101B245130BC4005A85EF80DFDF72
:10FE5000E24A130690058347C10283C4EA01918BED
:10FE6000B384C40213851404569595C35444B387D0
:10FE70009A0083C7070403C70600137707F8238097
:10FE8000E600584483460700D58F2300F700B25799
:10FE900003A609008146858B1D8EDA85EFD0EF9B86
:10FEA00015E9B25783A50900484413869406858B4B
:10FEB00056969D8DEFD0CF9411ED83270A0099EFD0
:10FEC000B257054791838D8B6387E7049DCF094720
:10FED0006389E7042285EF80DFF8F9B5EFB0AFEB77
:10FEE00085476309F5008347C102414793F707033C
:10FEF000E398E7FC835521025A85EF40907C69D155
:10FF000083172102E35EF0FAF1B7EFB08FC57D15DC
:10FF10001335150061D1014681452285EF70FFEF51
:10FF200055BFEFB04FE7E5B7EF123FE19764FF1F12
:10FF3000938444ED2685EF809FEB2A8419E16F10AE
:10FF40001FE21305C40005468145EFF0FFD122856D
:10FF5000EF803FF1C5B7EF125FDE4111AE842A8416
:10FF600093079503130715019306F10005466C00EE
:10FF7000268523060100EFD0CFBE1DEDA6854146A4
:10FF80002285EF8030468347F100930514022685D1
:10FF90002308F400EFD06FC805E19767FF1F938730
:10FFA000A71B9C4389EF1306940497C50000938513
:10FFB000E5DB2685EFD08FD441016F105FDA1306A1
:10FFC000940297C500009385E5DA2685EFD00FD31C
:10FFD00079D9DDB7EF12DFD49767FF1F9387C7EE9C
:10FFE0008043AE84B289368AAA8AEF80AF81131625
:10FFF000250081452285EF105FD79767FF1F238774
:020000040001F9
:1000000007EC9767FF1F938767DE03A4070B13F7BF
:1000100014003E89230FE400CE8525C713059408FC
:10002000EFF07FF301C555556F10DFD28947A30F5D
:10003000F4009767FF1F938727129C4303278900CB
:10004000858093B7170086072300F402231E54010E
:100050009767FF1F23AC47D985889377B7FF99C06F
:10006000936747001767FF1F2326F7D8228593075A
:1000700000061767FF1F2307F7DEEFF08FD3014558
:1000800065B713050403EFF01FED45D569BFEF1207
:10009000DFCAFD572310F5002311050023120500C8
:1000A000231305001306200481452105EF10FFCB23
:1000B0006F10FFCAEF12DFC64111AA84014417690D
:1000C000FF1F1309E9E09309A0042EC6EF80CF813A
:1000D000B2456344A40061550DA033053403832762
:1000E00009003E9583572500639CB70083570500A0
:1000F00063989700EFF0BFF9014541016F109FC56C
:100100000504E1B7EF12DFC19767FF1F938787CC24
:100110009C434111AA842E84B28903592500C1C38E
:100120009767FF1F83D747CF639B2707EF700F8623
:100130002A8903D5240093051002B305B40285472C
:100140002302F10093578900A302F1009357850021
:10015000A303F10083D744002304A100254613D74D
:1001600087002305F10083D76400A304E1004E85D6
:1001700013D78700A305E1002306F100138795003C
:1001800093879501A105B386B400A6974C002697E6
:1001900023032101EFD0EF9C41016F10BFBBEF6043
:1001A000FFFE51BFEF12DFB74111AA840144176966
:1001B000FF1F1309E9D19309A0043AC636C432C21D
:1001C0002EC0EF707FF282451246A246324763444A
:1001D000A400615599A0B307340303250900AA9729
:1001E00003D8070003D5C4016310A80495E91DEEE8
:1001F00091CA03C6E401930510023306B602250630
:100200003E9690C2014511CB83C6E401130610024D
:10021000B386C602E506B6971CC341016F109FB3B3
:1002200003D52700E305B5FC050441BF83C5E40100
:1002300013051002B385A502BE9583C58500230072
:10024000B6007DB7EF12DFAD5C4141112A8403DABD
:100250002700C167FD17AE843289630CFA0026853A
:10026000EF807F9A8D4763EDA7007D5541016F10A8
:100270007FAE2E85EF803F999D47E3E2A7FEF5B75D
:100280005C40268583D54700EF809F90835584008E
:100290002685EF80FF8F8D452685EF803F8EAA89CA
:1002A000EFF04FE0935705012380F9009357850045
:1002B000A380F9002381A9005840C167FD17834539
:1002C000A7006314FA0093E505082685EF801F8FC9
:1002D0009767FF1F938707B09C430840D9CF834798
:1002E000B400858BD9CB78003400130671008145AA
:1002F000EFF05FEB1DC98347B400184093069005EB
:10030000F99BA305F4008347E701B387D702B3063F
:10031000F70083C60604A303D100938617049387CE
:100320009706BA96BA9736C43EC61764FF1F1304E1
:10033000E4AB1C440C4026858983858B9D8D8347C7
:1003400071009E05DD8D93F5F50FEF803F871C440E
:10035000104022458983858BCA861D8EA685EFC0F5
:10036000DFCFE31505F01C440C40324689838840FA
:10037000858B9D8DEFC0DFC8D5BD8347B4001307C3
:100380009005F99BA305F4008347E501B387E702D5
:100390003307F50003470704A303E100138717049D
:1003A000938797062A973E953AC42AC6BDBFEF1297
:1003B0003F97032A45009307F00FAA840347AA003A
:1003C000AE89328436896316F700EFB06FAB230530
:1003D000AA00938AC9000146D6852685EFF09FE6DC
:1003E0002A8A21E51767FF1F130707D71843DC4048
:1003F00039C383C6A7000547638FE60283D547004C
:100400005685EF40102C05C9DC40839747006354A4
:10041000F00201CC1C4089C74A868145014582977C
:100420005C4081C7CA85014582974E85EF807FA3D6
:1004300052856F103F92DC4003D54700EF60BFD577
:1004400001E9DC4003D54700EF60DFE181471DCDC6
:1004500019C41C4089C74A868145014582974E854B
:10046000EF807F9FAA851765FF1F1305A599EF8071
:10047000DF9511C45C4081C7CA8501458297176525
:10048000FF1F13056597EF60F0368547D840854616
:100490000346A700E30BD6F8031747006353E000B9
:1004A000C9F74A86A2854E85EF703F97BDBFEF1210
:1004B0003F87AA8401441769FF1F130969A19309A3
:1004C000A004130A9508EF703FC26344A4000145DD
:1004D00035A033053403832709003E958357250053
:1004E00099E30504CDB70357050083D7C401E31A88
:1004F000F7FE52868545EFF0FFC065D56F109F85EA
:10050000EF121F82AA8401441769FF1F1309499C37
:100510009309A004EF705FBD6344A4006F109F8334
:1005200033053403832709003E958357250081CF87
:1005300083570500639997009305950213061002EF
:100540002105EF80206A0504F1B7EF120FFF034782
:10055000E5012A848347F5016307B70089E78145F0
:100560002E856F10CFFF230FB400054781C9E39894
:10057000E7FE8947A30FF4008545DDB7638BE702EB
:100580000947E39FE7FC2285EFF02FA59767FF1F40
:10059000938747849C4399E79757FF1F9387476D3D
:1005A0009C4389C70355C401EFF09FF5A30F0400D6
:1005B000E1B755D6C9BFEF12AFF6EFA0FFEE854702
:1005C0006312F508EF80EFCC1764FF1F1304C4B863
:1005D0001C4081CBEFA03FFC89476304F5001C4021
:1005E00082979757FF1F9387E77E9C43B9CF8297E7
:1005F0009757FF1F9387C7679C4391C382971754F0
:10060000FF1F1304A47E8327040B83D4C701EF606C
:10061000FFB78327040BAA85144003C6E7011C44D7
:100620008983858B99C31366260026854169EF402F
:10063000C03D8144D9497D19EF705FB063CAA40001
:100640006F104FF1EF800FCA41B7EF705F884DB761
:10065000B38734030327840ABA9703D527006308B6
:10066000250103C6470183D50700EF40A03B850461
:10067000E1B7EF12EFEA01449754FF1F9384047728
:100680001309400EFD59EF70FF98634FA404014415
:100690009754FF1F9384847513098002FD59EF70EE
:1006A0007F98634CA40401449754FF1F93840474FF
:1006B0005949FD59EF709FA8634AA40497F5FFFFBD
:1006C0009385450A1755FF1F1305057AEF60D0077C
:1006D00097050000938585851755FF1F1305C57184
:1006E000EF6050056F100FE73307240383A7040B57
:1006F0000504BA97239E370179B73307240383A7EC
:10070000C40A0504BA972390370151BF3307240365
:1007100083A7840A0504BA972391370161BFD441A6
:100720000387350085473356F5026377E600A54811
:1007300099E7238006008280B387E702EDB733583C
:10074000F502038735003375F502B3D7E7021307C7
:10075000000363DA080103C6050013077003118A5A
:1007600019E21307700585064297A38FE6FEC9B705
:1007700018451C416376F7005C41BA972380B700A7
:100780001C4585071CC58280EF122FDB4111AA870B
:100790002E85B285368636C6829763480500B246F6
:1007A000158D3335A0003305A04041016F102FDBBC
:1007B000EF120FD7056941112A8A23200600014450
:1007C0008149975AFF1F938A2A73056B7D1932C698
:1007D0002EC4EF703F85AA84EF70DF832695A24573
:1007E00032466346A4004E8541016F10AFD603A781
:1007F0000A0093171400BA9703D7070033776701ED
:1008000001E71CC20504E1B703D707009356D700E0
:10081000858AE39946FF33772701E315B7FEBE8942
:10082000D5B7EF128FD101112EC6B2843689EFB041
:100830002FEE2A84615501C8B24589E9232E0400B0
:1008400023200402014505616F106FD1A1463008D5
:10085000CA852685EFF05FF37DF583578101035745
:10086000A101231EF4008357C1012310E4022311C8
:10087000F4028357E101D207D1832312F402835794
:10088000E1011397370163560700FD57231FF4005A
:100890005DBF231F040045BFEF128FC81754FF1F11
:1008A0001304C4548327040B03D7C701C167FD1782
:1008B000630EF7109767FF1F9387478A9C4381C792
:1008C0000545EF406077C1690149930A400EFD1963
:1008D000176BFF1F130B4B88EF70CFF3634BA90E01
:1008E0001757FF1F034707589307F00563E4E70214
:1008F000EF704FED93050006B3C5A502B7F73600BC
:10090000938707E81755FF1F13050556B385F502B2
:10091000EF60A06F81451705000013058520EF608B
:10092000DFF8EFB0EFDE01CD0357C50109CB035768
:10093000E50111C78347050299C3EF60A06BEFB0D3
:100940006FDE31C51757FF1F0347875E9757FF1F9D
:100950009387075E0DCF03C717002304E50003C785
:100960002700A304E50003C737002305E50003C7FC
:100970004700A305E50003C757002306E50003C7AA
:10098000670083C77700A306E5002307F5001C4432
:1009900093E717001757FF1F232EF7445C4085E7A6
:1009A000EF708FEF0DC1EF702FEF44402A89EF7089
:1009B000AFEE33F5A4025C40FD17CA97898F175735
:1009C000FF1F2327F7420145EF70DF9F01456F109E
:1009D0006FB8B30459038327040BBE9483D7C401B3
:1009E00063883703138A0403D2855285EFF0AFD6AC
:1009F00005E183C7F40199CF938594082E85EFF024
:100A00008FD509C91306900581455285EF10EFB5C2
:100A10000509D9B583270B00268593B717008607EC
:100A20002380F402EFE0FFB8E5B7854763F8A7003D
:100A30009307F5FFBE953305A040E98D2E85828092
:100A40009841C167BA9713D707016304A7009CC1F7
:100A500082804207998FE5BFEF122FAE41112EC65B
:100A60003284B684EFB00FCCE15701C9B24591E9A9
:100A70009757FF1F238E074A81473E8541016F101C
:100A80000FAE9D461756FF1F1306964AA685228570
:100A9000EFF09FCFAA8775F105479756FF1F23896F
:100AA000E648E1BFEF12CFA7411191E99757FF1F29
:100AB00023A007340144228541016F10AFA9B685F8
:100AC00032858D467000EFF03FCC2A846DF5834768
:100AD000D1000347E1001759FF1F13092931A2076D
:100AE0004207D98F0347C100D98F1757FF1F232112
:100AF000F730EF706FDA61D1EF700FDA83244900BD
:100B0000AA89EF706FD933F5A40283274900FD1736
:100B1000CE97898F1757FF1F232CF72C69BFEF1231
:100B2000CFA11C45AA8491CFD84B01CF83D74700D2
:100B300089CBEF601F92AA8509C588446105EF60E3
:100B4000C04C9757FF1F9387E7289C43014489EFC8
:100B50006F10EFA09C4813171400BA9703D5070035
:100B600019C1EFE0CFCF0504EF70CFC7E344A4FE77
:100B7000C5B7EF128F9C011185E9EF605FDA014480
:100B80009757FF1F23A007309757FF1F23AE072E4D
:100B90009757FF1F23AC072E9757FF1F23AA072E37
:100BA000228505616F10AF9BB6873285C9467000FC
:100BB000BE85EFF07FBD2A8465F541469305E100CF
:100BC0001755FF1F1305052CEF80C0010355C10009
:100BD000EF608FD7F1B78DE19757FF1F23A807204C
:100BE0009757FF1F938787209C470145ED9B175719
:100BF000FF1F2321F7208280EF122F944111B68529
:100C0000328595463000EFF03FB815EDA2471757F3
:100C1000FF1F232DF71C9757FF1F9387271D94470E
:100C2000B24713F7B6FF13F6170019C213E74600D1
:100C3000858393F7F7079756FF1F23ADE61A1757DB
:100C4000FF1F2301F72241016F106F91EF124F8DAB
:100C500003841500DC412A89AE8485070387F7FFEA
:100C600019C36340800C8387240091C763558000BB
:100C70007D14620461849C40370700FF0907F98FE7
:100C80003707001009076392E70A6355800079145B
:100C90006204618483C70400858B95E39379F40F24
:100CA0004E8A93178A01E187634AF008A28763534B
:100CB000040081473384F9407D1462046184838594
:100CC000240081C54A85EFF0BFAA9C40370700FF8A
:100CD0000907F98F370700100907639AE70693059C
:100CE00000034A85EFF0DFA883C704009305800561
:100CF000918B99E3930580074A85EFF07FA783C71F
:100D00000400858B81CB1374F40F93178401E18762
:100D10006347F004C04005048305F4FFA1E96F10A8
:100D20006F837D14620461840DBF370700080907D3
:100D3000E392E7F6E35080F67D1499BF9305000235
:100D40004A857D1AEFF0DFA2137AFA0F99BF3707B1
:100D500000080907E395E7FA9305000371BF9305BF
:100D600000034A85EFF0DFA07D1471BF4A85EFF0E4
:100D70003FA055B7EF027FFCEF70CFAA2A84EF7037
:100D80006FA9229589450605EFE02FC6E55711C5E5
:100D90009757FF1F23A2A71681473E856F003FFC90
:100DA000930700026306F5005D1513355500828038
:100DB00005458280EF02DFF64111AA892A891304D2
:100DC00019008304F4FF32C62EC42685EFF05FFDC0
:100DD000A245324659E19307D0026392F408830496
:100DE00004000548130429009377F6FEC9E793072A
:100DF0000003639FF40E830704001307800593F735
:100E0000F7FD6399E7068304140041460904B70619
:100E100000806314080093C6F6FFB3FEC602814744
:100E2000254F654EFD5F33D3C602138704FD63680B
:100E3000EF06BA8463D5C408630DF5017D55636A76
:100E4000F3006394670063C69E000545B307F6028E
:100E5000A69705048304F4FFC9BF22898DB79307C1
:100E6000B0020148E392F4F8830404002A881304D2
:100E700029009DBF01CA8947E31BF6F893070003C9
:100E8000E397F4F8830704001307200493F7F7FDB2
:100E9000639BE70483041400094609048DBF13E72C
:100EA00004021307F7F9636CEE009388F4FB130751
:100EB000700363741E0113077005998CA5BF7D57DD
:100EC0006300E50263040800B307F04091C519C14F
:100ED0009309F4FF23A035013E8541016F009FE790
:100EE000B687FDF5D5BF9304000315F2214605B77B
:100EF00019FE294629BFEF02BFE2011161540DC559
:100F00003284AE89414681453689EFF0BFEA9314B9
:100F10000501C180639E09002685EF30102B014436
:100F200001C58145EF205016228505616F009FE2C3
:100F30002285CD467000CA85EFF01F852A846DF5A5
:100F40002685EF30902809E90356C1008345E10169
:100F50002685EF20500B01C941469305E10011059C
:100F6000EF705048D1B75D54C1B7EF027FDB01117C
:100F7000E15401CDB284AE89414681453689EFF016
:100F80007FE32A84639709008144268505616F0009
:100F90007FDC2685D1467000CA85EFF0EFFEAA847B
:100FA0006DF58357C100EDD3EF700F8E4205931797
:100FB00004014181C18363F9A702EFB08FB64204F7
:100FC000E14741803304F40241460C082A9413059A
:100FD0004400EF7030418357E1002311F400835740
:100FE000C1002310F40055B7E55445B7EF025FD3B5
:100FF0007971E15415C53284AE8941468145B68484
:10100000EFF05FDB1319050113590901639E090015
:101010004A85EF401065814401C58145EFB02FB18D
:10102000268545616F001FD3A685930630027000A8
:101030002285EFF06FF5AA8465F54A85EF4070626E
:101040002A8411E54A85EFB04F8C2A8431C5835735
:10105000C10023112401930964002310F400834785
:10106000E1009305F10041462302F4004E85EF7044
:1010700070371309740141469305F1014A85EF70F9
:101080007036930554004E85EFC04FBF9305640141
:101090004A85EFC0AFBE69B7DD5459B7EF025FC8EC
:1010A000797111E5E154268545616F00BFCAB284AC
:1010B000AE89414681453689EFF0DFCF131A05012D
:1010C000135A0A015285EFE06FCA2A846398090017
:1010D00071D98145EFB02FB48144F1B726859306CD
:1010E00010027000CA85EFF02FEAAA844DFD31C8C6
:1010F000B2479305D1004146858B230FF400B247D8
:1011000013050403858393F7F707A30FF400EF702B
:10111000702D41469305D10113059408EF70902C72
:1011200059B73304690383A70A0B3E948357C4015C
:10113000638337030509EF60FFEDE344A9FEDD5447
:101140009DB7C1690149975AFF1F938A2ACA130B99
:10115000400EFD19CDB7231E440159BF49CDEF0202
:101160003FBC4111B289AE8441468145368AEFF0D9
:101170007FC4931A050193DA0A010149175BFF1F27
:10118000130BCBC6EF601FE1634AA9000145ADCC4C
:1011900081441759FF1F130969C581A883274B0B89
:1011A000131439003E9483570400638857050509DA
:1011B000D1BF8327490B139434003E948357040016
:1011C00085E72310540191467000D2854E85EFF0DB
:1011D000AFDB1DE9B24713978700E1832183858B3D
:1011E00058C02301F4000DA08504EF60BFDAE3C20C
:1011F000A4FC5D5511A861558280F1F4214681451A
:101200002285EF009FB6014541016F00BFB41971FF
:10121000D2C4130AC10686CEA2CCA6CACAC8CEC6FC
:10122000D6C2B6D6BAD8BEDAC2DCC6DE52C4638134
:101230000524FD151C102ACC2ECA02CE3EC89304EC
:10124000B0021549A94983050600130416009DE163
:10125000F2465247E24763FBE620B6972380070039
:101260007245F6406644D6444649B649264A964AEF
:1012700009618280930750026386F5004808EFF009
:101280002FCFF5A88357C10023070100014593F72D
:10129000C70F2316F10081450148014701468146E9
:1012A0009308D00213030003130E300205048307D2
:1012B000F4FF99C7638C970463C3F404638BC70579
:1012C00001CA0346C100858A799AD18E2306D100CE
:1012D000630908008346C100098BF59A558F2306E0
:1012E000E10019C12307B100138707FD1377F70F3A
:1012F000A54663E2E6068146A545294535A0E38774
:1013000017FBE39F67FA0546FD564DB70545854532
:1013100071BF05487D5759BFB386A60205048307F0
:10132000F4FFBA96E206E18613F7F70F130607FDFE
:101330001376F60F63E5C500138707FDF1BF1306AB
:10134000F7F91376F60F636EC902138797FAE30570
:1013500037FDA306D100130790066385E704634BAE
:10136000F706130780056384E70A6345F702E38104
:1013700007EE1307500293055002E381E7F022863F
:10138000D9B51307F7FB1377F70FE364E9FC13876D
:1013900097FC75BF130730066386E70A13074006FC
:1013A000E39FE7FC03250A00A947A307F100930A7E
:1013B0004A00635805009307D0023305A040230775
:1013C000F1006C00EFF0AFB56C004808EFF01F883B
:1013D000568A75B713073007638EE7066341F70235
:1013E0001307F006638EE70413070007E399E7F895
:1013F0000347C100136727002306E10009A813076C
:101400005007638BE70213078007E39AE7F6938799
:1014100087FA414793B71700A307E1001397270006
:101420008347C100ED9BD98F2306F100930A4A0040
:101430006C0003250A0079B7A947A307F100FDB79F
:10144000A147E5BF83050A004808930A4A00EFF068
:101450002FB2BDBF83270A006C0048083EC8EFF0DA
:10146000EFFE1C10930A4A003EC89DB7BA97FDB321
:101470000145C5BBEF027F8C2A883685834648002C
:10148000BA8703475800A206D98E328717B60000E4
:101490001306869089E517B600001306A690BE8550
:1014A000EFF0FFD66F00BF8B9757FF1F9387C7A73B
:1014B0009C4381CFEF027F88D843B2862E8618479F
:1014C000AA853E8502976F009F8961558280EF0251
:1014D000DF868357050039712A84231EF100834774
:1014E00045009305650041461305F101230FF10006
:1014F000EF70406F9305740141461305F102EF70E0
:10150000606E8356240017B600001306E691E54589
:101510000A85EFF0DFCF6C08130630020A85EFF082
:10152000BFF821616F00BF83EF023F8139712A84C8
:101530009305050341461305D101EF70A06A930599
:10154000940841461305D102EF70C0698347E40156
:101550000347F4018356C401858B0607D98F17B65C
:1015600000001306268DE5450A85230EF100EFF0F5
:101570001FCA6C08130610020A85EFF0FFF2216102
:101580006F00EFFDEF02CFF937040001B70400FF51
:101590000111814A1759FF1F130949857D14938949
:1015A000F4FF17BA0000130A6A8DEF60BF9E63C58F
:1015B000AA0005616F000FFA8327490B13973A00C1
:1015C0003E978347370095CF5C43A30107005286BF
:1015D000B3F687008247E5454800E58FD58F3EC0CA
:1015E00083462700B3F73701858AE206D58F8356F5
:1015F00007003EC0EFF0BFC111468A854800EFF0FA
:10160000BFEA850A5DB7EF024FF301468145EFF06F
:10161000BFE96F00CFF483576500638E071A1D7111
:10162000A2CCA6CACAC886CECEC6D2C4D6C2DAC09A
:101630005EDE801013F717003289AA8431CBF99B44
:101640002313F500EF601F9906053D0541990A8BAC
:10165000C16A3301A1408A8B8149014AFD1AEF60BA
:101660007F97634CAA0C7947930604FB17A60000EA
:101670001306C67FCA852685EFF0DFDF638F090C6E
:1016800013961900DE85130504FBEFF0FFE15A8184
:1016900083D7640013F7270021CBF59B2393F40035
:1016A000EF605F9406053D0541998A8A3301A140A8
:1016B0000A8B8149014AEF60FF926345AA0A654798
:1016C000930604FB17A600001306C67ACA85268572
:1016D000EFF05FDA6387090A13961900DA851305BC
:1016E00004FBEFF07FDC568183D7640013F74700DB
:1016F00005CBED9B2393F4006547930604FB17A6E7
:10170000000013066677CA852685EFF0BFD69C4495
:1017100081C703D747003DEB130504FBEFF0BFEE95
:10172000130104FAF6406644D6444649B649264AAF
:10173000964A064BF25B25618280DC4413171A003F
:10174000BA9703D707006308570193971900DE97EC
:101750002390E7008509050A19B7130504FBEFF08C
:101760009FEA35B79C4813171A00BA9703D70700AA
:1017700019C793971900DA972390E7008509050A9E
:101780001DBF130504FBEFF01FE8B1BF2314E4FAFB
:1017900003D767008326C4FA2146520751832315D5
:1017A000E4FA370700F0758F9447930584FA130520
:1017B00004FB92069182558F2326E4FA83C77700B3
:1017C00013F707018347F4FABD9BD98FA307F4FAF7
:1017D000EFF09FCDB1B78280EF02AFD31744FF1F68
:1017E0001304C4600444797193F7F4FB1747FF1F97
:1017F0002322F76093F70404A1C78588A1E097A985
:1018000000009389A967EF60EFF863DBA4028327E8
:10181000440B139934003E998356090091CE4E86AD
:10182000E5454808EFF0BF9E4808EFF0DFDD2146B0
:1018300081454A85EF006FD38504F1B7EFF09FD45F
:101840001C4413F7F7F79746FF1F23A5E65A93F7B3
:1018500007086397071E1C4413F7F7EF9746FF1F0F
:1018600023AAE65813F707106318071E1844937746
:10187000F7DF9746FF1F23AFF6569376072095C6EE
:10188000058B630A072018408983858B3ACA034772
:10189000840715464C080607D98F17A500001305C5
:1018A000A55A230CF100EFF03FC01C4413F7F7BF1B
:1018B0009746FF1F23A0E65493F707408DC3835735
:1018C00044000D464C08231AF1008357640017A505
:1018D00000001305A557230BF100EFF0FFBC1844DF
:1018E000FD749387F47FF98F9746FF1F23A4F6506A
:1018F0009317470163DF0700EFA08FE119C98356F3
:10190000C5016391061A17A500001305A554EFF051
:101910009FCF1C447D777D177D8F9746FF1F23AB9C
:10192000E64C13973701635A0702858B6388071CBF
:10193000EFA04FDF1DC118458347E5001D463ACA99
:101940000357C5004C0817A5000013052551231C9B
:10195000E100230DF100EFF03FB51844F977FD17D2
:10196000F98F9746FF1F23A7F6489317270163D9DE
:101970000700814517050000130525CAEF50FFF247
:101980001844E177FD17F98F9746FF1F23A4F64609
:101990009317070163D30702EFA0BF982A848144FD
:1019A00017A900001309094CEF600FEE939704018B
:1019B0004205C183418163EAA71445616F00EFB816
:1019C00083A70A0093141900BE9483D7040033F749
:1019D00067011DCF1396170133F77701B3F637016F
:1019E0006352060417A600001306064409E717A66B
:1019F000000013062644E5454808EFF05F814808DB
:101A0000EFF07FC083D70400B3F747012390F400C1
:101A10000509EF602FE1AA84EF60CFDF2695E3414F
:101A2000A9FA15BD368519C7EF40A04361DDEFF077
:101A30001FAAC9BFEFD09FB371D5EFF0FFAED9B7E2
:101A400085697D7A0149974AFF1F938AEA4A056BA7
:101A5000896BFD197D1A75BF858B9DC7EF500FF3FC
:101A6000231AA10041469745FF1F9385A541130501
:101A70006101EF70201749464C0817A500001305B7
:101A8000253CEFF07FA2DDB317A500001305453B11
:101A9000EFF07FB7E1BB17A500001305E53AEFF0C3
:101AA0009FB621B50357E501C17785073E97835758
:101AB000A101FD14133717003207E58FD98F231DBD
:101AC000F100231AD100835605020357250221464F
:101AD000231BD100231CE100035745028566FD1638
:101AE000758FFD76F58FD98F4C0817A5000013056B
:101AF0006536231DF100EFF03F9B21BD17A50000C7
:101B00001305C535EFF03FB089BD5C4813F7E7FF1B
:101B100058C8858B89CFA6864A86C9450A85EFF0C5
:101B20000FEF8357040099E70A85EFF0DFAD8504D6
:101B300061049DBD231AF1008357240093054400DE
:101B400041462808231BF100EF70C00951464C089C
:101B50000A85EFF07F95E1BFEF022F9E8547339511
:101B6000A7009747FF1F938767289C47411181452E
:101B70005D8D9747FF1F23AFA7269377057085E3F9
:101B800093576500858BA1CBC167938707887D8DAF
:101B900005EDEF606FD19305803EB305B5021745A3
:101BA000FF1F1305A5352EC6EF50A03BB24519C146
:101BB0006349B50085C51745FF1F13052534EF5050
:101BC000C04441016F00AF99EF600FCE2A84EF60EF
:101BD000AFCEE360A4FCEF602FCE75BF0145EFF000
:101BE000BFBFC5B7EF026F957971AA860144174947
:101BF000FF1F1309A91F36C6EF60CFB9B246635C59
:101C0000A4028327490B93143400BE9483D70400A5
:101C10006396D70285C617A6000013062626E5455B
:101C20004808EFF0CFDE4808EFF0FF9D21468145E0
:101C30002685EF008F9345616F006F92050465BFA5
:101C400019C223200600814701C59306D00389E508
:101C50003E8582808505050583870500030705000D
:101C600099CF6394E700E397D7FE8147D5B79306F2
:101C7000D0038547E30ED7FC93371700D1BF9307F6
:101C8000F002E316F7FE854761D6050508C2C9B71D
:101C900099C123A0050081470DC11308D003130685
:101CA000F0023307F5008306070081CA6387060147
:101CB0006397C60099C1050798C13E858280850754
:101CC000CDB731C9EF02EF8441112E8A6C002A8909
:101CD000368BB28A97A400009384040EEFF05FFB6A
:101CE0002A8C0144A689B14B88406286CA85EF7070
:101CF000E01801ED0E044E945C403245DA865686BB
:101D0000D285829741016F004F840504A104E31D31
:101D100074FD6155C5BF7D55828099E5615582800E
:101D2000615505616F000F83EFF29EFF2E8A2A84B2
:101D300001118145B28452854146BA893689EFF056
:101D40006F8793150501C1811376F50FA181228557
:101D5000EF507FB12A8469D552854C08EFF05FF3CC
:101D6000524A2A8BE30E0AFA2A8697A50000938529
:101D7000E50F5285EF708010AA8A0DED7D5AEF6055
:101D80006FA563C5AA0099E8014561BF5C4413973C
:101D90001A00850ABA9723904701D5B74C442EC63E
:101DA000EF604FA3B245131615004E850299E34D1F
:101DB000A0FC85BF5A8697A500009385A50B528588
:101DC000EF70C00B0DE1032A0401EF60AFA1131601
:101DD000150081455285EFF05EF9DDD40C482EC622
:101DE000EF604FA0C1B75A8697A500009385C5083C
:101DF0005285EF70A00841E11C44A5CF81ECD4438B
:101E0000370700E0758F9447D8C33707001F758FD9
:101E100098C701BFA1463008CE854A85EFE0DF961E
:101E2000E31105F01844835781017D762312F700F2
:101E30008357A1019396470183576700D182F18FA1
:101E4000D58FF2467D767D16F182858AB206F18FB6
:101E5000D58F2313F7008347E1018356C101230582
:101E6000F7008347B7002314D700FD8BA305F700C5
:101E70004DBD7D557DB55A8697A50000938545F3E8
:101E80005285EF60B07FE31D05E81C4CE38A07E84C
:101E90009C43E38707E8CE864A86A68522858297FB
:101EA00049B5EFF29EE93687B2862E86AA850545AA
:101EB000EFF0BFE66FF0BEEAEFF23EE83687B2869B
:101EC0002E86AA850145EFF05FE56FF05EE9EFF23F
:101ED0003EE5411199C123A005009747FF1F938755
:101EE000A703804381441DC82E89AA8931141DC4CB
:101EF0000C4070004E85EFF0BFD419CD81E8A2846C
:101F0000630C0900B2472320F90039A08C40084037
:101F10000146EFF0FFD265F5404869F8268541019A
:101F20006FF05EE3184111CBEFF23EE1AE873E85E4
:101F3000B285368602976FF09EE235558280EFF2C9
:101F4000DEDF8357C50013D70501C205B387E7025B
:101F50001841C1814849BA95BE95EFF0BFFC6FF0BA
:101F60001EE0584111CBEFF25EDDAE873E85B285B3
:101F7000368602976FF0BEDE35558280184509CB54
:101F8000EFF2BEDBAE873E85B28502976FF03EDD95
:101F9000355582805C4599C7EFF23EDA2E858297EF
:101FA0006FF0FEDB35558280EFF29ED78329050066
:101FB000035AC5002A844849AE848145EFF09FFD4D
:101FC0002A890DE193D50401B38545030356C40066
:101FD0004848CE95EFF09FFA2A8909E5484885459B
:101FE000EFF05FFB4A856FF0FED6EFF27ED32A89D1
:101FF0000441035BC500484979712E848145B28A4A
:10200000368AEFF03FF941E193590401B38969033E
:10201000420441802694A29903440901330480407C
:102020003374440111CC03254901A2865686CE851E
:10203000EFF03FF3AA8431E1330A8A40A299A29AD1
:102040008144630C0A025286D6850808032449019C
:10205000EF605039834609011C089305F00F338661
:1020600046413385470136C6EFF03ED0B2461008F0
:10207000CE852285EFF0FFEEAA8403254901854530
:10208000EFF05FF1268545616FF0DECCEFF2FECA1E
:102090002E864C41A1462A84EFF03FF5AA840345E1
:1020A0000401A145EFE07F985C403385A74048C01C
:1020B00026856FF0DECA814797A600009386C6CCBE
:1020C0006393C70082803387F500034707008507C5
:1020D000398D135745003697034707001205398D90
:1020E0001375F50F13574500369703470700120580
:1020F000398D1375F50FE9B7EFF23EC42A84AA852E
:102100001D461305F00FEFF01FFB83477400338566
:10211000A7403335A0006FF09EC4EFF21EC24111FC
:10212000A1463000EFF0BFE109ED03578100C16720
:10213000FD1705456317F7002800EFF0FFFB333567
:10214000A00041016FF0BEC1EFF29EBDAE848C4194
:102150004111A1462A8903440501EFF05FDEAA89F7
:1021600039E9A1452285EFE05F8C9C400357C90007
:102170002A8AAA97939607019CC0C182098F639C03
:10218000E602C16513D70701B385B74011E7835550
:10219000E900FD15C205BE958CC0A1460A864A8598
:1021A000EFF0FFD9AA8901E90A85EFF0FFF401C930
:1021B000832749009CC04E8541016FF0BEB903578B
:1021C000C9008357210080403307474163DBE700A4
:1021D00033FA470363170A004177798C3E9480C035
:1021E000D9BF03450901A145417AEFE01F84098C5D
:1021F000AA8A80C0337A4401417B63648A008149A2
:102200005DBFA1463000A2854A85EFF05FD3AA8961
:102210005DF12800EFF05FEE11E98357A10003574D
:10222000C100337A6A0180C0BA973E9A33045441A0
:10223000E9B7EFF29EB02A84AA851D461305F00F78
:10224000EFF07FE7A303A4006FF07EB1EFF27EAC66
:102250002A84034505015D71A145EFE00FFD5C4057
:102260002A8B0355E4004179B3F727016C003EC681
:10227000EFE00FFD8355C400B247A1463008BE957C
:10228000B385654122852EC8EFF07FCBAA84634BCE
:1022900005002808EFF05FE611C9B2452285EFF08E
:1022A000BFD0AA84268561616FF03EAAC24703575A
:1022B000A101417C338B6741B3F72701BA973EC830
:1022C00010100C082285C24BEFF01FE8AA8479F9A0
:1022D0000810EFF07FE22DE95C403ECA30104C0858
:1022E00022855249EFF05FE6AA844DFD0357810233
:1022F000835701026316F7002810EFF0FFDF09C5CE
:102300005840D247E31CF7FC63902B0583574102EA
:1023100085CF83572102B3FA8B010810BE9A1C4463
:102320002311F102EFF0FFF083490401035A410247
:10233000B309304193F90902631B0A000C1022858E
:10234000EFF0DFD4AA8439FDE31C7BF7B9B74E89DF
:1023500063733A015289CA861018D6852285EFF038
:102360001FBEAA8421F1630909000C44CA86101813
:102370002285EFF09FC7AA8403450401CA85EFE0D8
:10238000CFEA1C443E9508C4E39E04F0330A2A4178
:10239000CA9A5DB7EFF2DE98411191E5FD542685AA
:1023A00041016FF03E9BC44983D725014CC904C14C
:1023B0002316F50003C705012A842317E50003C58A
:1023C000150193160701130700022308A400C18218
:1023D000E366A7FCE1D7B3E4F402E9F08547E3FF45
:1023E000D7FAA145EFE06FE4AA89014A0149835772
:1023F000C400931509012285BE95B38535412EC2CF
:10240000EFF0BFD119ED0355E4004C00050AEFE0F1
:102410002FE39245420A2285135A0A01EFF0FFCFBB
:1024200009E905098357E400420913590901E360EA
:10243000F9FC8357E40063944701D1548DB763944A
:1024400027039245A1463000B38535412285EFF040
:102450001FAF35E12800EFF03FCA11C50355E40076
:102460004C00EFE0EFDD9247C17A3387374158C027
:102470004177F98F1CC44C401C4463EEF500A14623
:1024800030002285EFF0BFAB1DE52800EFF0DFC67E
:10249000032A44001DC15C400355E4004179B3F7B1
:1024A00027014C003EC2EFE0AFD992452285EFF004
:1024B000DFC6635C0502AA84DDB512450359A1009D
:1024C000035BC10033F5AA002A9903450401DA85AC
:1024D000EFE0AFD54A9508C46314450163130B04BC
:1024E000330A3A412322440179B709C58547A30835
:1024F000F40075B54C402285EFF01FAB4DFD484010
:102500008357C40086093375A9003E9533053541CC
:1025100048C03375250108C42285EFF03FD379D533
:1025200059BF4D5549BF83471501C9CFEFF26EFE24
:102530002A840345050141112E8AA145BA893689AD
:10254000328BEFE08FCE8357C4000605898F7D550F
:1025500063E727075C4081443EC230004C0022857F
:10256000924AEFF07FBE21ED835B810063994B01BE
:102570002800EFF07FB801E58504C204C18058400F
:102580009247630BF702E3FA99FC8356C100615549
:102590009DC663E63403C175B3FABA006373D9000C
:1025A000CA868355A1005A862285D695EFF03F99B9
:1025B00019E50355C10021A06155E3884BFD410198
:1025C0006FF0AEF849558280EFF22EF70147EFF039
:1025D0009FF56FF0CEF8EFF24EF63284B2862E867B
:1025E000835545000841EFF03FFE635385002A8480
:1025F00022856FF0CEF6EFF24EF183471501397167
:10260000C954BDC7034B05012EC62A84A1455A856E
:102610003689328AEFE06FC10D473307E5028357F1
:10262000C400AA8DFD54998F63E427056304090053
:1026300063000A045C403ECA30084C082285524DB3
:10264000EFF09FB0AA8945ED835781013247639728
:10265000E7002808EFF05FAA630605105840D2474C
:10266000E31CF7FC8144631B090019A0814499E72E
:10267000268521616FF02EEDE35CA0FE5A85CA85A8
:10268000EFE0AFBA014B11C5330BB501420B135B41
:102690000B01014D7D5CC17B930C44008357E4002A
:1026A0006380A70D1C4444403307FB0063EBE40444
:1026B00032472311F1020810FD572310E1022312C3
:1026C00021032303F102EFF0DFB6630909000C4494
:1026D000CA8652862285EFF05F91AA8903450401DC
:1026E000CA85EFE08FB41C443E9508C46399090085
:1026F0000C102285EFF09F99AA89CA8435D9CE841F
:1027000085BF03450401A145EFE02FB2B387A400C4
:102710002311F1028357C400B3F474012310810321
:10272000BE94898C44C0081023120102EFF07FB0E0
:102730000C102285EFF09F95AA840355E400E685EE
:10274000EFE00FB05C40B3F777011CC4E39204F2F2
:102750002285EFF0BFAFAA84E31C05F0050D3DBF55
:10276000C15439B78357C101E30209F0E39827F157
:10277000C177034C0401B377FD00035DA101330C65
:102780008041137C0C023E9DD28ACA8CE28B63F39B
:102790008C01E68BDE861010EA852285EFF02FFA99
:1027A000AA84E31B05EC5E860C105685EF60204181
:1027B000AA84E31505ECB38C7C415E9DDE9AE39719
:1027C0000CFC7DB5EFF26ED781460146EFF0BFE21B
:1027D0006FF0EED8638C050EEFF2AED35D71054D50
:1027E00019C213BD160003590502B68B328B0509B9
:1027F0004209135909012E8A2A84CA89216C930A35
:102800008500E15C9304F9FFC204C180638F8405F5
:102810009306A0045000A6855685EFF0FFDA6357B3
:10282000050063139501A6892689E9BF9C083E959A
:10283000230A05FA4C005285EFF0AEDD75F563040E
:102840000D0883570402639597089387F4FF2310BC
:10285000F402894613060402A1655685EFF0BFD93C
:102860006358050661616FF04ECE0145E31C0DFE15
:102870000549B1675D55E387F9FE9165CE959304EF
:102880008400C205DE865A86C1812685EFF0BFD658
:10289000630D09005285EF60405DAA865286CE85A1
:1028A0002685EFF05FD5E34F05FA8357040263FFF7
:1028B000370323103403894613060402A1652685D5
:1028C000EFF07FD325A0A689014965B77D558280A9
:1028D000A6855685EFF01FEFE34605F89165FD15D7
:1028E000CA95C205C1815685EFF0DFEDE35CA0F625
:1028F00001458DBFEFF2EEC103540502916A1D71CF
:10290000050442042A89AE894180A16B130A85001F
:10291000FD1A130B05029304F4FFC204C180639DEA
:102920007405916B2164130A8900850B170C000054
:10293000130CACCA8357090293041400C204C1806B
:1029400085076383F40E5E949306A0045008A68561
:1029500052854204EFF05FC74180AA8A854613067C
:102960007100A2855285EFF03FC62A8B634750075E
:102970006347A00626847DBF56949306A0045008A2
:10298000A68552854204EFF03FC441802A8C8546DB
:1029900013067100A2855285EFF01FC3634C8003BC
:1029A000E351A0F883570902E39D97F69387F4FF5C
:1029B0002310F90289465A86A1655285EFF0BFC3FC
:1029C000A6855285EFF01FE0A2855285EFF09FDFCC
:1029D000268491B7E358A0FCA9B7634BA000A68555
:1029E0005285EFF03FDEA2855285EFF0BFDD59B78B
:1029F0009C10BE9A238A0AFA639109022C004808A7
:102A0000EFF0EFCC25D91C45224552C62318810092
:102A100074006286DA858297B1BF0146CE85480888
:102A2000EFF00FA261FDB9B7014525616FF0EEB17E
:102A3000EFF2AEB09737FF1F9387074E8043814474
:102A400009C42A893114814401E426856FF02EB12E
:102A5000631809005C4481EF404865D83114EDB734
:102A600008400146CA85EFF0AF9D6DF5F5B7829736
:102A7000E5F4AA84D5B7EFF24EAC9737FF1F9387E2
:102A8000274A8043AA8409EC2685EFF07FFAAA84BE
:102A90000144EF502FD0636CA40026856FF02EAC5C
:102AA0005C402285A6859C4382970040E9BF0504CF
:102AB0001374F40FF9BFEFF24EA80145EFF0BFFB1E
:102AC0006FF0EEA99737FF1F9387874523A0070074
:102AD00023A207008280EFF24EA69737FF1F93874D
:102AE000A74323A0070023A20700EFF0BFFD6FF06C
:102AF0000EA7EFF28EA44111130985002A84EF502E
:102B0000CFE5AA854A85EFF0FF88AA8419ED8946AA
:102B10001306E100A1654A85EFF01FABE17763443E
:102B200005008357E1002310F402268541016FF070
:102B30000EA39737FF1F9387A73E90430147B286A6
:102B400091EE05E3DC4310C11737FF1F232AA73C92
:102B500085EF9737FF1F23A7A73C828036879442D3
:102B6000C5B7144385E2DC432320050091EB97377A
:102B7000FF1F23A9A73A9737FF1F23A3A73A8280F5
:102B800088C3C1BF14C108C38280EFF20E9B173403
:102B9000FF1F130424342285EFF0BFF5AA8405E556
:102BA000179900001309492722859737FF1F23A58E
:102BB0002733EFF01FF89737FF1F23AF27319737E1
:102BC000FF1F23A3873626856FF06E999737FF1F67
:102BD00083C7C735795599EFEFF22E96EFF0BFEF27
:102BE000EFF0BFFA11E585471737FF1F2300F734D1
:102BF0006FF0EE968280EFF24E949737FF1F938727
